:020000040800F2
:10800000D0DD0020A1810008A981000805AB00088F
:10801000AD810008AF810008B181000800000000B8
:10802000000000000000000000000000B381000814
:10803000B581000800000000B7810008B981000880
:10804000BB810008BB810008BB810008BB81000820
:10805000BB810008BB810008BB810008BB81000810
:10806000BB810008BB810008BB810008BB81000800
:10807000BB810008BB810008379900083F990008C0
:10808000BB81000847990008BB810008BB8100083C
:10809000BB810008BB810008BB810008BB810008D0
:1080A000BB810008BB810008BB810008BB810008C0
:1080B00021AB0208BB810008BB810008BB8100081E
:1080C000BB810008BB810008BB810008BB810008A0
:1080D000BB81000857B702085FB7020867B70208FC
:1080E000A59D0008BB810008BB810008BB8100087A
:1080F000BB810008BB810008BB8100084F990008C4
:10810000BB810008BB810008BB810008BB8100085F
:1081100047B702084FB70208BB810008BB810008BF
:10812000BB810008BB810008BB810008BB8100083F
:10813000BB810008BB810008BB810008BB8100082F
:10814000BB810008BB810008BB810008BB8100081F
:10815000BB810008579900085F9900086FB70208B3
:10816000BB810008BB810008BB810008BB810008FF
:10817000BB810008BB810008BB810008BB810008EF
:10818000BB810008BB810008DFF810D000F058FC6C
:1081900000480047B1D50208AFF30080D0DD0020D1
:1081A0000648804706480047FEE7FEE7FEE7FEE791
:1081B000FEE7FEE7FEE7FEE7FEE7FEE7B9AA0208F4
:1081C000898100082DE9F0410024061B254671F144
:1081D000000605DA01240027D0EB070067EB010158
:1081E000161E73F1000605DA0027D2EB07020125FF
:1081F00067EB030300F0C1FA86460E4617469C461D
:10820000AC4204D00025D0EB050E65EB010624B18D
:108210000020D2EB000760EB030C704631463A4673
:108220006346BDE8F081202A06DBCB17203A41FAED
:1082300002F043EAE07306E041FA02F3D040C2F1F3
:108240002002914008431946704740EA01039B070A
:1082500003D009E008C9121F08C0042AFAD203E0BB
:1082600011F8013B00F8013B521EF9D27047421E43
:1082700012F8013F002BFBD111F8013B02F8013B42
:10828000002BF9D17047421C10F8011B0029FBD1CB
:10829000801A704730B505460020034600E05B1C9D
:1082A000934205D2EC5CC85C201A01D1002CF6D1B7
:1082B00030BD2DE9FE4F804681EA0300C00F0C4619
:1082C000009021F0004123F00045B8EB0200A941E5
:1082D00005D24046214690461C460B46024623F0F6
:1082E0000040104347D0270DC7F30A00C3F30A51DB
:1082F0000290401A019040286BDAC3F3130040F457
:10830000801B0098924620B10023D2EB030A63EB56
:108310000B0B01985946C0F14002504600F05EFA3E
:1083200006460D4650465946019AFFF77CFF10EB72
:1083300008006141002487EA115284EAE7731A4376
:1083400040D0009A62B3019A012A4FEA075215DC25
:10835000001B61EB02014FF0004202EA0752CDE937
:108360000042001C41F5801132462B4600F0EAFA2B
:1083700003B0BDE8F08F40462146F9E7001B61EBF2
:108380000201001C41F5801300185B412018A2F582
:10839000001747EB030140EAD570B6196D4111E0B3
:1083A0006D084FEA360645EAC0754FEA0752001BD2
:1083B00061EB0201001C41F5801149084FEA3000D1
:1083C0000019514132462B4603B0BDE8F04F00F092
:1083D000AABA0098012240000023D0EB020263EB0E
:1083E000E073009821464FEAE074B8EB000061EBBF
:1083F0000401E9E783F000435BE781F0004158E7BF
:108400002DE9FE4F81EA030404F0004421F000410D
:1084100000944FF0000B23F0004350EA01045ED0BB
:1084200052EA03045BD0C3F30A54C1F30A552C4447
:10843000A4F2F3340194A0FB0254C1F3130141F4FC
:108440008011C3F3130343F4801301FB024400FBC8
:10845000034E840A970A44EA815447EA8357A4FBEF
:10846000076802958D0A05FB07854FEA932C04FBEC
:108470000C542705029D4FEA065847EA1637B5EB1C
:1084800008056EEB070C870E920E47EA811742EA49
:108490008312A7FB0201B6EB0B0164EB00042B0D6A
:1084A00043EA0C335E1844EB1C50DA465146E7FBB6
:1084B0000201C5F313044FEA0B3343EA14534FEAA6
:1084C0000432019C43EA0603A4F10C040294009CCC
:1084D000CDE900B400F036FA03B0BDE8F08F00201B
:1084E0000146F9E72DE9F04D81EA030404F0004B61
:1084F00021F0004514464FF0000A23F0004150EAF5
:10850000050220D054EA01021DD0C5F30A570246E5
:10851000C5F31303C1F31300C1F30A5640F48015E9
:1085200043F48013A7EB0608101BD64608F2FD386B
:1085300073EB050002D308F1010801E092185B41DA
:10854000B8F1000F03DA00200146BDE8F08D0020ED
:108550004FF48011064684460EE0171B73EB0507A7
:1085600005D3121B63EB050306434CEA010C4908D3
:108570004FEA300092185B4150EA0107EDD152EA10
:10858000030012D082EA040083EA0501084305D003
:10859000101BAB4106D20122002306E000224FF05F
:1085A000004302E06FF0010253101AEB06004CEB9F
:1085B000085110EB0A0041EB0B01BDE8F04D00F053
:1085C000B2B9F0B4CA17CB0F50405140C61841F1B0
:1085D00000054FEAC372314628004FF0960303D0DE
:1085E000B623F0BC00F071B930460021F9E70EB5B2
:1085F000C10F80EAE0700844CA07002140F233430B
:108600008DE80E000A460B4600F09CF903B000BD51
:108610000EB540F2334102910021CDE900110A4626
:108620000B4600F08FF903B000BD3EB5CA17CB0F63
:10863000002450405140C0186141DA0740F23343F2
:108640000094CDE901232246234600F07BF903B0D4
:1086500030BD10B500F0004420F00040C20DC0F362
:10866000160040F400007F2A02DA0020014610BD07
:108670000021962A03DCC2F19602D04002E0963A2D
:1086800000F0ACF8002CF2D00023D0EB030063EB39
:10869000010110BD70B5C1F30A5201F0004500247C
:1086A000C1F3130140F2FF3341F480119A4201DA21
:1086B000002070BD40F233439A42A2F2334203DC01
:1086C000524200F09AF800E090402C43F1D0404232
:1086D00070BD70B5C1F30A5201F000450024C1F32A
:1086E000130140F2FF3341F480119A4202DA002074
:1086F000014670BD40F233439A42A2F2334203DC9A
:10870000524200F07AF801E000F068F82C43F0D013
:108710000023D0EB030063EB010170BD00F00042C9
:1087200030F000400AD0C10D01F56071C0F31600B1
:1087300042EA0151C2084007114370470020014638
:10874000704701F0004330B421F0004150EA0102CB
:1087500006D00A0DA2F56072C1F31301002A02DCF3
:1087600030BC00207047440F44EAC104C100E01847
:1087700030BC00EBC25000F09FB82DE9F05F054619
:10878000002092469B4688460646814640241BE0D0
:10879000284641464746224600F02FF853465A469F
:1087A000C01A914110D311461846224600F016F81F
:1087B0002D1A67EB01084F4622460120002100F0E8
:1087C0000DF817EB00094E41201EA4F10104DFDC77
:1087D000484631462A464346BDE8F09F202A04DB3E
:1087E000203A00FA02F1002070479140C2F12003C4
:1087F00020FA03F3194390407047202A04DB203A03
:1088000021FA02F00021704721FA02F3D040C2F1B0
:108810002002914008431946704700000FB400231E
:1088200000B589B00CA900910B996FF00042CB60A4
:108830001E4B06931E4B07930423CDE901321D4ABC
:10884000089202466B46002000F0A6F909B05DF8D8
:1088500014FB70B586B006464FF0FF300091CDE9AD
:108860000101002015460C4604903246694604A8D2
:10887000FFF7D4FF02460498211825B108B1084635
:1088800000E020462860049800280DD0002A02DD70
:108890000098884208D0081B0094CDE901043246B4
:1088A000694604A8FFF7BAFF06B070BDD18D000875
:1088B000EF8D0008658A00080029A8BF7047401C9A
:1088C000490008BF20F00100704710B4B0FA80FCE6
:1088D00000FA0CF050EA010404BF10BC704749B123
:1088E000CCF1200421FA04F411FA0CF118BF012193
:1088F00021430843A3EB0C01CB1D4FEA00614FEA73
:10890000102042BF002010BC704700EBC350104441
:108910000029A4BF10BC7047401C490008BF20F0CC
:10892000010010BC704710B5141E73F1000408DA82
:10893000401C41F1000192185B411A4301D120F023
:10894000010010BD2DE9F04D92469B4611B1B1FAE0
:1089500081F202E0B0FA80F220329046FFF73EFF4B
:1089600004460F4640EA0A0041EA0B0153465A46C4
:10897000084313D0114653EA010019D0C8F1400250
:108980005046FFF73AFF05460E46504659464246C6
:10899000FFF724FF084305D0012004E020463946B4
:1089A000BDE8F08D0020054346EAE0762C433743CE
:1089B0000A986305E40AA0EB08000022FD0A44EAD5
:1089C00047540A3002D500200146E9E70105101995
:1089D0006941DDE9084500196941BDE8F04DA2E7AC
:1089E00070B521F0004303430CD0C1F30A550024B5
:1089F000D5EB040564EB0403D617AD1AB34102DBD3
:108A00000020014670BD201841EB025170BD0000EE
:108A100030B5041E71F1000404DB4FF00044404205
:108A200064EB0101141E73F1000405DB1C464FF0DA
:108A30000043524263EB0403994208BF904230BDA9
:108A4000064C074D06E0E06840F0010394E807009B
:108A500098471034AC42F6D3FFF79AFB785B0308D3
:108A6000985B0308C0B24FF4F05100F03BBA00002D
:108A70002DE9FF4F087883B09946FF2805D0491C9F
:108A80002D2804D00024002008E000200BE0012461
:108A9000F9E700EB800003EB4000491C0B78FF2B4B
:108AA000F7D104B1404200230293147819461D46C1
:108AB0002D2C01D02B2C04D1521C2D2C13D0002492
:108AC0000294AA461478FF2C0FD00A25A3FB057840
:108AD00001FB05814FF0000C03FB0C11521CE31944
:108AE0004AEB0101EEE70124EAE7814453EA010081
:108AF00002D019F5C87F06DA03980021C0E90011F9
:108B000007B0BDE8F08F0025AE4E2F46DFF8B882E3
:108B1000184600F0FBF9CDE90001B9F1000002DAD6
:108B2000C9F1000400E004460023A74A1AEB030B36
:108B300042EB045A12E0E00707D02A463346384693
:108B40004146FFF75DFC074688462A4633461046F5
:108B50001946FFF755FC05460E466410002CEAD175
:108B6000DDE90001B9F1000F5A46534606DAFFF776
:108B7000B9FC3A464346FFF7B5FC05E0FFF740FC79
:108B80003A464346FFF73CFC029A0AB181F00041A5
:108B9000039AC2E90001B3E72DE9FF4F1F468DB0EC
:108BA000D7E901464FF0FF382E2045464FF0000927
:108BB0000B90B9696D1C0E988847396A82468847C0
:108BC0000028F6D1BAF1FF3F0AD024F4D064002E79
:108BD00011DDBAF12B0F08D0BAF12D0F0BD102E045
:108BE000404611B08DE744F48064B9696D1C0E985D
:108BF00088478246761E6946600501D52D2000E033
:108C00002B208DF8000001F1010B0DF1200809E087
:108C1000B9696D1C0E98884782460F9844F4007419
:108C2000761E0560002E02DDBAF1300FF0D00B99F0
:108C30008A453ED144F0800406E00F99681CA9F1F2
:108C4000010944F400740860B9696D1C761E0E9821
:108C5000884782463028F0D02BE00B998A4505D111
:108C6000200603D444F08004761E18E0504624F019
:108C7000B9F808B30DF11301761E44F400748B4566
:108C800008D2AAF130000BF8010B200607D5A9F194
:108C9000010003E0200602D409F101008146A0058D
:108CA00002D50F99681C0860B9696D1C0E98884739
:108CB0008246002ED1DC53E0002E51DDBAF1650F63
:108CC00002D0BAF1450F4BD1A00549D5B9696D1C49
:108CD00024F44074761E0E9888478246002E0CDDE0
:108CE0002B2804D0BAF12D0F07D144F48074B96950
:108CF0006D1C0E9888478246761EE00501D52D2111
:108D000000E02B2108F8011BCDF82C8021E00DF1AB
:108D10002901761E44F4007488450CD2AAF1300073
:108D200010F0FF0088F8000002D10B99884509D99E
:108D300008F1010806E0E00501D5244801E042F20F
:108D40000F708146B9696D1C0E98884782460F984E
:108D50000560002E04DD504624F044F80028D6D1EA
:108D6000F9690E988847FF208BF8000088F800000A
:108D70000020069007904B466A4608A906A8FFF710
:108D800077FEA00502D46FF001002AE714F0240F4B
:108D90000AD0E00714D1DDE906123868031D3B60F4
:108DA0000068C0E900120BE0DDE90601FFF7C9FC2D
:108DB0000146E00704D13868021D3A60006801608E
:108DC00028460EE7000014400000F03FF1D8FFFFF6
:108DD000426842B1016811F8013B23B1521EC0E95B
:108DE0000012184670470121C160881E7047426812
:108DF0005AB1C368016843B983688B4205D0491EE4
:108E0000521CC0E90012002070474FF0FF3070473D
:108E10002DE9F04D00231A461B1A8A4103DB00207E
:108E20000146BDE8F08DC1F30A52C1F3130141F4CC
:108E300080154FF0000BD10702D100186D41521E72
:108E40000027044640F2FF11384601EB620A3E4615
:108E50008046024600204FF48011FFF7CEFCC21975
:108E60007141BB1846EB0100B4EB030C75EB000C31
:108E700004D3E41A65EB000517460E46241908F1E1
:108E800001006D4180463428E3DDF91946EB060008
:108E9000091BA84103D24FF0FF32134601E0002224
:108EA00013461BEB070046EB0A51BDE8F04DFFF7F8
:108EB0003ABD000030B5041E71F1000404DB4FF030
:108EC0000044404264EB0101141E73F1000405DB11
:108ED0001C464FF00043524263EB04038B4208BF31
:108EE000824230BD7F2801D9002208E0064A02EB09
:108EF0005002C007127800D1120902F00F020120BF
:108F00009040084070470000385B03080EB540F2FF
:108F1000334202920022CDE900221346FFF712FDF0
:108F200003B000BD70B58C1810F8015B15F0070395
:108F300001D110F8013B2A1106D110F8012B03E0F2
:108F400010F8016B01F8016B5B1EF9D12B0705D4FA
:108F50000023521E0DD401F8013BFAE710F8013B43
:108F6000CB1A921C03E013F8015B01F8015B521E5F
:108F7000F9D5A142D8D3002070BD10B502461078B3
:108F800003E012F8014B2318D8B20B1EA1F1010423
:108F9000A1B2F6D110BD000070B5ADF5287D044634
:108FA0000D460020A790A690002604EB44004549FA
:108FB00001EBC000408AA84203DC00200DF5287DAB
:108FC00070BD0020A69077E004EB44003D4B03EB1E
:108FD000C000028A04EB440003EBC00080892844EF
:108FE00081B2394800F010F90020A79011E004EB9D
:108FF0004400344901EBC0004068BDF89C12405C5D
:1090000001A9BDF89C228854BDF89C02401C80B286
:10901000A79004EB44002B4901EBC000008ABDF887
:109020009C128842E3DC04EB4400264A02EBC000B9
:10903000008A401E81B201A8FFF79FFF23490870F4
:1090400004EB44001F4901EBC000008A401E01A947
:10905000085C1E490978884226D10020A79016E0B6
:1090600004EB4400174901EBC0004068BDF89C12B6
:10907000405C04EB4401134A02EBC1018968BDF86E
:109080009C228854BDF89C02401C80B2A79004EB3F
:1090900044000C4901EBC000008A401EBDF89C1240
:1090A0008842DDDC012089E7642024F0D9F8BDF88E
:1090B0009802401C80B2A690BDF89802062883DB77
:1090C00000207BE7A43303083C970020310A0020EE
:1090D0002DE9F043ADF5257D04460E460025002719
:1090E000A846A94604EB4400324901EBC000408A7F
:1090F000B04204DC00200DF5257DBDE8F08300259D
:1091000018E004EB44002B4901EBC0008068405D8F
:1091100004EB4401274A02EBC1014968485504EBBE
:109120004400114601EBC0004068405D0DF80500A9
:10913000681C85B204EB44001E4901EBC000008AA4
:10914000401EA842DDDC04EB44000A4602EBC000EE
:10915000008A401E81B26846FFF70FFF04EB44010E
:10916000144A02EBC101098A491E0DF801000027CB
:109170001BE004EB44000F4B03EBC000028A04EB3E
:10918000440003EBC0008089304481B2684600F09F
:109190004FF931462046FFF7FFFE012800D1AAE72C
:1091A000642024F05DF8781C87B2062FE1DB0020F4
:1091B000A1E70000A433030808B5002000901EF0CA
:1091C0002BFF0F49087000F09BF80D480078242809
:1091D00004D0272807D028280FD109E0002109480A
:1091E00080F8091D09E00121064880F8091D04E006
:1091F0000221044880F8091D00BF00BF08BD00001F
:109200002C0A0020BC2200202DE9F04106460D4624
:1092100017460024012023F0DBFD002028490880A8
:109220000DE01EF0DBFE00F0800000B10BE001203D
:1092300024F016F822480088401C21490880204864
:109240000088C828EDDB00BF1D480088C82832DA36
:1092500010211C4801F04AFC08211A4801F048FC82
:10926000E82000F031F8C5F3871000F02DF8A906CA
:10927000080E00F029F8002000F026F8002404E091
:10928000002000F021F8601C84B2042CF8DB0024DC
:1092900005E0FF2000F018F83055601C84B2BC4295
:1092A000F7DB1021074801F023FC002023F090FD9C
:1092B0000120BDE8F081002023F08AFD0020F8E7BE
:1092C0002E0A00200000024010B5044600BF022113
:1092D0000A481EF0B1FF0028F9D0214607481EF0C9
:1092E000B7FF00BF012105481EF0A6FF0028F9D0F6
:1092F00002481EF0AAFFC0B210BD000000300140BD
:1093000010B5012023F064FD00201E4908800DE007
:109310001EF064FE00F0800000B10BE0012023F09D
:109320009FFF18480088401C16490880154800888F
:10933000C828EDDB00BF13480088C8281CDA1021BC
:10934000114801F0D3FB08210F4801F0D1FB3D206B
:10935000FFF7BAFF2A20FFF7B7FF8020FFF7B4FF1F
:10936000A720FFF7B1FF1021074801F0C1FB002043
:1093700023F02EFD012010BD002023F029FD002048
:10938000F9E700002E0A00200000024070B50546F3
:109390000E460024012023F01BFD002022490880F6
:1093A0000DE01EF01BFE00F0800000B10BE001207C
:1093B00023F056FF1C480088401C1B4908801A48AF
:1093C0000088C828EDDB00BF17480088C82825DAC8
:1093D0001021164801F08AFB0821144801F088FB8F
:1093E0008420FFF771FF0020FFF76EFF0020FFF7DA
:1093F0006BFF0020FFF768FF002404E0285DFFF703
:1094000063FF601C84B2B442F8DB1021074801F00E
:109410006FFB002023F0DCFC012070BD002023F056
:10942000D7FC0020F9E700002E0A002000000240CF
:1094300070B506460C461546012023F0C9FC2946A6
:109440003046FFF7A3FF08B9002070BD00201F4978
:1094500008800DE01EF0C2FD00F0800000B10BE0BE
:10946000012023F0FDFE19480088401C17490880A0
:1094700016480088C828EDDB00BF14480088C828BB
:109480001EDA1021124801F031FB0821104801F0CA
:109490002FFB8320FFF718FFC4F38710FFF714FF9B
:1094A000A106080EFFF710FF0020FFF70DFF1021A7
:1094B000074801F01DFB002023F08AFC0120C4E7CF
:1094C000002023F085FC0020BFE700002E0A0020CA
:1094D0000000024030B502460020002304E012F8EC
:1094E000014B60405C1CE3B28B42F8DB30BD0000F6
:1094F00010B50446392024F0F5F8E0B224F012F952
:10950000C4F3072024F00EF9C4F3074024F00AF94D
:10951000200E24F007F94FF48051034801F0E8FAD7
:1095200022F068FA10BD0000000402402DE9F0416D
:1095300007460E4614463A2024F0D4F8F0B224F040
:10954000F1F8301224F0EEF84FF480510F4801F09A
:10955000CFFA19E022F04EFA05461D2D11D13846FA
:1095600000F0ACF805463B2024F0BCF84FF48051E5
:10957000064801F0BDFA2F4434B1208828442080E9
:1095800002E02846BDE8F081E4E700000004024064
:109590002DE9F04107460E4614463C2024F0A2F87F
:1095A000F0B224F0BFF8301224F0BCF84FF4805130
:1095B000104801F09DFA0CB10020208019E022F043
:1095C00019FA05461E2D11D1384600F02BF9054633
:1095D0003D2024F087F84FF48051064801F088FAC6
:1095E0002F4434B120882844208002E02846BDE87A
:1095F000F081E4E70004024010B51EF0E7FB08B17B
:1096000000F02EF8302000F0A9F810BD10B5044687
:109610002146362000F08EF810BD10B5044614B176
:10962000204600F0ABF8342000F098F810BD10B5DB
:109630000446204600F0A2F820785C2802D020786A
:109640002F2803D10021642000F008F9322000F017
:1096500085F810BD10B5682000F04CF810BD000072
:1096600010B5222024F03EF824F031F804464FF4DF
:109670008051024801F03CFA204610BD000402402F
:109680002DE9F04124F023F8044624F020F80546A3
:1096900024F01DF8064624F01AF807464FF48051CE
:1096A000054801F025FA44EA052040EA064040EA70
:1096B0000760BDE8F08100000004024070B5044678
:1096C000272024F00FF824F002F80646054646B19C
:1096D00000BF23F0FCFF2070641C701EC0B2061E89
:1096E000F7D14FF48051024801F002FA284670BDCC
:1096F0000004024010B504460C2023F0F3FF20467E
:1097000024F010F8FFF7BCFF10BD000070B5044650
:109710000A2023F0E7FF204624F004F823F0D7FFC7
:1097200005464FF48051024801F0E2F9284670BD29
:109730000004024070B505460C46284623F0D2FFCF
:10974000204623F0EFFF4FF48051034801F0D0F999
:1097500022F050F970BD00000004024010B504462C
:10976000204623F0BFFF4FF48051034801F0C0F9B9
:1097700022F040F910BD0000000402402DE9F04144
:109780000646012023F0AEFF23F0A1FF43282BDA89
:109790002B20FFF7BBFF102826DA2F2023F0A2FF93
:1097A000002023F0BFFF3220FFF7D8FF0446142C1F
:1097B0001AD1CF20FFF7AAFF0446ACB14C20FFF727
:1097C00099FF00EB042739464C2000F047F8502061
:1097D000FFF790FF00EB04273946502000F03EF8D9
:1097E0000021702000F03AF82F2023F07BFF35781D
:1097F000284623F097FF09E0761C35785C2D01D0D0
:109800002F2D00D10025284623F08CFF002DF3D109
:109810004FF48051024801F06BF9BDE8F08100007F
:109820000004024070B504462D2023F05BFF23F0B6
:109830004EFF0646054646B100BF207823F072FF72
:10984000641C701EC0B2061EF7D14FF4805102484E
:1098500001F04EF9284670BD0004024070B505467F
:109860000C460D2023F03EFF284623F05BFFE0B2BC
:1098700023F058FFC4F3072023F054FFC4F307403C
:1098800023F050FF200E23F04DFF4FF4805102488B
:1098900001F02EF970BD00000004024070B50246D0
:1098A0000C46FF25FF2309E012F8010B80EA0501B1
:1098B0000648405C80EA03050548435C201EA4F18D
:1098C0000106B4B2F0D145EA032070BD0C310308A3
:1098D0000C3203082DE9F04103460C4600200146F6
:1098E000024606E013F8010B411842F10002601E27
:1098F00084B2002CF6DC080C40EA024C100C8DB24D
:109900001CEB050140F10002080C40EA024041183E
:109910006FEA010080B2BDE8F08130B50246002058
:10992000002305E012F8015B2C18E0B25C1CE3B2E6
:109930008B42F7DB30BD10B515F040F810BD10B507
:1099400014F0DAFF10BD10B514F0A6FF10BD10B56D
:1099500015F002F810BD10B516F096FF10BD10B549
:109960001DF0B0FD10BD00000246094B9A4201D225
:10997000084801E00648103801F000531BB1064BBF
:109980000B40C36002E0044B0B4083607047000053
:1099900010640240006002407D0F7D0F21B102681B
:1099A00042F00102026003E0026822F0010202605C
:1099B00070470000016821F0010101600021016091
:1099C00041608160C1600161212141614A49884251
:1099D00004D13D21484A103A91608CE04649183143
:1099E000884205D14FF47461434A103A916082E095
:1099F00041493031884205D14FF474113E4A103A42
:109A0000916078E03C494831884205D14FF074615B
:109A1000394A103A91606EE037496031884204D18A
:109A20003649354A103AD16065E033497831884289
:109A300004D13349304A103AD1605CE02E4990316C
:109A4000884204D12F492C4A103AD16053E02A4968
:109A5000A831884205D14FF03D51274A103AD160D4
:109A600049E02949884204D13D21274A083A11603A
:109A700041E025491831884205D14FF47461224AEA
:109A8000083A116037E020493031884205D14FF45F
:109A900074111D4A083A11602DE01B494831884273
:109AA00005D14FF07461184A083A116023E0164955
:109AB0006031884204D11149134A121F11601AE023
:109AC00011497831884204D10D490F4A121F1160A3
:109AD00011E00D499031884204D10A490A4A121F07
:109AE000116008E00849A831884204D14FF03D5187
:109AF000054A121F11607047106002403D000020AF
:109B0000400F002000003D201064024010B501F01D
:109B100080034BB122B1436943F08003436103E00A
:109B2000436923F08003436180290BD02AB1036885
:109B300001F01E042343036004E0036801F01E04E7
:109B4000A343036010BD000010B500220268134B50
:109B50001A40CC680B6823434C6923438C69234328
:109B6000CC6923430C6A23434C6A23438C6A234306
:109B70004C6B23438C6B23431A430260426922F0EF
:109B80000702D1E90B3423431A4342610B69436056
:109B90004B6883608B68C36010BD00003F801CF081
:109BA0001CB50024012120201EF01CF9302000905B
:109BB00001208DF8040000208DF8060003208DF8A8
:109BC000050000208DF807006946174800F01AFFCD
:109BD0003021154800F08CFF0021144880F834161D
:109BE00000201349887001204870C8704FF4FA7043
:109BF000886000F021F80F4890F80C0F592811DD0B
:109C000024200A49F4394871082008713020C870AE
:109C100014208870202048700021064880F80C1F0E
:109C200000F04EF81CBD000000140240BC320020C1
:109C3000F0380020BC2200201CB523F019FCD020F5
:109C400023F0E2FB23F048FC002023F0DDFB23F0AF
:109C500043FC23F00DFCD12023F0D6FB23F03CFC89
:109C600000240EE0062C05DA012023F09DFB0DF800
:109C7000040004E0002023F097FB0DF80400601CB2
:109C8000C4B2072CEEDB23F00DFC9DF806000A4958
:109C900048719DF8050008719DF80400C8709DF892
:109CA000020088709DF8010048709DF8001003487C
:109CB00080F80C1F1CBD0000C8310020BC22002011
:109CC0001CB500241B4890F80C0F8DF800001A48B2
:109CD00040788DF80100184880788DF80200012046
:109CE0008DF803001448C0788DF8040012480079FC
:109CF0008DF80500104840798DF8060023F0B8FB78
:109D0000D02023F081FB23F0E7FB002023F07CFB35
:109D100023F0E2FB00BF07E01DF8040023F074FB12
:109D200023F0DAFB601CC4B2072CF5DB23F0BAFB8E
:109D30001CBD0000BC220020C831002070B50246C6
:109D40000C460025002309E012F8010B80EA05010A
:109D50000648405C80EA03050548435C201EA4F1E8
:109D60000106B4B2F0D145EA032070BD0C310308FE
:109D70000C32030810B504460B460021072A00DD0B
:109D8000072244EA042001462BB901FA02F081B20D
:109D90000912084610BD012B02D11141C8B2F9E7E2
:109DA00000BFF7E710B51DF073FE10BD0149086054
:109DB00070470000143C0140014600200022074B80
:109DC0001B6803EA0102054B14331B680B4013B1F7
:109DD0000AB1012000E0002070470000003C014073
:109DE000002123498279002A3AD00A461268036882
:109DF0009A430B461A600A1D126803689A430B1DAA
:109E00001A60027911440A6803681A430A60184A02
:109E10000832126803689A43154B08331A601A1DFA
:109E2000126803689A43124B0C331A604279102A65
:109E30000ED11A1F126803681A430D4B08331A60BB
:109E40001A1D126803681A43094B0C331A600DE09F
:109E50000749427911440A6803681A430A6005E019
:109E6000027911440A6803689A430A607047000047
:109E7000003C014010B504460B460021072A00DDD6
:109E8000072244EA0420014613B91141C8B210BDAB
:109E9000012B05D101FA02F081B209120846F6E75A
:109EA00000BFF4E7F0B5ADF21C5D04460D4600209E
:109EB000CDF81805CDF81405002604EB44005849E8
:109EC00001EBC000408AA84203DC00200DF21C5DBB
:109ED000F0BD0020CDF814059AE051480122C16878
:109EE000504800F0A9FA4E48406800788DF800000C
:109EF0009DF8000038287DD104EB4400484B03EB6B
:109F0000C000C06804EB4403454F07EBC3031B8A42
:109F100003FB050104EB44003B4603EBC000028A4F
:109F2000404800F089FA0020CDF8180512E004EB53
:109F300044003B4901EBC0004068BDF81815405C87
:109F4000BDF818250DF80200BDF81805401C80B2B8
:109F5000CDF8180504EB4400314901EBC000008A3C
:109F6000BDF818158842E2DC04EB44002C4A02EBF1
:109F7000C000008A401E81B2684600F023FB0646FE
:109F800004EB4400264901EBC000008A401E1DF886
:109F90000000B04233D10020CDF8180520E004EBDA
:109FA00044001F4901EBC0004068BDF81815415C32
:109FB00004EB44001A4A02EBC0008068BDF8182583
:109FC000024404EB4400164B03EBC000008A401E21
:109FD00068431154BDF81805401C80B2CDF818052F
:109FE00004EB44000E4901EBC000008A401EBDF89E
:109FF000181500E003E08842D1DC012066E7642008
:10A0000023F02EF9BDF81405401C80B2CDF81405DC
:10A01000BDF814050628FFF660AF002056E70000E3
:10A02000F8E102088C6900202DE9F041ADF5A36D3F
:10A0300004460E4600250027A8460020009004EBA9
:10A040004400494901EBC000408AB04204DC0020D2
:10A050000DF5A36DBDE8F0814448807B002878D1E0
:10A0600000210846FFF71EFF01287AD1002520E0D5
:10A0700004EB44003C4901EBC0008068411904EB4B
:10A080004400394A02EBC000008A401E7043085C5D
:10A0900004EB440102EBC1014968485504EB44005C
:10A0A000114601EBC0004068405D01A94855681C9D
:10A0B00085B204EB44002C4901EBC000008AA842A1
:10A0C000D6DC00274BE004EB4400274B03EBC00039
:10A0D000C06804EB4403DFF890C00CEBC3031B8A99
:10A0E00003FB060104EB4400634603EBC000008A57
:10A0F000401E82B21E4800F021FA04EB44001A4AC6
:10A1000002EBC000008A401E81B201A800F05AFA9A
:10A11000009004EB4400144A02EBC000C06804EB5A
:10A120004402114B03EBC202128A104404EB4402B6
:10A1300003EBC202128A02FB0600411E012268469E
:10A1400000F0FCF931462046FFF7ACFE012801D1B2
:10A150007EE706E0642023F083F8781C87B2062FA0
:10A16000B1DB002074E70000F8E10208BC12002017
:10A170008C690020F0B5ADF21C5D002500240020A4
:10A180000190002600210120FFF78CFE4B4890F83B
:10A19000FC6C00204A49088080E000256FE0002424
:10A1A00014E04748008800EB4000464951F8300071
:10A1B000005D4349098801EB4101424A02EBC101BC
:10A1C0004968085502A90855601C84B23C480088BB
:10A1D00000EB40003B4901EBC000008A401EA0425A
:10A1E000DFDC3748008800EB40000A4602EBC00085
:10A1F000008A401E81B202A800F0E4F901903048C4
:10A20000008800EB40002F4B03EBC000C0682C4BD4
:10A210001B8803EB43032B4F07EBC3031B8A03FB92
:10A2200005012748008800EB40003B4603EBC000D7
:10A23000008A401E82B2244800F080F9204800883D
:10A2400000EB40003A4602EBC000C0681C4A12888E
:10A2500002EB42023B4603EBC202128A1044184A48
:10A26000128802EB420203EBC202128A02FB0500D3
:10A27000411E012201A800F061F9681C85B2104856
:10A28000008800EB40000F4901EBC000408AA84263
:10A2900085DC0B480088401C094908800848008874
:10A2A0000D28FFF67AAF054880F8FC6C00210120EC
:10A2B000FFF7BAFE0DF21C5DF0BD0000BC220020CD
:10A2C00010000020F8E102088C6900201CB5012173
:10A2D00008461DF087FD01208DF8040002208DF84E
:10A2E000050000208DF8060001208DF807001820D9
:10A2F00000906946144800F085FB0522114612487B
:10A3000000F0C8FB052206210F4800F0C3FB052220
:10A3100007210D4800F0BEFBA020009002208DF820
:10A32000040003208DF8050000208DF806008DF84C
:10A3300007006946044800F065FB4020009069462C
:10A34000014800F05FFB1CBD000002402DE9F8430E
:10A35000002400250027002000908046FFF7B6FF6C
:10A3600000F0BCF80A2022F07BFF6E4608212D4841
:10A3700000F0BCFB10212B4800F0BAFB062000F0D7
:10A3800091F80821274800F0B3FB0821254800F088
:10A39000ADFB1021234800F0ABFB012000F082F858
:10A3A000002000F07FF808211E4800F0A1FB1E48A5
:10A3B000D0F82C11B0F83021B0F8320102FB0010B7
:10A3C000B0F5003F02D900BE00BFFEE717480068A5
:10A3D00008B9FFF7CFFE00201549088017E00024D8
:10A3E00006E0134908782146FFF75CFD601C84B243
:10A3F0000F48008800EB40000B4901EBC000408A89
:10A40000A042EEDC0A480088401C09490880084840
:10A4100000880D28E3DB0748D0F80C020549C87313
:10A42000BDE8F88300000240F8E102081C02434244
:10A4300010000020BC1200202DE9F04105460C461A
:10A4400016460027012022F0C0FC0821144800F025
:10A450004DFB1021124800F04BFB032000F022F8C6
:10A46000C4F3074000F01EF8C4F3072000F01AF808
:10A47000E0B200F017F800BF06E0002000F012F88C
:10A4800028706D1C781C87B2B742F6DB082104489F
:10A4900000F02EFB002022F098FCBDE8F0810000C7
:10A4A0000000024010B5044600BF02210A481DF01A
:10A4B000C3FE0028F9D0214607481DF0C9FE00BFA1
:10A4C000012105481DF0B8FE0028F9D002481DF012
:10A4D000BCFEC0B210BD00000030014000B585B028
:10A4E000012108031DF0CEFC13481DF079FE002069
:10A4F000ADF80000ADF80400ADF80600ADF80800B6
:10A500004FF40070ADF80A000820ADF80C000020F0
:10A51000ADF80E000720ADF810004FF48270ADF8D2
:10A520000200694604481DF095FE012102481DF015
:10A530004BFE05B000BD0000003001402DE9F041A8
:10A5400005460C4616460027012022F03EFC082155
:10A550001B4800F0CBFA1021194800F0C9FA062078
:10A56000FFF7A0FF0821164800F0C2FA082114489E
:10A5700000F0BCFA1021124800F0BAFA0220FFF7EE
:10A5800091FFC4F30740FFF78DFFC4F30720FFF7E7
:10A5900089FFE0B2FFF786FF00BF05E02878FFF7EC
:10A5A00081FF6D1C781C87B2B742F7DB0821044895
:10A5B00000F09EFA002022F008FCBDE8F0810000C7
:10A5C0000000024010B50246107803E012F8014B7B
:10A5D0002318D8B20B1EA1F10104A1B2F6D110BD0F
:10A5E0002C48807F012854D100212A4881772A48AD
:10A5F0000078C0B901202849087028480068C000C8
:10A600002749D1F8301240EA81002549D1F82C12AF
:10A6100040EA41002249D1F8281208430F21814322
:10A620002048017017E000201B4908701B48006893
:10A63000C0001B49D1F8301240EA81001849D1F816
:10A640002C1240EA41001649D1F8281208430F2184
:10A6500081431548017013480078134909788842EE
:10A6600017D1104800781149087008460078104941
:10A67000097888420DD00D480078064908760B48C5
:10A6800000780B4908700948007810B10120014991
:10A69000C8757047BC120020DE0A00203402424216
:10A6A00000004242DF0A0020E00A0020E10A002008
:10A6B000DD0A002010B5ADF57C7D00247DA000688A
:10A6C000FB9000200090FEF797FF14287CD17A4879
:10A6D000FEF7ADFF7949087008460078142874D158
:10A6E000FEF7B8FF0021764A03C2BDF80000FEF76E
:10A6F000FFFE6A464FF4FA7101A8FEF717FF71A139
:10A7000001A822F08BFF714908800846008810B329
:10A7100000BF04E000216E480155601C84B2282C63
:10A72000F8DB01A9694A128888186AA122F076FF2D
:10A7300069490880002409E064480088C01C20445E
:10A7400001A9095C62480155601C84B26248008816
:10A75000001FA042F0DC61A101A822F05FFF5B496D
:10A7600008800846008820B3002405E000215848EE
:10A7700028300155601C84B2282CF7DB01A9534A0C
:10A780001288881853A122F049FF534908800024F9
:10A790000AE04E4800880830204401A9095C4C4872
:10A7A00028300155601C84B24B4800880938A0420B
:10A7B000EFDC4DA101A822F031FF44490880084692
:10A7C000008830B3002407E06BE05BE000214048E4
:10A7D00050300155601C84B2142CF7DB01A93B4AB0
:10A7E000128888183BA122F019FF3B4908800024F9
:10A7F0000AE0364800880C30204401A9095C34483E
:10A8000050300155601C84B2334800880D38A04296
:10A81000EFDC39A101A822F001FF2C49088008468D
:10A82000008820B3002405E0002029494639085556
:10A83000601C84B2322CF7DB01A9244A12888818E4
:10A8400024A122F0EBFE2449088000240AE01F48DE
:10A850000088801D204401A9085C1D49463908551F
:10A86000601C84B21C480088C01FA042EFDC00219D
:10A870000320FFF7D9FB0120FEF7C8FE01200DF5EC
:10A880007C7D10BD0D480078422803D10A48FEF7B0
:10A89000C4FE0CE00120FEF7B9FE00200749087055
:10A8A00005E00021164880F80B1F22F04BFE00BF88
:10A8B000E5E700000D0A0000480A0020380A0020E1
:10A8C000400A002041504E3D000000005E0A00207A
:10A8D000D03900203B0000005C0A0020574946495F
:10A8E0004E414D453D0000005749464950415353A4
:10A8F000574F52443D0000005345525645523D00CB
:10A90000BC22002010B504463548844208D10121FC
:10A9100008461DF077FA002101201DF073FA5EE071
:10A920003048844208D1012102201DF06BFA002139
:10A9300002201DF067FA52E02B48844208D1012121
:10A9400004201DF05FFA002104201DF05BFA46E0B0
:10A950002648844208D1012108201DF053FA002125
:10A9600008201DF04FFA3AE02148844208D1012125
:10A9700010201DF047FA002110201DF043FA2EE0B0
:10A980001C48844208D1012120201DF03BFA0021FF
:10A9900020201DF037FA22E01748844208D1012117
:10A9A00040201DF02FFA002140201DF02BFA16E068
:10A9B0001248844208D1012180201DF023FA002191
:10A9C00080201DF01FFA0AE00D48844207D10121C2
:10A9D00080151DF017FA0021A0151DF013FA10BD07
:10A9E000000002400004024000080240000C024047
:10A9F000001002400014024000180240001C0240F7
:10AA000000200240F0B50A4600210023002400BFC8
:10AA10003DE0012505FA01F3156805EA03049C42AF
:10AA200034D105684F000326BE40B5430560157953
:10AA30004E00B5400668354305601579012D02D0FA
:10AA40001579022D16D185684F000326BE40B54307
:10AA5000856055794E00B540866835438560456808
:10AA600001268E40B5434560456896798E40B6B262
:10AA700035434560C5684F000326BE40B543C560F9
:10AA8000D5794E00B540C6683543C560491C1029CC
:10AA9000BFD3F0BDF0B5002300244D07ED0E02FA40
:10AAA00005F3CE1000F1200555F826504E07F70E9D
:10AAB0000F26BE40B543CF1000F1200646F82750C0
:10AAC000CE1000F1200555F8265045EA0304CE10BB
:10AAD00000F1200545F82640F0BD0246002013692C
:10AAE0000B400BB1012000E000207047418370470C
:10AAF000018370470249087E0021014A11767047A0
:10AB0000BC1200200E48006800F0010000B100BE39
:10AB1000012080F3138800BF00BFBFF34F8F0848A8
:10AB2000E438006800F4E06006490843001D044969
:10AB3000E4390860BFF34F8F00BF00BFFEE700009D
:10AB4000F0ED00E00000FA054AF6AA20014908608D
:10AB5000704700000030004030B50246002400235A
:10AB600005E012F8015B2819C4B2581CC3B28B422D
:10AB7000F7DB6042C0B230BD10B5002422F0E2FC29
:10AB8000642022F06DFB10BD2DE9F043ADF2DC7DB9
:10AB900080460E46144699460025002783A000688B
:10ABA000CDF8D80700200190042C7CDC8048007987
:10ABB000302101EB101004EBC40101EB04117D4ABC
:10ABC000114408717A48007900F00F00303004EB2E
:10ABD000C40101EB0411114448717548C07830215B
:10ABE00001EB101004EBC40101EB04111144887156
:10ABF0006F48C07800F00F00303004EBC40101EB67
:10AC000004111144C871FEF7F7FC14287ED16A487C
:10AC10000078142809D004EBC40101EB0411654A43
:10AC20008818FEF704FD644908706348007814280A
:10AC30006DD1B6F57A7F01DD4FF47A76FEF70AFD25
:10AC400000215E4A03C25D480068FEF751FC584887
:10AC5000C078302101EB10108DF808005448C078FE
:10AC600000F00F0030308DF809005148807801EB7A
:10AC700010108DF80A004E48807800F00F00303038
:10AC80008DF80B004A48407801EB10108DF80C004D
:10AC90004748407800F00F0030308DF80D004848EC
:10ACA00090F80C0F00E07CE001EB10108DF80E0026
:10ACB000434890F80C0F00F00F0030308DF80F0073
:10ACC000B9F1000F03D154208DF8100005E0B9F15F
:10ACD000010F02D152208DF810003A208DF811009A
:10ACE00000252CE0284605EBD071491018F801101A
:10ACF0000F110A2097FBF0F0C0EBC00107F1300004
:10AD00000844C1B202AA05F10A0001E043E02EE0C6
:10AD10001154284605EBD071491018F8011001F0C4
:10AD20000F070A2097FBF0F0C0EBC00107F13000DD
:10AD30000844C1B205F10B001154A81C85B2B5EB53
:10AD4000460FCFDB0A2000EB460081B201AA02A821
:10AD5000FEF71EFC01AA02210DF5FB60FEF718FCB0
:10AD60000120FEF753FC00201349087019E0124837
:10AD70000078422808D104EBC40101EB04110D4A0C
:10AD80008818FEF74AFC0CE00120FEF73FFC00208B
:10AD90000949087005E00021094880F80B1F22F0DE
:10ADA000D1FB0DF2DC7DBDE8F08300000D0A000050
:10ADB000C8310020600A0020380A0020400A002024
:10ADC000BC22002070B5B8B0002137913691359182
:10ADD0003491339132913191309100222E922F9201
:10ADE0002C922D922B912A9129912891279126918D
:10ADF0002591249123911591149113911291119100
:10AE000010910F919FEDFE0A8DED0E0AFDA006C870
:10AE1000CDE90C12FDA006C8CDE90A12BAE0FD4842
:10AE2000807858B30020FB498870FB48B0F8700662
:10AE3000FA490968C1F57A7188421FD1F74800685C
:10AE4000C0F57A7081B2F448A0F868160021F34882
:10AE5000001FFEF7A3FDF249F048001FFEF784FD36
:10AE60000120F04908704FF47A70EC498C39C1F830
:10AE70008C000121E948001FFEF790FDE548807B2A
:10AE800050B30021E3488173E7484088E3498C3997
:10AE9000496CC1F57A7188421ED1E0488C38406C0B
:10AEA000C0F57A70E049083948800021DB484C3809
:10AEB000FEF774FDDD49D9484C38FEF755FD0120F9
:10AEC000DB4908704FF47A70D4498C394864012109
:10AED000D2484C38FEF762FDCE48807E50B3002148
:10AEE000CC488176D0488088CC498C394969C1F5F5
:10AEF0007A7188421ED1C9488C384069C0F57A7091
:10AF0000C949083988800021C4487C38FEF746FDCD
:10AF1000C849C2487C38FEF727FD0120C6490870A1
:10AF20004FF47A70BD498C3948610121BB487C38A7
:10AF3000FEF734FDB74890F8260058B30021B54815
:10AF400080F82610B848C088B4498C39C96AC1F560
:10AF50007A7188421ED1B1488C38C06AC0F57A70C7
:10AF6000B1490839C8800021AC486438FEF716FDA5
:10AF7000B249AA486438FEF7F7FC0120B0490870CE
:10AF80004FF47A70A5498C39C8620121A34864380E
:10AF9000FEF704FD9F488178807B01449D48807EB8
:10AFA00001449C4890F82600084400287FF437AFFD
:10AFB0000CF08BBE9B48007820B1002099490870A6
:10AFC0002B9019E09A48007828B100209849087021
:10AFD00001202B9010E09848007828B10020964975
:10AFE000087002202B9007E09548007820B10020DF
:10AFF0009349087003202B909DF8AC1001EB4100A1
:10B00000C0EBC1108F4911F83000C12836D19DF82E
:10B01000AC1001EB4100C0EBC1108A4901EBC0004C
:10B02000807808282AD101217B4880F8C0169DF835
:10B03000AC0030B101280AD002280ED0032818D164
:10B0400011E04FF480418048FFF750FD11E04FF4CC
:10B0500000517D48FFF74AFD0BE04FF480517A48DC
:10B06000FFF744FD05E04FF400617748FFF73EFD30
:10B0700000BF00BF00207549086099E765480C389B
:10B080009DF8AC1010F811000121B1EBD01F4CF06D
:10B0900075846F4890F80B0FB8B1634908399DF873
:10B0A000AC0031F8101009919DF8AC0000EB4001A4
:10B0B000C1EBC011634800EBC101012308919DF869
:10B0C000AC20DDE90801FFF75FFD9DF8AC1001EB56
:10B0D000410000EB01105F4901EB001081792A91DA
:10B0E0009DF8A80009288CF01384DFE810F01164A3
:10B0F00009006E15B427BD36EB38F93C514865554B
:10B100009DF8AC0000EB4001C1EBC0104D4901EBD4
:10B11000C000417808460991002113F0DBFAC1B262
:10B120002691002134911CE09DF8AC0000EB400119
:10B1300001EB0010474901EB00113031BDF8D000A0
:10B1400001EB001041789DF89800814204D1BDF8D0
:10B15000D000C1B2269112E0BDF8D000401C81B2EF
:10B1600034919DF8AC1001EB410000EB011039491E
:10B1700001EB0010C179BDF8D0008142D4DC00BFE2
:10B180009DF8AC0000EB4001C1EBC0102D4901EB74
:10B19000C000807800F0F000A0280DD19DF8AC1020
:10B1A00001EB4100C0EBC110264901EBC0008078E3
:10B1B00000F00F0127910AE09DF8AC1001EB41006F
:10B1C000C0EBC1101F4901EBC00081782791BDF889
:10B1D0009C0008B9102127919DF8AC1001EB4100AB
:10B1E000C0EBC110174901EBC001BDF89C00401C29
:10B1F000095C2491BDF89C00401C81B209912BE0B0
:10B200000000000001693230313030000169323015
:10B2100045303000D83D0020BC6200208C600240E8
:10B2200000880020120000202C69002000802010DF
:10B23000130000202080001014000020008800105F
:10B2400015000020A4770020001802408802424226
:10B25000BC220020044000209DF8AC0000EB40011F
:10B26000C1EBC011FE4800EBC1010891DDE9080106
:10B2700013F0C0FE35909DF8AC0000EB4001C1EB2F
:10B28000C010F74901EBC001BDF89C00801C095CAF
:10B29000BDF8D400814242F096849DF8AC0000EBEA
:10B2A0004001C1EBC010EE4901EBC000407800281E
:10B2B00042F389849DF8AC0000EB4001C1EBC01063
:10B2C000E74901EBC001BDF89C00C01C0A5C9DF879
:10B2D000AC0040F2231110FB01F0E24901EBC00188
:10B2E00018319DF8980000EBC00001EB001080F8C9
:10B2F0003C200021DC4A9DF8AC0002EB00129DF8D6
:10B3000098001154D94890F82800012840D19DF8A0
:10B31000AC0000EB400101EB0010D54901EB00103F
:10B3200030309DF8981000EB0110801C09900078D7
:10B3300020F08000803009990870BDF89000B62890
:10B3400014D0C52819D0D52802D0D9281CD106E0A0
:10B35000BDF89C00032801DA0021249117E0BDF814
:10B360009C00032801DA0021249110E0BDF89C0024
:10B37000032801DA0021249109E0BDF89C0003288C
:10B3800001DA0021249102E00021249100BF00BFD6
:10B39000BDF89000C52801F08A8418DCB5287CD05F
:10B3A0000DDC112802F0A082122802F0DF8213289F
:10B3B00002F06883B22842F0058401F044BCB6284C
:10B3C00001F01083B92869D0C328F4D1FEE3D9284D
:10B3D00065D007DCCA287CD0CE2802F09681D5281B
:10B3E000E9D109E0E12802F0A381E52802F0BE815D
:10B3F000E728E0D102F061BA9DF8AC1001EB410002
:10B40000C0EBC110964901EBC000C178994880F8A3
:10B41000021D9DF8AC1040F2231011FB00F0914981
:10B4200001EBC00118319DF8980000EBC00001EB62
:10B43000001001789DF8AC0040F2231210FB02F0DE
:10B44000884A02EBC000407981427DDA9DF8AC1059
:10B4500001EB410000EB0110854901EB0010303099
:10B460009DF8981000EB0110801C0990814890F81D
:10B47000020D0121A1EBD0100999097860F30001B8
:10B48000099801707B4890F8020DC0F34010E0BBB2
:10B490009DF8AC0000EB400102E0FDE3FDE3FDE3BD
:10B4A00001EB0010724901EB001030309DF898104C
:10B4B00000EB01108078C0F3401030B39DF8AC0071
:10B4C00000EB400101EB0010694901EB0010303046
:10B4D00000E0FDE39DF8981000EB0110801C09903E
:10B4E000007820F00200801C099908709DF8AC10CB
:10B4F00040F2231011FB00F0114601EBC0001830A0
:10B500009DF8981001EBC10100E00EE000EB011086
:10B5100018300990007820F00200801C099908700A
:10B520009DF8AC100220FEF77FFD00219DF8AC00D5
:10B5300040F2231210FB02F04A4A02EBC0000171F4
:10B5400002229DF8AC0000E021E040F2231110FB44
:10B5500001F0444901EBC00118319DF8980000EB5F
:10B56000C00001EB00100270B6229DF8AC0040F262
:10B57000231110FB01F03B4901EBC00018309DF88E
:10B58000981001EBC10100EB01104271FEE3394854
:10B5900090F8020DC0F3C00090B9E5229DF8AC0010
:10B5A00040F2231110FB01F02E4901EBC0001830CE
:10B5B0009DF8981001EBC10100EB01104271E5E329
:10B5C0009DF8AC1001EB410000EB0110284901EBA4
:10B5D000001030309DF8981000EB0110801C09908D
:10B5E000244890F8020D0121A1EBD01209980078AF
:10B5F00062F30000099908709DF8AC1001EB41005E
:10B6000000EB01101A4901EB001030309DF8981042
:10B6100000EB0110801C0990164890F8020D4209B9
:10B620000998007862F34100099908709DF8AC0010
:10B6300000EB400101EB00100D4901EB0010303030
:10B640009DF8981000EB01108078C0F340029DF83F
:10B65000AC0040F2231110FB01F002490CE00000A5
:10B66000A4770020C4440020383E0020BC120020F3
:10B6700004400020BC22002001EBC00018309DF8DF
:10B68000981001EBC10100EB0110007EC0F34000F7
:10B69000824277D09DF8AC1040F2231011FB00F0ED
:10B6A000FE4901EBC00018309DF8981001EBC10174
:10B6B00000EB0110183009909DF8AC0000EB400140
:10B6C00001EB0010F64901EB001030309DF89810A6
:10B6D00000EB0110807842080998007862F341007D
:10B6E000099908709DF8AC1001EB410000EB0110C6
:10B6F000EB4901EB001030309DF8981000EB011081
:10B700008078C0F34000E0B3D9229DF8AC0040F24D
:10B71000231110FB01F0E14901EBC00018309DF846
:10B72000981001EBC10100EB01104271DD4890F867
:10B73000900700287BD19DF8AC0040F2231110FB4C
:10B7400001F0D64901EBC00018309DF8981001EBCC
:10B75000C10100EB011090F87E00002867D0112392
:10B760009DF8AC0040F2231110FB01F0CB4901EB36
:10B77000C00118319DF8980000EBC00001EB0010EB
:10B7800001E055E043E190F87F0040F2231110FB07
:10B7900001F0C24901EBC00118319DF8AC0040F244
:10B7A000231210FB02F0BD4A02EBC00218329DF8D2
:10B7B000980000EBC00002EB001090F8800000EB56
:10B7C000C00001EB001080F87730F3239DF8AC0047
:10B7D00040F2231110FB01F0B04901EBC001183118
:10B7E0009DF8980000EBC00001EB001090F87F007E
:10B7F00040F2231110FB01F0A84901EBC001183100
:10B800009DF8AC0040F2231210FB02F0A34A02EBB9
:10B81000C00018309DF8982002EBC20200EB021025
:10B8200090F8800000EBC00001EB00104371E9E0EC
:10B8300001229DF8AC0040F2231110FB01F0974962
:10B8400001EBC00118319DF8980000EBC00001EB3E
:10B8500000104273D9229DF8AC0040F2231110FB76
:10B8600001F08E4901EBC00118319DF8980000EB02
:10B87000C00001EB0010427101229DF8AC0040F2C3
:10B88000231110FB01F0854901EBC00018309DF831
:10B89000981001EBC10100EB011080F83E208148B7
:10B8A00090F89007E8BB9DF8AC0040F2231110FB24
:10B8B00001F07A4901EBC00018309DF8981001EBB7
:10B8C000C10100EB011090F87E0050B39DF8AC1060
:10B8D00040F2231011FB00F0704901EBC001183158
:10B8E0009DF8980000EBC00001EB001090F87F106D
:10B8F00001EB410000EB0110694901EB001130310F
:10B900009DF8AC0040F2231210FB02F0634A02EBF8
:10B91000C00218329DF8980000EBC00002EB001046
:10B9200000E06FE090F8800001EB0010801C0990AF
:10B93000007820F004020998027000239DF8AC0002
:10B9400040F2231110FB01F0544901EBC000183004
:10B950009DF8981001EBC10100EB011090F87F00F9
:10B9600040F2231110FB01F04C4901EBC0001830EC
:10B970009DF8AC1040F2231211FB02F1474A02EB92
:10B98000C10218329DF8981001EBC10102EB0111C0
:10B9900091F8801001EBC10100EB011080F87730C5
:10B9A000F3239DF8AC0040F2231110FB01F03B495A
:10B9B00001EBC00018309DF8981001EBC10100EBBD
:10B9C000011090F87F0040F2231110FB01F0334981
:10B9D00001EBC00018309DF8AC1040F2231211FBAF
:10B9E00002F12E4A02EBC10118319DF8982002EBBA
:10B9F000C20201EB021191F8801001EBC10100EBD2
:10BA0000011043719DF8AC100220FEF70DFB9DF86C
:10BA1000AC0000EB400101EB0010214901EB0011EB
:10BA200030319DF8980001EB0010807800F00102A1
:10BA30009DF8AC0040F2231110FB01F0174901EB17
:10BA4000C00018309DF8981001EBC10100EB011007
:10BA5000007E00F0010082427DD09DF8AC0040F2F3
:10BA6000231110FB01F00D4901EBC00018309DF8C7
:10BA7000981001EBC10100EB0110183009909DF8FE
:10BA8000AC0000EB400101EB0010054901EB001098
:10BA900030309DF8981000EB011005E0C444002000
:10BAA00004400020BC320020807809990A7860F3B5
:10BAB00000020A709DF8AC1001EB410000EB011090
:10BAC000FE4901EB001030309DF8981000EB01109A
:10BAD000807800F00100E8BB9DF8AC1001EB41005C
:10BAE00000EB0110F54901EB001030309DF8981083
:10BAF00000EB01108078C0F3401068B39DF8AC10E3
:10BB000040F2231011FB00F0ED4901EBC0001830AA
:10BB10009DF8981001EBC10100EB011090F83E0078
:10BB2000D0B99DF8AC1040F2231011FB00F0E449AD
:10BB300001EBC00018309DF8981001EBC10100EB3B
:10BB40000110407B40B99DF8AC0000EB400101EBD7
:10BB5000001002E05BE069E239E0D84901EB001037
:10BB600030309DF8981000EB01108078C0F3400051
:10BB700068BB01229DF8AC0040F2231110FB01F0DC
:10BB8000CF4901EBC00118319DF8980000EBC000CF
:10BB900001EB00104273D9229DF8AC0040F2231152
:10BBA00010FB01F0C64901EBC00118319DF8980067
:10BBB00000EBC00001EB0010427101229DF8AC00C7
:10BBC00040F2231110FB01F0BD4901E0F5E30AE06A
:10BBD00001EBC00018309DF8981001EBC10100EB9B
:10BBE000011080F83E2000229DF8AC0040F22311A5
:10BBF00010FB01F0B24901EBC00118319DF898002B
:10BC000000EBC00001EB001080F83D2009E29DF838
:10BC1000AC0040F2231110FB01F0A94901EBC00078
:10BC200018309DF8981001EBC10100EB011090F85D
:10BC30003E0098B901229DF8AC0040F2231110FBA0
:10BC400001F09F4901EBC00018309DF8981001EBFE
:10BC5000C10100EB011080F83D202BE000229DF88F
:10BC6000AC0040F2231110FB01F0954901EBC0013B
:10BC700018319DF8980000EBC00001EB001080F82F
:10BC80003D209DF8AC1001EB410000EB01108B4909
:10BC900001EB0011303102E0FEE3FEE356E39DF8D4
:10BCA000980001EB0010801C0990007820F0010240
:10BCB00009980270834890F8900790B19DF8AC10F5
:10BCC00001EB410000EB01107C4901EB001000E0AA
:10BCD000F0E330309DF8981000EB0110807A0228D4
:10BCE00094D1794890F8290001288FD17648D0F86E
:10BCF0000C027549498D884288D29DF8AC1040F2FB
:10BD0000231011FB00F06E4901EBC00018309DF8C4
:10BD1000981001EBC10100EB011090F83D000128E3
:10BD200050D19DF8AC0040F2231110FB01F06449A2
:10BD300001EBC00018309DF8981001EBC10100EB39
:10BD4000011090F87E00E8BB9DF8AC0000EB4001CC
:10BD500001EB0010594901EB001130319DF89800BA
:10BD600001EB001001789DF8AC0040F2231210FBAB
:10BD700002F0534A02EBC0004170C3229DF8AC00B0
:10BD800040F2231110FB01F04D4900E0BBE101EB53
:10BD9000C00118319DF8980000EBC00001EB0010C5
:10BDA000427100229DF8AC0000EB400101EB001055
:10BDB000424901EB001130319DF8980001EB001071
:10BDC000426000E057E001229DF8AC0000EB40012A
:10BDD00001EB0010394901EB001130319DF898005A
:10BDE00001EB0010C2729DF8AC100220FEF71CF9A6
:10BDF0000021379119E000229DF8AC0040F2231198
:10BE000010FB01F02E4901EBC00118319DF898009C
:10BE100000EBC00001EB00113F31BDF8DC000A541B
:10BE2000BDF8DC00401C81B23791BDF8DC0006286B
:10BE3000E1DB0021379119E000229DF8AC0040F2CF
:10BE4000231110FB01F01E4901EBC00118319DF8D0
:10BE5000980000EBC00001EB00115B31BDF8DC0085
:10BE60000A54BDF8DC00401C81B23791BDF8DC00FB
:10BE70000F28E1DBD5E09DF8AC1040F2231011FB58
:10BE800000F00F4901EBC00018309DF8981001EB4D
:10BE9000C10100EB011090F83D0001287ED19DF812
:10BEA000AC1040F2231011FB00F0054901EBC0017A
:10BEB00018319DF8980000EBC00007E00440002016
:10BEC000C4440020BC320020BC12002001EB001052
:10BED00090F87F1040F2231011FB00F0FC4901EBB9
:10BEE000C00118319DF8AC0040F2231210FB02F0A3
:10BEF000F74A02EBC00018309DF8982002EBC2020E
:10BF000000EB021090F8800000EBC00001EB001085
:10BF100090F87700032841D100239DF8AC0040F24F
:10BF2000231110FB01F0EA4901EBC00118319DF823
:10BF3000980000EBC00001EB001090F87F0040F289
:10BF4000231110FB01F0E24901EBC00118319DF80B
:10BF5000AC0040F2231210FB02F0DD4A02EBC002FB
:10BF600018329DF8980000EBC00002EB001090F82A
:10BF7000800000EBC00001EB001080F877309DF8E6
:10BF8000AC0000EB400101EB0010D24901EB0011C5
:10BF900030319DF8980001EB001000E041E001789D
:10BFA0009DF8AC0040F2231210FB02F0C84A02EBED
:10BFB000C0004170C3229DF8AC0040F2231110FB79
:10BFC00001F0C34901EBC00118319DF8980000EB66
:10BFD000C00001EB0010427100229DF8AC0000EBA4
:10BFE000400101EB0010BB4901EB001130319DF81D
:10BFF000980001EB0010426002229DF8AC0000EBBB
:10C00000400101EB0010B34901EB001130319DF804
:10C01000980001EB0010C2729DF8AC100220FEF7F0
:10C0200003F89DF8AC100220FDF7FEFF9DF8AC0070
:10C0300000EB400101EB0010A64901EB001030308D
:10C040009DF8981000EB01108078C0F3400088B193
:10C05000D9229DF8AC0040F2231110FB01F09C495D
:10C0600001EBC00018309DF8981001EBC10100EB06
:10C07000011042719DF8AC0040F2231110FB01F059
:10C08000934901EBC00018309DF8981001EBC101F5
:10C0900000EB01108078B22835D19DF8AC0000EBA0
:10C0A000400101EB00108B4901EB001030309DF88E
:10C0B000981000EB01108078C0F3400018BB9DF889
:10C0C000AC0000EB400101EB0010824901EB0010D5
:10C0D00030309DF8981000EB01108078C0F34010CC
:10C0E00088B9E5229DF8AC0040F2231110FB01F065
:10C0F000774901EBC00018309DF8981001EBC101A1
:10C1000000EB011042719DF8AC0000EB400101EB27
:10C110000010704901EB001030309DF8981000EBD2
:10C12000011080780121B1EBD01F75D19DF8AC00D2
:10C1300000EB400101EB0010664901EB00103030CC
:10C140009DF8981000EB0110807800F001000028A5
:10C1500062D19DF8AC0040F2231110FB01F05C4964
:10C1600001EBC00018309DF8981001EBC10100EB05
:10C17000011090F83E0000284ED19DF8AC0000EB75
:10C18000400101EB0010534901EB001030309DF8E5
:10C19000981000EB01108078C0F3C000E0BB9DF860
:10C1A000AC0000EB400101EB00104A4901EB00102C
:10C1B00030309DF8981000EB0110407A00F001003B
:10C1C00050B39DF8AC0040F2231110FB01F0404940
:10C1D00001EBC00018309DF8981001EBC10100EB95
:10C1E000011090F88E0000F00100A8B99DF8AC0095
:10C1F00040F2231110FB01F0354901EBC00018306B
:10C200009DF8981001EBC10100EB011090F881003E
:10C2100010B1002137912AE096E09DF8AC0040F281
:10C22000231110FB01F02A4901EBC00118319DF8E0
:10C23000980000EBC00001EB001000F18201BDF896
:10C24000DC000A5C9DF8AC0000EB400101EB001043
:10C25000204901EB00100E30BDF8DC10405C82423A
:10C2600000D008E0BDF8DC00401C81B23791BDF879
:10C27000DC000628D1DB00BFBDF8DC00062863D156
:10C28000062137912DE09DF8AC0040F2231110FB00
:10C2900001F00F4901EBC00118319DF8980000EB47
:10C2A000C00001EB001000F18201BDF8DC000A5C67
:10C2B0009DF8AC0000EB400101EB0010054901EBDB
:10C2C00000100E30BDF8DC10405C824204D00CE05F
:10C2D000C444002004400020BDF8DC00401C81B2B2
:10C2E0003791BDF8DC000A28CDDB00BFBDF8DC00CB
:10C2F0000A2829D09DF8AC1040F2231011FB00F061
:10C30000FE4901EBC00018309DF8981001EBC10107
:10C3100000EB01108E300990007820F00100401CE5
:10C320000999087012229DF8AC0040F2231110FB0D
:10C3300001F0F24901EBC00018309DF8981001EBB4
:10C34000C10100EB0110427101F03CBC9DF8AC1042
:10C3500001EB410000EB0110E94901EB0010007B0B
:10C3600060BBBDF89C00082800D0EDE700213791A4
:10C370002AE09DF8AC1001EB4100C0EBC110E1498F
:10C3800001EBC001BDF8DC00C01C085C00F00F0030
:10C39000092800DD1CE09DF8AC1001EB4100C0EB6A
:10C3A000C110D84901EBC001BDF8DC00C01C085C1D
:10C3B00000F0F000902802DD0AE0F3E17BE0BDF838
:10C3C000DC00401C81B23791BDF8DC000628D0DBD0
:10C3D00000BFBDF8DC00062800DAB5E79DF8AC1018
:10C3E00001EB4100C0EBC110C64901EBC000C078B1
:10C3F00001049DF8AC0000EB4002C2EBC010C14A42
:10C4000002EBC000007941EA00219DF8AC0000EB8E
:10C410004002C2EBC010BB4A02EBC00040790143AE
:10C420009DF8AC0040F2231210FB02F0B34A02EB7D
:10C43000C00218329DF8980000EBC00002EB00101B
:10C44000C0F81A109DF8AC1001EB4100C0EBC11010
:10C45000AC4901EBC000807901049DF8AC0000EB11
:10C460004002C2EBC010A74A02EBC000C07941EA0B
:10C4700000219DF8AC0000EB4002C2EBC010A14AC5
:10C4800002EBC000007A01439DF8AC0040F2231299
:10C4900010FB02F0994A01E0CCE137E202EBC00068
:10C4A00018309DF8982002EBC20200EB0210C0F891
:10C4B0001E10BBE0ABE1BDF89C000A2800D043E7AA
:10C4C0000021379128E09DF8AC1001EB4100C0EB52
:10C4D000C1108C4901EBC001BDF8DC00C01C085C38
:10C4E00000F00F00092800DD1AE09DF8AC1001EB08
:10C4F0004100C0EBC110834901EBC001BDF8DC0075
:10C50000C01C085C00F0F000902800DD08E0BDF8D9
:10C51000DC00401C81B23791BDF8DC000828D2DB7A
:10C5200000BFBDF8DC00082800DA0DE79DF8AC106C
:10C5300001EB4100C0EBC110724901EBC000C078B3
:10C5400001069DF8AC0000EB4002C2EBC0106D4A42
:10C5500002EBC000007941EA00419DF8AC0000EB1D
:10C560004002C2EBC010674A02EBC000407941EACA
:10C5700000219DF8AC0000EB4002C2EBC010614A04
:10C5800002EBC000807901439DF8AC0040F2231219
:10C5900010FB02F0594A02EBC00218329DF89800D5
:10C5A00000EBC00002EB0010C0F81A109DF8AC10B0
:10C5B00001EB4100C0EBC110524901EBC000C07952
:10C5C00001069DF8AC0000EB4002C2EBC0104D4AE2
:10C5D00002EBC000007A41EA00419DF8AC0000EB9C
:10C5E0004002C2EBC010474A02EBC000407A41EA69
:10C5F00000219DF8AC0000EB4002C2EBC010414AA4
:10C6000002EBC000807A01439DF8AC0040F2231297
:10C6100010FB02F0394A02EBC00018309DF8982058
:10C6200002EBC20200EB0210C0F81E109DF8AC0035
:10C6300040F2231110FB01F0304901EBC001183129
:10C640009DF8980000EBC00001EB001001789DF808
:10C65000AC0040F2231210FB02F0284A02EBC000AB
:10C66000407981422FDA00219DF8AC0040F223127C
:10C6700010FB02F0214A02EBC000017104229DF878
:10C68000AC0040F2231110FB01F01C4901EBC0018A
:10C6900018319DF8980000EBC00001EB001002700B
:10C6A000C5229DF8AC0040F2231110FB01F01349A4
:10C6B00001EBC00018309DF8981001EBC10100EBB0
:10C6C000011042716DE09DF8AC1001EB410000EBF0
:10C6D00001100B4901EB001030309DF8981000EB71
:10C6E00001108078C0F34000C8B1D5229DF8AC009D
:10C6F00040F2231110FB01F0004905E0C444002082
:10C7000004400020A477002001EBC00018309DF801
:10C71000981001EBC10100EB0110427141E09DF85E
:10C72000AC1040F2231011FB00F0FE4901EBC000F9
:10C7300018309DF8981001EBC10100EB0110807BCF
:10C7400001282ED100229DF8AC0040F2231110FBED
:10C7500001F0F44901EBC00118319DF8980000EB9D
:10C76000C00001EB00108273B6229DF8AC0040F2CD
:10C77000231110FB01F0EB4901EBC00118319DF8CA
:10C78000980000EBC00001EB0010427100219DF801
:10C79000AC0040F2231210FB02F0E24A02EBC000B0
:10C7A0000171D1E5D5229DF8AC0040F2231110FBB8
:10C7B00001F0DC4901EBC00118319DF8980000EB55
:10C7C000C00001EB0010427101219DF8AC0040F265
:10C7D000231210FB02F0D34A02EBC00001719DF856
:10C7E000AC1001EB410000EB0110A2F5986101EBE8
:10C7F000001130319DF8980001EB0010801C099069
:10C80000007820F020002030099908709CE5D5229E
:10C810009DF8AC0040F2231110FB01F0C14901EB7F
:10C82000C00018309DF8981001EBC10100EB011019
:10C83000427189E59DF8AC1040F2231011FB00F025
:10C84000B84901EBC0001830BDF8D01001EBC101B0
:10C8500000EB0110807901283AD100229DF8AC004C
:10C8600040F2231110FB01F0AE4901EBC001183179
:10C87000BDF8D00000EBC00001EB00108271D522A2
:10C880009DF8AC0040F2231110FB01F0A54901EB2B
:10C89000C00118319DF8980000EBC00001EB0010BA
:10C8A00042719DF8AC0000EB400101EB00109E4985
:10C8B00001EB001130319DF8980001EB0010801C55
:10C8C0000990007820F00400001D099908701CE010
:10C8D000C3229DF8AC0040F2231110FB01F09149F6
:10C8E00001EBC00118319DF8980000EBC00001EB8E
:10C8F0000010427100219DF8AC0040F2231210FBA1
:10C9000002F0884A02EBC00001711DE59DF8AC0001
:10C9100040F2231110FB01F0824901EBC0001830F6
:10C92000BDF8D01001EBC10100EB011080790128A6
:10C930003AD100229DF8AC0040F2231110FB01F027
:10C94000784901EBC0011831BDF8D00000EBC00000
:10C9500001EB00108271D5229DF8AC0040F223114A
:10C9600010FB01F06F4901EBC00118319DF89800F0
:10C9700000EBC00001EB001042719DF8AC0000EB31
:10C98000400101EB0010684901EB001130319DF8C6
:10C99000980001EB0010801C0990007820F0040042
:10C9A000001D099908701CE0C3229DF8AC0040F2FC
:10C9B000231110FB01F05B4901EBC00118319DF818
:10C9C000980000EBC00001EB0010427100219DF8BF
:10C9D000AC0040F2231210FB02F0524A02EBC000FE
:10C9E0000171B1E49DF8AC0000EB400101EB0010D7
:10C9F0004D4901EB0010007B38BB9DF8AC0000EB0B
:10CA00004001C1EBC010494901EBC00001799DF81C
:10CA1000AC0000EB4002C2EBC010444A02EBC00085
:10CA2000C07841EA00229DF8AC0040F2231110FBCF
:10CA300001F03C4901EBC00118319DF8980000EB72
:10CA4000C00001EB0010426332E09DF8AC1001EB36
:10CA50004100C0EBC110354901EBC000C0780104B2
:10CA60009DF8AC0000EB4002C2EBC0102F4A02EB75
:10CA7000C000007941EA00219DF8AC0000EB4002C3
:10CA8000C2EBC010294A02EBC000407901439DF877
:10CA9000AC0040F2231210FB02F0224A02EBC0006D
:10CAA00018309DF8982002EBC20200EB021041639F
:10CAB0009DF8AC1040F2231011FB00F0194901EB76
:10CAC000C00118319DF8980000EBC00001EB001088
:10CAD00001789DF8AC0040F2231210FB02F0114ADD
:10CAE00002EBC0004079814236DA00219DF8AC00AB
:10CAF00040F2231210FB02F00A4A02EBC00001715F
:10CB000003229DF8AC0040F2231110FB01F005490F
:10CB100001EBC00118319DF8980000EBC00001EB5B
:10CB2000001005E0C444002004400020A477002049
:10CB30000270D9229DF8AC0040F2231110FB01F0E5
:10CB4000FC4901EBC00018309DF8981001EBC101C1
:10CB500000EB0110427175E09DF8AC1040F223101B
:10CB600011FB00F0F34901EBC0001830BDF8D01004
:10CB700001EBC10100EB01108079012845D10022B1
:10CB80009DF8AC0040F2231110FB01F0E94901EBE4
:10CB9000C0011831BDF8D00000EBC00001EB00105F
:10CBA0008271D9229DF8AC0040F2231110FB01F0F4
:10CBB000E04901EBC00118319DF8980000EBC0007E
:10CBC00001EB001042719DF8AC1001EB410000EB4D
:10CBD0000110D94901EB001130319DF8980001EBAB
:10CBE0000010801C0990007820F00400001D0999B5
:10CBF000087001209DF8AC1040F2231211FB02F1E5
:10CC0000CC4A02EBC10108711CE0C5229DF8AC00C2
:10CC100040F2231110FB01F0C64901EBC0011831AD
:10CC20009DF8980000EBC00001EB0010427100215C
:10CC30009DF8AC0040F2231210FB02F0BD4A02EB5B
:10CC4000C00001713BE400219DF8AC0040F22312CA
:10CC500010FB02F0B74A02EBC00001719DF8AC0076
:10CC600000EB400101EB0010B34901EB0011303142
:10CC70009DF8980001EB0010801C0990007820F0CE
:10CC80000400001D09990870D5229DF8AC0040F2FF
:10CC9000231110FB01F0A74901EBC00018309DF8EB
:10CCA000981001EBC10100EB0110427107E49DF8FF
:10CCB000AC1001EB410000EB01109F4901EB0010AB
:10CCC000007BD0BBBDF89C000C2800D02DE40020D8
:10CCD000379028E09DF8AC1001EB4100C0EBC1108B
:10CCE000964901EBC001BDF8DC00C01C085C00F0F7
:10CCF0000F00092800DD1AE09DF8AC1001EB41009F
:10CD0000C0EBC1108D4901EBC001BDF8DC00C01CB7
:10CD1000085C00F0F000902800DD08E0BDF8DC00C1
:10CD2000401C81B23791BDF8DC000A28D2DB00BF7D
:10CD3000BDF8DC000A2801DA33E57CE000202C9005
:10CD40002D90002137911EE0DDE92C10000240EA11
:10CD500011620902CDE92C129DF8AC1001EB4100E3
:10CD6000C0EBC110754901EBC001BDF8DC00C01C6F
:10CD7000085CDDE92C341843CDE92C04BDF8DC0057
:10CD8000401C80B23790BDF8DC000528DCDB9DF844
:10CD9000AC00DDE92C1240F2231310FB03F0654BCD
:10CDA00003EBC00318339DF8980000EBC00003EBC1
:10CDB000001040F8221F426000222C922D92002188
:10CDC00037911EE0DDE92C10000240EA11620902F1
:10CDD000CDE92C129DF8AC1001EB4100C0EBC11065
:10CDE000564901EBC001BDF8DC000830085CDDE904
:10CDF0002C341843CDE92C04BDF8DC00401C80B273
:10CE00003790BDF8DC000528DCDB9DF8AC00DDE9DF
:10CE10002C2140F2231310FB03F0464B03EBC00020
:10CE200018309DF8983003EBC30300EB0310223059
:10CE30008260C160BCE0BDF89C000E2800D0B0E468
:10CE40000021379128E09DF8AC1001EB4100C0EBC8
:10CE5000C1103A4901EBC001BDF8DC00C01C085C00
:10CE600000F00F00092800DD1AE09DF8AC1001EB7E
:10CE70004100C0EBC110314901EBC001BDF8DC003D
:10CE8000C01C085C00F0F000902800DD08E0BDF850
:10CE9000DC00401C81B23791BDF8DC000C28D2DBED
:10CEA00000BFBDF8DC000C2800DA7AE400202C90EA
:10CEB0002D90002137911EE0DDE92C10000240EAA0
:10CEC00011620902CDE92C129DF8AC1001EB410072
:10CED000C0EBC110194901EBC001BDF8DC00C01C5A
:10CEE000085CDDE92C341843CDE92C04BDF8DC00E6
:10CEF000401C80B23790BDF8DC000628DCDB9DF8D2
:10CF0000AC00DDE92C2140F2231310FB03F0094BA8
:10CF100003EBC00318339DF8980000EBC00003EB4F
:10CF2000001040F8222F416000222C922D92002107
:10CF3000379124E0C444002004400020A47700205E
:10CF4000DDE92C10000240EA11620902CDE92C1241
:10CF50009DF8AC1001EB4100C0EBC110FE4901EBA4
:10CF6000C001BDF8DC000930085CDDE92C34184351
:10CF7000CDE92C04BDF8DC00401C80B23790BDF830
:10CF8000DC000628DCDB9DF8AC00DDE92C2140F25A
:10CF9000231310FB03F0F14B03EBC00018309DF896
:10CFA000983003EBC30300EB031022308260C160B2
:10CFB0009DF8AC1040F2231011FB00F0E74901EBA3
:10CFC000C00118319DF8980000EBC00001EB001083
:10CFD00001789DF8AC0040F2231210FB02F0DF4A0A
:10CFE00002EBC000407981427ED19DF8AC009DF8F3
:10CFF000981001EB0010C217CDE92C02D84890F828
:10D00000900708B39DF8AC1001EB410000EB011054
:10D01000D44901EB001030309DF8981000EB01105E
:10D02000807A022810D09DF8AC1001EB410000EB93
:10D030000110CC4901EB001030309DF8981000EB46
:10D040000110C07A00287CDD00229DF8AC0000EBC6
:10D05000400101EB0010C34901EB001030309DF896
:10D06000981000EB0110C272BF48D0F80C020521E5
:10D07000B0FBF1F201FB120000EB4001BA482C308A
:10D0800000EB41100D3009909DF8AC0040F22311E7
:10D0900010FB01F1B14800EBC10018309DF8981069
:10D0A00001EBC10100EB0110223010220146089073
:10D0B0000998FBF7CAF8AC48D0F80C020521B0FB80
:10D0C000F1F201FB120000EB4001A7482C3000EB0D
:10D0D00041129DF8AC0040F2231110FB01F09F4972
:10D0E00001EBC001183100E0AAE29DF8980000EBC6
:10D0F000C00001EB001050F81A1F42F8011F4068F1
:10D1000050609948D0F80C020521B0FBF1F201FB08
:10D11000120000EB400194482C3000EB41129DF8C6
:10D12000AC0000EB400101EB00108E4901EB001157
:10D1300030319DF8980001EB0010007810708A489B
:10D1400000E07DE1D0F80C020521B0FBF1F201FB1B
:10D15000120000EB400184482C3000EB4111834861
:10D16000C26841F81D2F008A88807F48D0F80C02E1
:10D170000521B0FBF1F201FB120000EB40017A48FF
:10D180002C3000EB41129DF8AC0040F2231110FB53
:10D1900001F0724901EBC00118319DF8980000EBD5
:10D1A000C00001EB0010406BC2F809006E48D0F8D7
:10D1B0000C020521B0FBF1F201FB120000EB400173
:10D1C00069482C3000EB41129DF8AC0000EB4001A7
:10D1D00001EB0010634901EB001130319DF898001C
:10D1E00001EB00104068C2F8230000229DF8AC005B
:10D1F00000EB400101EB00105A4901EB0011303106
:10D200009DF8980001EB00104260002137914BE03F
:10D210005548D0F80C020521B0FBF1F201FB1200D9
:10D2200000EB400150482C3000EB41112731BDF894
:10D23000DC409DF8AC0040F2231210FB02F0474A9C
:10D2400002EBC00218329DF8980000EBC00002EB20
:10D25000001090F87F0040F2231210FB02F03F4ACA
:10D2600002EBC00218329DF8AC0040F2231310FB11
:10D2700003F03A4B03EBC00318339DF8980000EB22
:10D28000C00003EB001090F8800000EBC00002EB40
:10D2900000123F32BDF8DC00001D105C0855BDF8DF
:10D2A000DC00401C81B23791BDF8DC000628AFDB02
:10D2B0000020379039E000239DF8AC0040F22311A4
:10D2C00010FB01F0254901EBC00118319DF89800D1
:10D2D00000EBC00001EB001090F87F0040F223113A
:10D2E00010FB01F01D4901EBC00118319DF8AC00A5
:10D2F00040F2231210FB02F0184A02EBC00218326F
:10D300009DF8980000EBC00002EB001090F8800040
:10D3100000EBC00001EB00113F31BDF8DC000B5405
:10D32000BDF8DC00401C81B23791BDF8DC000A2852
:10D33000C1DB0D48D0F80C020521B0FBF1F080B242
:10D34000014609900220FBF7C3FE00210620FCF7EE
:10D350006BFE05480CE00000A4770020C4440020C8
:10D36000BC32002004400020BC120020BC31002050
:10D37000D0F80C02F849498D884206D2F648D0F818
:10D380000C02401CF449C1F80C0200210520FCF7F6
:10D390004BFE9DF8AC0000EB400101EB0010EF49A3
:10D3A00001EB001030309DF8981000EB0110801C4C
:10D3B0000990007820F00400001D09990870E648E3
:10D3C000D0F80C020521B0FBF1F201FB120000EBDA
:10D3D0004001E1482C3000EB4110D0F823202C987C
:10D3E00000EB4001DE4800EB4110C0F82320002094
:10D3F000379020E0D848D0F80C020521B0FBF1F2BC
:10D4000001FB120000EB4001D3482C3000EB41102F
:10D410002730BDF8DC10425C2C9800EB4001D0486E
:10D4200000EB41112731BDF8DC000A54BDF8DC00E7
:10D43000401C81B23791BDF8DC000628DADB56E0EB
:10D440009DF8AC0000EB400101EB0010C34901EB7B
:10D45000001030309DF8981000EB0110801C0990EE
:10D46000007820F008000830099908709DF8AC0099
:10D4700000EB400101EB0010B84901EB0010303027
:10D480009DF8981000EB011042682C9800EB4001C9
:10D49000B34800EB4110C0F823200020379022E071
:10D4A0009DF8AC0040F2231110FB01F0AD4901EBF7
:10D4B000C00118319DF8980000EBC00001EB00118D
:10D4C0003F31BDF8DC000A5C2C9800EB4001A44819
:10D4D00000EB41112731BDF8DC000A54BDF8DC0037
:10D4E000401C81B23791BDF8DC000628D8DB9DF8DE
:10D4F000AC0000EB400101EB0010984901EB00107B
:10D5000030309DF8981000EB0110801C09900078D5
:10D5100020F02002099802709DF8AC100220FCF760
:10D5200083FD9DF8AC0040F2231110FB01F08D4902
:10D5300001EBC00018309DF8981001EBC10100EB21
:10D540000110223009902C9800EB4001844800EB38
:10D5500041100D30102208900999FAF776FE9DF8D7
:10D56000AC0040F2231110FB01F07E4901EBC00139
:10D5700018319DF8980000EBC00001EB00112C98C9
:10D5800000EB4002764800EB421051F81A2F40F8A9
:10D59000012F496841609DF8AC0000EB400101EBB0
:10D5A00000106E4901EB001130319DF8980001EB3D
:10D5B000001001782C9800EB4002694800EB421003
:10D5C00001702C9800EB4001654800EB4111664862
:10D5D000C26841F81D2F008A88809DF8AC0040F297
:10D5E000231110FB01F05F4901EBC00118319DF8D8
:10D5F000980000EBC00001EB0010416B2C9800EB91
:10D600004002574800EB4210C0F809102C9881B234
:10D6100008200991FCF708FD00229DF8AC0040F2BB
:10D62000231110FB01F04F4901EBC00018309DF8A9
:10D63000981001EBC10100EB011080F83E2051E091
:10D640009DF8AC0000EB400101EB0010434901EBF9
:10D65000001030309DF8981000EB0110801C0990EC
:10D66000007820F00400001D099908709DF8AC00B6
:10D6700000EB400101EB0010384901EB00103030A5
:10D680009DF8981000EB0110801C0990007820F0A4
:10D69000800080300999087001209DF8AC1040F29C
:10D6A000231211FB02F12F4A02EBC10108719DF810
:10D6B000AC0040F2231110FB01F0114601EBC00059
:10D6C00042799DF8AC0040F2231110FB01F025498E
:10D6D00001EBC00018309DF8981001EBC10100EB80
:10D6E00001100270D5229DF8AC0040F2231110FB0E
:10D6F00001F01C4901EBC00018309DF8981001EBB7
:10D70000C10100EB011042715CE2D5229DF8AC0032
:10D7100040F2231110FB01F0124901EBC000183058
:10D720009DF8981001EBC10100EB0110427149E234
:10D73000D5229DF8AC0040F2231110FB01F00949FD
:10D7400001EBC00018309DF8981001EBC10100EB0F
:10D750000110427136E20000BC120020044000209B
:10D76000D8140020C4440020BC3100200121FE4810
:10D7700080F8B4169DF8AC0040F2231110FB01F0C4
:10D78000FA4901EBC00118319DF8980000EBC00088
:10D7900001EB001001789DF8AC0040F2231210FB61
:10D7A00002F0F24A02EBC000407981422FDA0021F8
:10D7B0009DF8AC0040F2231210FB02F0EB4A02EBA2
:10D7C000C000017101229DF8AC0040F2231110FB52
:10D7D00001F0E64901EBC00118319DF8980000EB1B
:10D7E000C00001EB0010027011229DF8AC0040F265
:10D7F000231110FB01F0DD4901EBC00018309DF84A
:10D80000981001EBC10100EB0110427154E09DF84A
:10D81000AC1040F2231011FB00F0D44901EBC00022
:10D8200018309DF8981001EBC10100EB01108078D1
:10D83000B2282FD100219DF8AC0040F2231210FB3A
:10D8400002F0CA4A02EBC0000171B2229DF8AC009E
:10D8500040F2231110FB01F0C44901EBC001183163
:10D860009DF8980000EBC00001EB0010427100220F
:10D870009DF8AC0040F2231110FB01F0BB4901EB15
:10D88000C00018309DF8981001EBC10100EB0110A9
:10D89000827011E0D5229DF8AC0040F2231110FBFC
:10D8A00001F0B24901EBC00018309DF8981001EB6F
:10D8B000C10100EB0110427184E10021AA4880F807
:10D8C000B416D5229DF8AC0040F2231110FB01F0F4
:10D8D000A64901EBC00018309DF8981001EBC1017A
:10D8E00000EB011042716DE101229DF8AC0040F2A5
:10D8F000231110FB01F09D4901EBC00118319DF887
:10D90000980000EBC00001EB001080F8812000219E
:10D91000379126E09DF8AC1001EB4100C0EBC1103F
:10D92000934901EBC001BDF8DC00C01C0A5C9DF806
:10D93000AC0040F2231110FB01F08C4901EBC00157
:10D9400018319DF8980000EBC00001EB001000F1C9
:10D950008201BDF8DC000A54BDF8DC00401C81B235
:10D960003791BDF8DC000A28D4DB2BE19DF8AC1020
:10D9700001EB4100C0EBC1107D4901EBC000C07854
:10D9800001049DF8AC0000EB4002C2EBC010784AE5
:10D9900002EBC000007941EA00209DF8AC1001EBD9
:10D9A0004102C2EBC111724A02EBC101497908433D
:10D9B000B0F5E13F65D19DF8AC1001EB410000EB03
:10D9C00001106C4901EB001030309DF8981000EB0D
:10D9D0000110801C0990007820F004020998027060
:10D9E00000229DF8AC0040F2231110FB01F05F49CA
:10D9F00001EBC00018309DF8981001EBC10100EB5D
:10DA00000110A0F88C2013229DF8AC0040F22311E5
:10DA100010FB01F0554901EBC00018309DF898103B
:10DA200001EBC10100EB011042719DF8AC1001EB5C
:10DA3000410000EB01104F4901EB00104079034613
:10DA40004FF480524FF4E13109909DF8AC0011F091
:10DA5000E3FA9DF8AC1040F2231011FB00F04349AB
:10DA600001EBC00118319DF8980000EBC00001EBFC
:10DA700000108E300990007820F0080008300999D5
:10DA800008709FE09DF8AC1001EB4100C0EBC110A5
:10DA9000374901EBC00001799DF8AC0000EB400272
:10DAA000C2EBC010324A02EBC000C07841EA00224B
:10DAB0009DF8AC0040F2231110FB01F02B4901EB63
:10DAC000C00118319DF8980000EBC00001EB001078
:10DAD000A0F88C209DF8AC1040F2231011FB00F050
:10DAE000224901EBC00118319DF8980000EBC000FD
:10DAF00001EB0010B0F88C109DF8AC0000EB400278
:10DB000002EB00101B4A02EB0010408B814258DBF5
:10DB1000E5229DF8AC0040F2231110FB01F01349FF
:10DB200001EBC00118319DF8980000EBC00001EB3B
:10DB30000010427100229DF8AC0040F2231110FB4E
:10DB400001F00A4901EBC00118319DF8980000EB83
:10DB5000C00001EB001002709DF8AC1001EB410019
:10DB600000EB0110034907E0BC320020C444002050
:10DB7000A47700200440002001EB001130319DF813
:10DB8000980001EB0010801C0990007820F08002C2
:10DB9000099802709DF8AC1040F2231011FB00F0C0
:10DBA000FE4901EBC00018309DF8981001EBC1014F
:10DBB00000EB01108E300990007820F001020998E6
:10DBC000027000BF00BF09F0A3BE9DF8AC1001EBCE
:10DBD0004100C0EBC110F24911F83000042801D116
:10DBE00024900BE09DF8AC1001EB4100C0EBC1109C
:10DBF000EB4911F83000152800D124909DF8AC10A5
:10DC000001EB4100C0EBC110E54901EBC0004178D8
:10DC10009DF8AC0000EB4002C2EBC010E04A12F8E5
:10DC2000300041EA002041F23001884202D1A620B2
:10DC300024903DE09DF8AC1001EB4100C0EBC11019
:10DC4000D74901EBC00041789DF8AC0000EB4002E1
:10DC5000C2EBC010D24A12F8300041EA002041F273
:10DC60003101884202D1A720249021E09DF8AC1018
:10DC700001EB4100C0EBC110C94911F83000022886
:10DC800016D19DF8AC1001EB4100C0EBC110C449A6
:10DC900001EBC00001799DF8AC0000EB4002C2EB43
:10DCA000C010BF4A02EBC000C07841EA00212491B5
:10DCB0009DF8AC1040F2231011FB00F0B74901EBC6
:10DCC000C000817826910021B64A9DF8AC0002EB95
:10DCD00000129DF898001154B34890F828000128CC
:10DCE00015D19DF8AC1001EB410000EB0110AF49DC
:10DCF00001EB001030309DF8981000EB0110801CF3
:10DD00000990007820F08000803009990870BDF8F3
:10DD1000901043F23002881A91427DD009DC042928
:10DD20007BD015297AD0A62910D0A72942F090815E
:10DD300043E1B0F5C06F72D0A0F2016000286FD04F
:10DD400001286ED00428F1D101F056BD00219DF8C4
:10DD5000AC0040F2231210FB02F0904A02EBC0002C
:10DD600001719DF8AC0040F2231110FB01F0114647
:10DD700001EBC00018309DF8981001EBC10100EBD9
:10DD800001100078052824DC06229DF8AC0040F242
:10DD9000231110FB01F0814901EBC00118319DF8FE
:10DDA000980000EBC00001EB00100270A8229DF863
:10DDB000AC0040F2231110FB01F0784901EBC000E8
:10DDC00018309DF8981001EBC10100EB0110427171
:10DDD000F1E09DF8AC0040F2231110FB01F06F4917
:10DDE00001EBC00018309DF8981001EBC10100EB69
:10DDF000011000780A282BDC0B229DF8AC0040F2C1
:10DE0000231110FB01F0654901EBC00118319DF8A9
:10DE1000980000EBC00005E084E1FAE1FEE3FEE3D8
:10DE2000FEE3FEE301EB00100270A9229DF8AC00B6
:10DE300040F2231110FB01F0584901EBC0001830EB
:10DE40009DF8981001EBC10100EB01104271B2E0A6
:10DE50009DF8AC0040F2231110FB01F04F4901EB9B
:10DE6000C00018309DF8981001EBC10100EB0110C3
:10DE700000780F2824DC10229DF8AC0040F223111A
:10DE800010FB01F0454901EBC00118319DF89800E5
:10DE900000EBC00001EB00100270A2229DF8AC0064
:10DEA00040F2231110FB01F03C4901EBC000183097
:10DEB0009DF8981001EBC10100EB011042717AE06E
:10DEC0009DF8AC0040F2231110FB01F0334901EB47
:10DED000C00018309DF8981001EBC10100EB011053
:10DEE0004079A52815D19DF8AC0000EB400101EB6D
:10DEF00000102E4901EB001030309DF8981000EB17
:10DF00000110801C0990007820F00400001D099980
:10DF100008709DF8AC0040F2231110FB01F01F497E
:10DF200001EBC00018309DF8981001EBC10100EB27
:10DF300001108078A1283ED09DF8AC0040F223115A
:10DF400010FB01F0154901EBC00118319DF8980054
:10DF500000EBC00001EB001082789DF8AC0040F2AD
:10DF6000231110FB01F00D4901EBC00118319DF8A0
:10DF7000980000EBC00001EB00104271A1229DF857
:10DF8000AC0040F2231110FB01F0044901EBC0008A
:10DF900018309DF8981001EBC10109E0C44400203D
:10DFA000A4770020383E0020BC120020044000204E
:10DFB00000EB0110827002F04BB800219DF8AC001C
:10DFC00040F2231210FB02F0FE4A02EBC000017186
:10DFD0009DF8AC0040F2231110FB01F0114601EB5B
:10DFE000C00018309DF8981001EBC10100EB011042
:10DFF000007808281DDC00219DF8AC0040F22312B7
:10E0000010FB02F0EF4A02EBC000017108229DF8FC
:10E01000AC0040F2231110FB01F0EA4901EBC00013
:10E0200018309DF8981001EBC10100EB011002704F
:10E0300024E09DF8AC0040F2231110FB01F0E1490F
:10E0400001EBC00018309DF8981001EBC10100EB06
:10E05000011000780B2811DC0C229DF8AC0040F276
:10E06000231110FB01F0D74901EBC00018309DF8D7
:10E07000981001EBC10100EB011002709DF8AC009B
:10E0800040F2231110FB01F0CE4901EBC000183023
:10E090009DF8981001EBC10100EB01104079A42814
:10E0A0002DD19DF8AC0000EB400101EB0010C649FA
:10E0B00001EB001030309DF8981000EB0110801C2F
:10E0C0000990007820F02000203009990870002283
:10E0D0009DF8AC0040F2231110FB01F0B94901EBAF
:10E0E000C00018309DF8981001EBC10100EB011041
:10E0F00080F83D209DF8AC100220FBF795FFA1228F
:10E100009DF8AC0040F2231110FB01F0AD4901EB8A
:10E11000C00018309DF8981001EBC10100EB011010
:10E12000427148E70020379015E09DF8AC0000EB05
:10E130004001C1EBC010A54901EBC001BDF8DC00F6
:10E14000C01C0A5C16A9BDF8DC000A54BDF8DC004E
:10E15000401C81B23791BDF8DC000628E5DB0621C2
:10E1600016A81FF0C1F80021CDE92E01DDE92E210E
:10E17000100A40EA0164A21841EB2120CDE90820F1
:10E180004FF480724FF00003DDE90801FAF71AF846
:10E190009DF8AC0040F2231110FB01F0894901EB1E
:10E1A000C00018309DF8981001EBC10100EB011080
:10E1B000027100209DF8AC1040F2231211FB02F115
:10E1C000804A02EBC101087104229DF8AC0040F2C4
:10E1D000231110FB01F07B4901EBC00018309DF8C2
:10E1E000981001EBC10100EB01100270A7229DF80D
:10E1F000AC0040F2231110FB01F0724901EBC000AA
:10E2000018309DF8981001EBC10100EB011042712C
:10E21000D1E69DF8AC0040F2231110FB01F06949F2
:10E2200001EBC00018309DF8981001EBC10100EB24
:10E230000110007804286ADA00219DF8AC0040F251
:10E24000231210FB02F05F4A02EBC0000171A12211
:10E250009DF8AC0040F2231110FB01F0594901EB8D
:10E26000C00118319DF8980000EBC00001EB0010D0
:10E2700042719DF8AC0040F2231110FB01F05149AE
:10E2800001EBC00118319DF8980000EBC00001EBD4
:10E29000001109910878401CC1B2099801709DF8DD
:10E2A000AC0040F2231110FB01F0464901EBC00025
:10E2B00018309DF8981001EBC10100EB01100078B7
:10E2C000042823D10A229DF8AC0040F2231110FB50
:10E2D00001F03C4901EBC00118319DF8980000EBBA
:10E2E000C00001EB00100270A3229DF8AC0040F2C8
:10E2F000231110FB01F0334901EBC00018309DF8E9
:10E30000981001EBC10100EB01104271ACE29DF8E5
:10E31000AC0040F2231110FB01F02A4901EBC000D0
:10E3200018309DF8981001EBC10100EB0110007846
:10E3300004282FD100219DF8AC0040F2231210FBDD
:10E3400002F0204A02EBC000017105229DF8AC00EA
:10E3500040F2231110FB01F01A4901EBC001183102
:10E360009DF8980000EBC00001EB00100270A322A2
:10E370009DF8AC0040F2231110FB01F0114901EBB4
:10E38000C00018309DF8981001EBC10100EB01109E
:10E39000427169E29DF8AC0040F2231110FB01F0DC
:10E3A000084901EBC00018309DF8981001EBC1013D
:10E3B00000EB01100078082837DC00219DF8AC0044
:10E3C00006E00000C444002004400020A4770020A0
:10E3D00040F2231210FB02F0FE4A02EBC000017172
:10E3E00009229DF8AC0040F2231110FB01F0F9491D
:10E3F00001EBC00118319DF8980000EBC00001EB63
:10E4000000100270A7229DF8AC0040F2231110FB0F
:10E4100001F0F04901EBC00018309DF8981001EBB5
:10E42000C10100EB011042711EE29DF8AC0040F208
:10E43000231110FB01F0E74901EBC00018309DF8F3
:10E44000981001EBC10100EB0110007809282FDCC6
:10E4500000219DF8AC0040F2231210FB02F0DD4ACF
:10E4600002EBC00001710A229DF8AC0040F22311BA
:10E4700010FB01F0D74901EBC00118319DF898005D
:10E4800000EBC00001EB00100270A3229DF8AC006D
:10E4900040F2231110FB01F0CE4901EBC00018300F
:10E4A0009DF8981001EBC10100EB01104271DBE116
:10E4B0009DF8AC0040F2231110FB01F0C54901EBBF
:10E4C000C00018309DF8981001EBC10100EB01105D
:10E4D00000780D282FDC00219DF8AC0040F22312BB
:10E4E00010FB02F0BB4A02EBC00001710E229DF846
:10E4F000AC0040F2231110FB01F0B64901EBC00162
:10E5000018319DF8980000EBC00001EB001002707C
:10E51000A1229DF8AC0040F2231110FB01F0AD499F
:10E5200001EBC00018309DF8981001EBC10100EB21
:10E530000110427198E19DF8AC0040F2231110FBEC
:10E5400001F0A44901EBC00018309DF8981001EBD0
:10E55000C10100EB011000780E282FDC00219DF88E
:10E56000AC0040F2231210FB02F09A4A02EBC0000A
:10E5700001710F229DF8AC0040F2231110FB01F055
:10E58000944901EBC00118319DF8980000EBC000E0
:10E5900001EB00100270A3229DF8AC0040F22311A1
:10E5A00010FB01F08B4901EBC00018309DF898106A
:10E5B00001EBC10100EB0110427155E19DF8AC0087
:10E5C00040F2231110FB01F0824901EBC00018302A
:10E5D0009DF8981001EBC10100EB011000781028A4
:10E5E0007EDC11229DF8AC0040F2231110FB01F0FB
:10E5F000784901EBC00118319DF8980000EBC0008C
:10E6000001EB00100270A1229DF8AC0040F2231132
:10E6100010FB01F06F4901EBC00103E025E153E17C
:10E62000A0E181E118319DF8980000EBC00001EBFA
:10E63000001042719DF8AC0040F2231110FB01F074
:10E64000644901EBC00118319DF8980000EBC0004F
:10E6500001EB001082709DF8AC0000EB400101EB73
:10E6600000105D4901EB001130319DF8980001EB7D
:10E670000010801C0990007820F0800080300999FB
:10E6800008709DF8AC0000EB400101EB001052490E
:10E6900001EB001030309DF8981000EB0110801C49
:10E6A0000990007820F00400001D099908709DF879
:10E6B000AC0000EB400101EB0010474901EB0010FA
:10E6C00030309DF8981000EB01108078C0F34010B6
:10E6D000F0B39DF8AC0000EB400101EB001000E04E
:10E6E0003EE03D4901EB001030309DF8981000EB02
:10E6F0000110801C0990007820F020020998027017
:10E700009DF8AC0000EB400101EB0010324901EB39
:10E71000001030309DF8981000EB01108078C0F3A5
:10E720004000B8B99DF8AC0000EB400101EB0010CF
:10E73000294901EB001030309DF8981000EB0110D2
:10E74000801C0990007820F008000830099900E04A
:10E750006CE008709DF8AC100220FBF765FC83E0CC
:10E760009DF8AC0040F2231110FB01F0194901EBB8
:10E77000C00118319DF8980000EBC00001EB0010BB
:10E7800001789DF8AC0040F2231210FB02F0114A10
:10E7900002EBC0004079814266D19DF8AC0040F2A6
:10E7A000231110FB01F0114601EBC00018309DF859
:10E7B000981001EBC10100EB01108078A12836D040
:10E7C000A3229DF8AC0040F2231110FB01F0014997
:10E7D00004E00000C44400200440002001EBC0011C
:10E7E00018319DF8980000EBC00001EB0010427159
:10E7F0009DF8AC0040F2231110FB01F0FE4901EB43
:10E80000C00018309DF8981001EBC10100EB011019
:10E810008078A22828D000209DF8AC1040F2231266
:10E8200011FB02F1F44A02EBC10108711CE0A122C4
:10E830009DF8AC0040F2231110FB01F0EE4901EB12
:10E84000C00118319DF8980000EBC00001EB0010EA
:10E85000427101219DF8AC0040F2231210FB02F03E
:10E86000E54A02EBC00001715BE4A1229DF8AC0017
:10E8700040F2231110FB01F0DF4901EBC001183118
:10E880009DF8980000EBC00001EB001082709DF82D
:10E89000AC0040F2231110FB01F0D74901EBC0019D
:10E8A00018319DF8980000EBC00001EB0010427198
:10E8B00000219DF8AC0040F2231210FB02F0CE4A7A
:10E8C00002EBC00001712CE400219DF8AC0040F285
:10E8D000231210FB02F0C84A02EBC00001710922AA
:10E8E0009DF8AC0040F2231110FB01F0C24901EB8E
:10E8F000C00118319DF8980000EBC00001EB00103A
:10E900000270A7229DF8AC0040F2231110FB01F029
:10E91000B94901EBC00018309DF8981001EBC10116
:10E9200000EB0110427173E400219DF8AC0040F24D
:10E93000231210FB02F0B04A02EBC0000171A722C3
:10E940009DF8AC0040F2231110FB01F0AA4901EB45
:10E95000C00018309DF8981001EBC10100EB0110C8
:10E96000427155E400219DF8AC0040F2231210FBE7
:10E9700002F0A14A02EBC0000171A7229DF8AC0091
:10E9800040F2231110FB01F09B4901EBC00118314B
:10E990009DF8980000EBC00001EB001042719DF85B
:10E9A000AC0000EB4001C1EBC010944901EBC0008A
:10E9B000407930287ED19DF8AC0040F2231110FB45
:10E9C00001F08D4901EBC00118319DF8980000EB72
:10E9D000C00001EB001001789DF8AC0040F223125A
:10E9E00010FB02F0844A02EBC0004079814261D101
:10E9F0009DF8AC0040F2231110FB01F0114601EB31
:10EA0000C00018309DF8981001EBC10100EB011017
:10EA1000C07831282ED19DF8AC0000EB400101EB0D
:10EA20000010A2F5986101EB001030309DF89810AD
:10EA300000EB0110801C0990007820F0200209985A
:10EA4000027000229DF8AC0040F2231110FB01F08F
:10EA5000694901EBC00118319DF8980000EBC00036
:10EA600001EB001080F83D209DF8AC100220FBF770
:10EA7000DBFA4EE09DF8AC0040F2231110FB01F0F0
:10EA80005D4901EBC00018309DF8981001EBC10101
:10EA900000EB0110C07833283BD19DF8AC0000EBAF
:10EAA000400101EB0010564901EB001030309DF899
:10EAB000981000E058E000EB0110801C09900078ED
:10EAC00020F020020998027001229DF8AC0040F26B
:10EAD000231110FB01F0484901EBC00018309DF8EC
:10EAE000981001EBC10100EB011080F83E20A92233
:10EAF0009DF8AC0040F2231110FB01F03E4901EB00
:10EB0000C00018309DF8981001EBC10100EB011016
:10EB100082709DF8AC0000EB400101EB0010384919
:10EB200001EB001030309DF8981000EB0110801CB4
:10EB30000990007820F00102099802709DF8AC005D
:10EB400000EB400101EB00102D4901EB00103030CB
:10EB50009DF8981000EB0110801C0990007820F0BF
:10EB60000202099802708BE39DF8AC0000EB4001B3
:10EB7000C1EBC010214901EBC000407931287DD1A3
:10EB80009DF8AC0040F2231110FB01F01A4901EB93
:10EB9000C00118319DF8980000EBC00001EB001097
:10EBA00001789DF8AC0040F2231210FB02F0124AEB
:10EBB00002EBC0004079814260D19DF8AC0040F288
:10EBC000231110FB01F0114601EBC00018309DF835
:10EBD000981001EBC10100EB011090F83E0078BBEA
:10EBE00001229DF8AC0040F2231110FB01F0024914
:10EBF00001EBC001183105E0C4440020A4770020D7
:10EC0000044000209DF8980000EBC00001EB0010CC
:10EC100080F83D209DF8AC1001EB410000EB0110A5
:10EC2000FE4901EB001130319DF8980001EB001016
:10EC3000801C0990007820F00100401C09990870A0
:10EC40009DF8AC1001EB410000EB0110F34901EB22
:10EC5000001030309DF8981000EB0110801C0990D6
:10EC6000007820F0020209980270ED4890F89007B1
:10EC7000002873D1EB4890F8290000E0BCE101289E
:10EC8000F7D1E848D0F80C02E649498D884265D2B0
:10EC90009DF8AC1040F2231011FB00F0E24901EBAB
:10ECA000C00018309DF8981001EBC10100EB011075
:10ECB00090F83D00012850D19DF8AC1040F223108F
:10ECC00011FB00F0D84901EBC00018309DF89810F6
:10ECD00001EBC10100EB011090F87E00E8BB0122BE
:10ECE0009DF8AC0000EB400101EB0010CB4901EBBB
:10ECF000001130319DF8980001EB0010C272002223
:10ED00009DF8AC0000EB400101EB0010C34901EBA2
:10ED1000001130319DF8980001EB001042604FF077
:10ED200010429DF8AC0040F2231110FB01F0BE49E7
:10ED300001EBC00118319DF8980000EBC00001EB19
:10ED4000001082609DF8AC1001EB410000EB011057
:10ED5000B24901EB0011303101E063E061E09DF860
:10ED6000980001EB001001789DF8AC0040F22312EE
:10ED700010FB02F0AC4A02EBC00041709DF8AC10F1
:10ED800040F2231011FB00F0114601EBC0011831D5
:10ED90009DF8980000EBC00001EB001001789DF891
:10EDA000AC0040F2231210FB02F09F4A02EBC000BD
:10EDB0004079814235D100229DF8AC0040F2231108
:10EDC00010FB01F0984901EBC00118319DF8980043
:10EDD00000EBC00001EB0010C271A4229DF8AC0052
:10EDE00040F2231110FB01F08F4901EBC0011831F3
:10EDF0009DF8980000EBC00001EB00108270A32288
:10EE00009DF8AC0040F2231110FB01F0864901EBA4
:10EE1000C00018309DF8981001EBC10100EB011003
:10EE200042712DE29DF8AC1040F2231011FB00F06E
:10EE30007D4901EBC00018309DF8981001EBC1012D
:10EE400000EB011090F83D0001287CD19DF8AC103A
:10EE500040F2231011FB00F0734901EBC00118319F
:10EE60009DF8980000EBC00001EB001090F87F10B7
:10EE700040F2231011FB00F06B4901EBC001183187
:10EE80009DF8AC0040F2231210FB02F0664A02EB40
:10EE9000C00018309DF8982002EBC20200EB02106F
:10EEA00090F8800000EBC00001EB001090F87700B4
:10EEB000032848D102229DF8AC0000EB400101EB91
:10EEC0000010564901EB001130319DF8980001EB1C
:10EED0000010C2724FF010429DF8AC0040F22311B6
:10EEE00010FB01F0504901EBC00118319DF898006A
:10EEF00000EBC00001EB001082609DF8AC1001EB4C
:10EF0000410000EB0110454901EB001130319DF843
:10EF1000980001EB001001789DF8AC0040F223123C
:10EF200010FB02F0404A02EBC00041709DF8AC10AB
:10EF300040F2231011FB00F0114601EBC001183123
:10EF40009DF8980000E097E100EBC00001EB001095
:10EF500001789DF8AC0040F2231210FB02F0324A17
:10EF600002EBC0004079814235D100229DF8AC000F
:10EF700040F2231110FB01F02B4901EBC0011831C5
:10EF80009DF8980000EBC00001EB0010C271A422B4
:10EF90009DF8AC0040F2231110FB01F0224901EB77
:10EFA000C00118319DF8980000EBC00001EB001083
:10EFB0008270A3229DF8AC0040F2231110FB01F0F7
:10EFC000194901EBC00018309DF8981001EBC10100
:10EFD00000EB0110427100229DF8AC0000EB4001F3
:10EFE00001EB00100D4901EB001030309DF8981036
:10EFF00000EB0110426043E19DF8AC1001EB4100D1
:10F00000C0EBC110094901EBC000407933287DD124
:10F010009DF8AC1001EB41000AE000000440002024
:10F02000BC320020BC120020C4440020A477002081
:10F0300000EB0110FE4901EB001030309DF89810F4
:10F0400000EB0110801C0990007820F00100401CAA
:10F05000099908709DF8AC1001EB410000EB01101C
:10F06000F34901EB001030309DF8981000EB0110CF
:10F07000801C0990007820F02002099802709DF809
:10F08000AC1001EB410000EB0110E94901EB00106D
:10F0900030309DF8981000EB0110801C099000782A
:10F0A00020F00200801C099908709DF8AC1040F215
:10F0B000231011FB00F0DF4901EBC00042799DF8FD
:10F0C000AC0040F2231110FB01F0DA4901EBC00063
:10F0D00018309DF8981001EBC10100EB011002708F
:10F0E0009DF8AC1001EB410000EB0110D04901EBA1
:10F0F000001030309DF8981000EB0110801C099032
:10F10000007820F080008030099900E02AE0087043
:10F110009DF8AC1001EB410000EB0110C44901EB7C
:10F12000001030309DF8981000EB01108078C0F38B
:10F13000400020B99DF8AC100220FAF775FFA2221A
:10F140009DF8AC0040F2231110FB01F0B94901EB2E
:10F15000C00018309DF8981001EBC10100EB0110C0
:10F1600082708DE09DF8AC0000EB4001C1EBC01057
:10F17000B14901EBC000407934287DD19DF8AC0045
:10F1800000EB400101EB0010A94901EB0010303009
:10F190009DF8981000EB0110801C0990007820F079
:10F1A0002002099802709DF8AC0000EB400101EBD1
:10F1B00000109F4901EB001030309DF8981000EBD3
:10F1C0000110801C0990007820F00202099802705A
:10F1D00001229DF8AC0040F2231110FB01F095498B
:10F1E00001EBC00118319DF8980000EBC00001EB65
:10F1F000001080F83E20A9229DF8AC0040F22311B7
:10F2000010FB01F08B4901EBC00118319DF898000B
:10F2100000EBC00001EB001082709DF8AC0040F2E2
:10F22000231110FB01F0834901EBC00042799DF8E6
:10F23000AC0040F2231110FB01F07E4901EBC0014C
:10F2400018319DF8980000EBC00001EB001002702F
:10F250009DF8AC0000EB400101EB0010744901EB9C
:10F26000001130319DF8980001EB0010801C0990CE
:10F27000007820F0800000E002E0803009990870FA
:10F2800000202C902D900021379122E0DDE92C10F8
:10F29000000140EA11720901CDE92C129DF8AC0081
:10F2A00000EB4001C1EBC010634901EBC001BDF8A8
:10F2B000DC00801D085C3038C117DDE92C341843B0
:10F2C00041EA0402CDE92C02BDF8DC00401C80B20A
:10F2D0003790BDF8DC000628D8DB9DF8AC002C99EF
:10F2E00040F2231210FB02F0524A02EBC002183225
:10F2F0009DF8980000EBC00002EB0010C0F81A1057
:10F3000000222C922D920021379122E0DDE92C1071
:10F31000000140EA11720901CDE92C129DF8AC0000
:10F3200000EB4001C1EBC010434901EBC001BDF847
:10F33000DC000D30085C3038C117DDE92C3418438F
:10F3400041EA0402CDE92C02BDF8DC00401C80B289
:10F350003790BDF8DC000428D8DB9DF8AC002C9970
:10F3600040F2231210FB02F0324A02EBC0021832C4
:10F370009DF8980000EBC00002EB001041630022F2
:10F380002C922D920021379122E0DDE92C10000112
:10F3900040EA11720901CDE92C129DF8AC0000EB96
:10F3A0004001C1EBC010244901EBC001BDF8DC00F5
:10F3B0001130085C3038C117DDE92C34184341EABC
:10F3C0000402CDE92C02BDF8DC00401C80B237906D
:10F3D000BDF8DC000628D8DB9DF8AC002C9940F283
:10F3E000231210FB02F0134A02EBC00218329DF800
:10F3F000980000EBC00002EB0010C0F81E109DF852
:10F40000AC0000EB4001C1EBC0100B4901EBC000A8
:10F4100042799DF8AC0040F2231110FB01F0054940
:10F4200001EBC00118319DF8980000EBC00005E029
:10F4300004400020C4440020A477002001EB001009
:10F44000C2709DF8AC0000EB400101EB0010FE49DA
:10F4500001EB001130319DF8980001EB001082782B
:10F460009DF8AC0040F2231110FB01F0F74901EBCD
:10F47000C00118319DF8980000EBC00001EB0010AE
:10F4800002769DF8AC0040F2231110FB01F0EF4929
:10F4900001EBC00118319DF8980000EBC00001EBB2
:10F4A000001001789DF8AC0040F2231210FB02F02E
:10F4B000E64A02EBC000407981427DDA9DF8AC005B
:10F4C00040F2231110FB01F0114601EBC00018308F
:10F4D0009DF8981001EBC10100EB011000780F2896
:10F4E0006ADD00219DF8AC0040F2231210FB02F00F
:10F4F000D64A02EBC0000171A7229DF8AC0040F291
:10F50000231110FB01F0D14901EBC00118319DF826
:10F51000980000EBC00001EB0010427101219DF842
:10F52000AC0040F2231210FB02F0C84A02EBC0000C
:10F5300001719DF8AC0040F2231110FB01F011465F
:10F5400001EBC00042799DF8AC0040F2231110FBA2
:10F5500001F0BE4901EBC00118319DF8980000EBA5
:10F56000C00001EB00100270A1229DF8AC0040F237
:10F57000231110FB01F0B54901EBC00118319DF8D2
:10F58000980000EBC00001EB001042719DF8AC0048
:10F5900000EB400101EB0010AB4901EB00113031F1
:10F5A0009DF8980001EB0010801C0990007820F075
:10F5B00080008030099900E078E008709DF8AC0088
:10F5C00000EB400101EB00109F4901EB00103030CF
:10F5D0009DF8981000EB0110801C0990007820F035
:10F5E0000400001D099908709DF8AC0000EB400173
:10F5F00001EB0010944901EB001030309DF8981099
:10F6000000EB01108078C0F3401088B99DF8AC0081
:10F6100000EB400101EB00108B4901EB0010303092
:10F620009DF8981000EB01108078C0F34000E8B31B
:10F630009DF8AC0000EB400101EB0010824901EBAA
:10F64000001030309DF8981000EB0110801C0990DC
:10F65000007820F02002099802709DF8AC0000EBC1
:10F66000400101EB0010784901EB001030309DF8AB
:10F67000981000EB0110801C0990007820F0020225
:10F68000099802709DF8AC0000EB400101EB0010FE
:10F690006D4901EB001030309DF8981000EB01101F
:10F6A000801C0990007820F0080000E0A3E00830FA
:10F6B000099908709DF8AC009DF8981001EB0010B6
:10F6C000C217CDE92C029DF8AC0040F2231110FBCB
:10F6D00001F15E4800EBC10018309DF8981001EB75
:10F6E000C10100EB0110223009902C9800EB400181
:10F6F000574800EB41110D3110220891DDE9080156
:10F70000F8F7A3FD9DF8AC0040F2231110FB01F0C7
:10F710004E4901EBC00118319DF8980000EBC00084
:10F7200001EB00112C9800EB4002494800EB42101D
:10F7300051F81A2F40F8012F496841609DF8AC003C
:10F7400000EB400101EB00103F4901EB00113031AB
:10F750009DF8980001EB001001782C9800EB400216
:10F760003B4800EB421001702C9800EB40013848F8
:10F7700000EB41113748C26841F81D2F008A88808C
:10F780009DF8AC0040F2231110FB01F02F4901EB72
:10F79000C00118319DF8980000EBC00001EB00108B
:10F7A000416B2C9800EB4002294800EB4210C0F856
:10F7B00009109DF8AC0000EB400101EB001022495C
:10F7C00001EB001130319DF8980001EB0010416809
:10F7D0002C9800EB40021E4800EB4210C0F82310AA
:10F7E0002C9881B208200991FAF71EFC9DF8AC1004
:10F7F0000220FAF719FCFDE300202C902D90002147
:10F8000037912DE0DDE92C10000140EA1172090169
:10F81000CDE92C129DF8AC0000EB4001C1EBC0100B
:10F820000D4901EBC001BDF8DC000B30085C30383D
:10F83000C117DDE92C34184341EA0402CDE92C025A
:10F84000BDF8DC00401C09E004400020C444002056
:10F85000D8140020BC310020A477002080B237905B
:10F86000BDF8DC000A28CDDB9DF8AC00DDE92C12E8
:10F8700040F2231310FB03F0FE4B03EBC0031833DD
:10F880009DF8980000EBC00003EB001040F8221F29
:10F89000426000222C922D920021379122E0DDE976
:10F8A0002C10000140EA11720901CDE92C129DF8DB
:10F8B000AC0000EB4001C1EBC010EF4901EBC0010F
:10F8C000BDF8DC001530085C3038C117DDE92C3498
:10F8D00040EA03022143CDE92C21BDF8DC00401CA5
:10F8E00081B23791BDF8DC000A28D8DB9DF8AC0066
:10F8F000DDE92C1240F2231310FB03F0DD4B03EB88
:10F90000C00318339DF8980000EBC00003EB001013
:10F9100022308160C26000219DF8AC0040F22312C9
:10F9200010FB02F0D34A02EBC00001719DF8AC005D
:10F9300040F2231110FB01F0114601EBC00018301A
:10F940009DF8981001EBC10100EB011000780C2824
:10F9500012DC0D229DF8AC0040F2231110FB01F0E7
:10F96000C44901EBC00018309DF8981001EBC101AB
:10F9700000EB0110027046E39DF8AC0040F2231149
:10F9800010FB01F0BB4901EBC00118319DF8980054
:10F9900000EBC00001EB001001789DF8AC0040F2D4
:10F9A000231210FB02F0B34A02EBC00040798142FF
:10F9B000E1D19DF8AC009DF8981001EB0010C21742
:10F9C000CDE92C02AD4890F8900708B39DF8AC0043
:10F9D00000EB400101EB0010A94901EB00103030B1
:10F9E0009DF8981000EB0110807A022810D09DF845
:10F9F000AC0000EB400101EB0010A14901EB00104D
:10FA000030309DF8981000EB0110C07A00287DDDA1
:10FA100000229DF8AC0000EB400101EB001098497A
:10FA200001EB001030309DF8981000EB0110C2720D
:10FA30009448D0F80C020521B0FBF1F201FB120052
:10FA400000EB40018F482C3000EB41100D30099045
:10FA50009DF8AC0040F2231110FB01F0854901EB49
:10FA6000C00018309DF8981001EBC10100EB0110A7
:10FA700022301022014608900998F8F7E6FB8148E9
:10FA8000D0F80C020521B0FBF1F201FB120000EBF3
:10FA900040017C482C3000EB41129DF8AC0040F254
:10FAA000231110FB01F0734901EBC00118319DF8DF
:10FAB000980000EBC00001EB001050F81A1F42F84C
:10FAC000011F406850606F48D0F80C020521B0FB60
:10FAD000F1F201FB120000EB40016A482C3000EB10
:10FAE00041129DF8AC0000EB400101EB00106449AD
:10FAF00001EB001130319DF8980001EB0010007807
:10FB000010706048D0F80C02052100E078E1B0FBED
:10FB1000F1F201FB120000EB40015A482C3000EBDF
:10FB200041129DF8AC0040F2231110FB01F0514945
:10FB300001EBC00118319DF8980000EBC00001EB0B
:10FB40000010406BC2F809004E48D0F80C020521A5
:10FB5000B0FBF1F201FB120000EB400149482C30F0
:10FB600000EB41114848C26841F81D2F008A888087
:10FB70004448D0F80C020521B0FBF1F201FB120061
:10FB800000EB40013F482C3000EB41129DF8AC00E7
:10FB900000EB400101EB0010394901EB001130315D
:10FBA0009DF8980001EB00104068C2F82300002285
:10FBB0009DF8AC0000EB400101EB0010304901EB77
:10FBC000001130319DF8980001EB001042600021D7
:10FBD00037914BE02B48D0F80C020521B0FBF1F235
:10FBE00001FB120000EB400126482C3000EB4111D4
:10FBF0002731BDF8DC409DF8AC0040F2231210FB29
:10FC000002F01C4A02EBC00218329DF8980000EB8B
:10FC1000C00002EB001090F87F0040F2231210FBAE
:10FC200002F0144A02EBC00218329DF8AC0040F218
:10FC3000231310FB03F00F4B03EBC00318339DF8A5
:10FC4000980000EBC00003EB001090F8800000EB80
:10FC5000C00002EB00123F32BDF8DC00001D105C5A
:10FC60000855BDF8DC00401C81B23791BDF8DC00BE
:10FC700006280BE0C4440020A4770020BC320020FA
:10FC800004400020BC120020BC310020A2DB002078
:10FC9000379039E000239DF8AC0040F2231110FBAF
:10FCA00001F0FE4901EBC00118319DF8980000EB0E
:10FCB000C00001EB001090F87F0040F2231110FB10
:10FCC00001F0F64901EBC00118319DF8AC0040F29B
:10FCD000231210FB02F0F14A02EBC00218329DF829
:10FCE000980000EBC00002EB001090F8800000EBE1
:10FCF000C00001EB00113F31BDF8DC000B54BDF832
:10FD0000DC00401C81B23791BDF8DC000A28C1DB61
:10FD1000E348D0F80C020521B0FBF1F080B20146B7
:10FD200009900220F9F7D4F900210620FAF77CF9AE
:10FD3000DB48D0F80C02DA49498D884206D2D8480F
:10FD4000D0F80C02401CD649C1F80C020021052055
:10FD5000FAF76AF99DF8AC0000EB400101EB0010E6
:10FD6000D04901EB001030309DF8981000EB0110E5
:10FD7000801C0990007820F0080209980270C84899
:10FD8000D0F80C020521B0FBF1F201FB120000EBF0
:10FD90004001C3482C3000EB4110D0F823202C98B0
:10FDA00000EB4001C04800EB4110C0F823200020C8
:10FDB000379020E0BA48D0F80C020521B0FBF1F2F0
:10FDC00001FB120000EB4001B5482C3000EB411064
:10FDD0002730BDF8DC10425C2C9800EB4001B248A3
:10FDE00000EB41112731BDF8DC000A54BDF8DC00FE
:10FDF000401C81B23791BDF8DC000628DADB56E002
:10FE00009DF8AC0000EB400101EB0010A54901EBAF
:10FE1000001030309DF8981000EB0110801C099004
:10FE2000007820F008000830099908709DF8AC00AF
:10FE300000EB400101EB00109A4901EB001030305B
:10FE40009DF8981000EB011042682C9800EB4001DF
:10FE5000954800EB4110C0F823200020379022E0A5
:10FE60009DF8AC0040F2231110FB01F08B4901EB2F
:10FE7000C00118319DF8980000EBC00001EB0011A3
:10FE80003F31BDF8DC000A5C2C9800EB400186484D
:10FE900000EB41112731BDF8DC000A54BDF8DC004D
:10FEA000401C81B23791BDF8DC000628D8DB002267
:10FEB0009DF8AC0040F2231110FB01F0774901EBF3
:10FEC000C00118319DF8980000EBC00001EB001054
:10FED00080F83E209DF8AC100220FAF7A5F89DF8B6
:10FEE000AC0040F2231110FB01F06C4901EBC001A2
:10FEF00018319DF8980000EBC00001EB0010223093
:10FF000009902C9800EB4001674800EB41100D3040
:10FF1000102208900999F8F798F99DF8AC0040F282
:10FF2000231110FB01F05D4901EBC00118319DF870
:10FF3000980000EBC00001EB00112C9800EB400290
:10FF4000594800EB421051F81A2F40F8012F496828
:10FF500041609DF8AC0000EB400101EB00105149FD
:10FF600001EB001130319DF8980001EB0010017891
:10FF70002C9800EB40024C4800EB421001702C988A
:10FF800000EB4001484800EB41114848C26841F885
:10FF90001D2F008A88809DF8AC0040F2231110FBD1
:10FFA00001F03E4901EBC00118319DF8980000EBCB
:10FFB000C00001EB0010416B2C9800EB40023A4866
:10FFC00000EB4210C0F809109DF8AC0000EB4001B6
:10FFD00001EB0010334901EB001130319DF898001E
:10FFE00001EB001041682C9800EB40022E4800EB1A
:10FFF000421000E02CE0C0F823102C9881B20820B9
:020000040801F1
:100000000991FAF711F8A7229DF8AC0040F22311EC
:1000100010FB01F0214901EBC00118319DF8980057
:1000200000EBC00001EB00104271A2229DF8AC0071
:1000300040F2231110FB01F0184901EBC000183009
:100040009DF8981001EBC10100EB0110827000BF18
:1000500000BF07F05DBC9DF8AC0000EB4001C1EBB8
:10006000C010134911F83000042801D124900BE08E
:100070009DF8AC0000EB4001C1EBC0100C4911F839
:100080003000152800D124909DF8AC0000EB400111
:10009000C1EBC010064901EBC0000BE0C4440020D6
:1000A000BC12002004400020D8140020BC310020E5
:1000B000A477002041789DF8AC0000EB4002C2EB31
:1000C000C010FE4A12F8300041EA002041F230012F
:1000D000884202D1A62024903DE09DF8AC0000EBC0
:1000E0004001C1EBC010F54901EBC00041789DF81B
:1000F000AC0000EB4002C2EBC010F04A12F8300036
:1001000041EA002041F23101884202D1A720249027
:1001100021E09DF8AC0000EB4001C1EBC010E749C5
:1001200011F83000022816D19DF8AC0000EB400118
:10013000C1EBC010E14901EBC00001799DF8AC00B2
:1001400000EB4002C2EBC010DC4A02EBC000C078FA
:1001500041EA002124919DF8AC0040F2231110FBEC
:1001600001F0D74901EBC000817826910021D54AE2
:100170009DF8AC0002EB00129DF898001154D24893
:1001800090F82800012815D19DF8AC0000EB400143
:1001900001EB0010CD4901EB001030309DF89810B4
:1001A00000EB0110801C0990007820F08000803066
:1001B00009990870BDF89000A7287DD007DC0428B5
:1001C0007BD015287AD0A62841F04B864BE0A0F5CD
:1001D0005850303820B1112871D01228F4D1FDE3E5
:1001E0009DF8AC0040F2231110FB01F0B44901EB83
:1001F000C00018309DF8981001EBC10100EB011010
:10020000007870BB00219DF8AC0040F2231210FB77
:1002100002F0AB4A02EBC000017101229DF8AC0074
:1002200040F2231110FB01F0A54901EBC001183188
:100230009DF8980000EBC00001EB00100270A722AF
:100240009DF8AC0040F2231110FB01F09C4901EB3A
:10025000C00018309DF8981001EBC10100EB0110AF
:10026000427101F0FEBD00219DF8AC0040F2231266
:1002700010FB02F0924A02EBC00001719DF8AC0045
:1002800040F2231110FB01F0114601EBC0001830C1
:100290009DF8981001EBC10100EB011000780228D5
:1002A00029DC03229DF8AC0040F2231110FB01F081
:1002B000834901EBC00103E0C6E030E15AE288E285
:1002C00018319DF8980000EBC00001EB001002709F
:1002D000A9229DF8AC0040F2231110FB01F07849EF
:1002E00001EBC00018309DF8981001EBC10100EB44
:1002F00001104271A7E09DF8AC0040F2231110FB01
:1003000001F06F4901EBC00018309DF8981001EB27
:10031000C10100EB01100078052824DC06229DF8BD
:10032000AC0040F2231110FB01F0654901EBC00164
:1003300018319DF8980000EBC00001EB001002702E
:10034000A2229DF8AC0040F2231110FB01F05C49A1
:1003500001EBC00018309DF8981001EBC10100EBD3
:10036000011042716FE09DF8AC0040F2231110FBC8
:1003700001F0534901EBC00018309DF8981001EBD3
:10038000C10100EB01104079A52815D19DF8AC0002
:1003900000EB400101EB00104C4901EB0010303044
:1003A0009DF8981000EB0110801C0990007820F057
:1003B0000400001D099908709DF8AC0040F223115B
:1003C00010FB01F03E4901EBC00018309DF8981079
:1003D00001EBC10100EB01108078A12833D09DF81A
:1003E000AC0040F2231110FB01F0354901EBC001D4
:1003F00018319DF8980000EBC00001EB00108278E6
:100400009DF8AC0040F2231110FB01F02C4901EBE8
:10041000C00118319DF8980000EBC00001EB0010FE
:100420004271A1229DF8AC0040F2231110FB01F0B3
:10043000234901EBC00018309DF8981001EBC10171
:1004400000EB011082700CE79DF8AC0040F2231124
:1004500010FB01F01A4901EBC00018309DF898100C
:1004600001EBC10100EB01104079A42839D19DF8BE
:10047000AC0000EB400101EB0010144901EB00104F
:1004800030309DF8981000EB0110801C0990007826
:1004900020F0200020300999087000229DF8AC005F
:1004A00040F2231110FB01F0054901EBC0001830A8
:1004B0009DF8981001EBC1010AE00000A47700202C
:1004C000C4440020383E0020BC120020044000201C
:1004D00000EB011080F83D209DF8AC100220F9F7E8
:1004E000A3FD00219DF8AC0040F2231210FB02F0A6
:1004F000FE4A02EBC0000171A1229DF8AC0040F25F
:10050000231110FB01F0F94901EBC00018309DF8F0
:10051000981001EBC10100EB01104271A1E69DF8BA
:10052000AC0040F2231110FB01F0F04901EBC000D8
:1005300018309DF8981001EBC10100EB0110007814
:1005400001282FDC00219DF8AC0040F2231210FBA3
:1005500002F0E64A02EBC000017102229DF8AC00F5
:1005600040F2231110FB01F0E04901EBC00118310A
:100570009DF8980000EBC00001EB00100270A32270
:100580009DF8AC0040F2231110FB01F0D74901EBBC
:10059000C00018309DF8981001EBC10100EB01106C
:1005A0004271E6E09DF8AC0040F2231110FB01F02F
:1005B000CE4901EBC00018309DF8981001EBC10145
:1005C00000EB0110007804282FDC00219DF8AC001E
:1005D00040F2231210FB02F0C44A02EBC00001718A
:1005E00005229DF8AC0040F2231110FB01F0BF4939
:1005F00001EBC00118319DF8980000EBC00001EB41
:1006000000100270A3229DF8AC0040F2231110FBF1
:1006100001F0B64901EBC00018309DF8981001EBCD
:10062000C10100EB01104271A3E09DF8AC0040F263
:10063000231110FB01F0AD4901EBC00018309DF80B
:10064000981001EBC10100EB01100078062812DCC4
:10065000A1229DF8AC0040F2231110FB01F0A34948
:1006600001EBC00018309DF8981001EBC10100EBC0
:10067000011042717DE09DF8AC0040F2231110FBA7
:1006800001F09A4901EBC00118319DF8980000EB88
:10069000C00001EB001001789DF8AC0040F223127D
:1006A00010FB02F0914A02EBC0004079814260D118
:1006B0009DF8AC0040F2231110FB01F0114601EB54
:1006C000C00018309DF8981001EBC10100EB01103B
:1006D0008078A12830D0A3229DF8AC0040F22311ED
:1006E00010FB01F0814901EBC00118319DF8980021
:1006F00000EBC00001EB001042719DF8AC0040F22D
:10070000231110FB01F0794901EBC00018309DF86E
:10071000981001EBC10100EB01108078A22828D0CD
:1007200000209DF8AC1040F2231211FB02F16F4A39
:1007300002EBC10108711CE0A1229DF8AC0040F25F
:10074000231110FB01F0694901EBC00118319DF83C
:10075000980000EBC00001EB0010427101219DF8F0
:10076000AC0040F2231210FB02F0604A02EBC00022
:10077000017176E5A1229DF8AC0040F2231110FB37
:1007800001F05A4901EBC00118319DF8980000EBC7
:10079000C00001EB001042719DF8AC0040F2231143
:1007A00010FB01F0514901EBC00118319DF8980090
:1007B00000EBC00001EB0010827000219DF8AC003E
:1007C00040F2231210FB02F0484A02EBC000017114
:1007D00047E500219DF8AC0040F2231210FB02F027
:1007E000424A02EBC0000171A7229DF8AC0040F222
:1007F000231110FB01F03D4901EBC00118319DF8B8
:10080000980000EBC00001EB001042719DF8AC00B5
:1008100000EB4001C1EBC010354901EBC00040794D
:10082000302862D19DF8AC0040F2231110FB01F09A
:100830002E4901EBC00118319DF8980000EBC00073
:1008400001EB001001789DF8AC0040F2231210FB80
:1008500002F0264A02EBC0004079814245D19DF862
:10086000AC0000EB400101EB0010A2F5986101EB38
:10087000001030309DF8981000EB0110801C09909A
:10088000007820F00102099802709DF8AC0000EB9E
:10089000400101EB0010174901EB001030309DF8CA
:1008A000981000EB0110801C0990007820F00202E3
:1008B000099802709DF8AC0040F2231110FB01F082
:1008C0000A4901EBC00018309DF8981001EBC101F6
:1008D00000EB0110C078312834D19DF8AC0000EB5A
:1008E000400101EB0010034906E052E0C44400203F
:1008F000A47700200440002001EB001030309DF868
:10090000981000EB0110801C0990007820F0200264
:100910000998027000229DF8AC0040F2231110FBF0
:1009200001F0FE4901EBC00018309DF8981001EB72
:10093000C10100EB011080F83D209DF8AC100220B1
:10094000F9F772FB9DF8AC0040F2231110FB01F0A7
:10095000F24901EBC00018309DF8981001EBC1017D
:1009600000EB011090F83E00012811D1A9229DF85A
:10097000AC0040F2231110FB01F0E84901EBC0008C
:1009800018309DF8981001EBC10100EB0110827046
:1009900085E39DF8AC0000EB4001C1EBC010E049DD
:1009A00001EBC000407931287ED19DF8AC0040F2C7
:1009B000231110FB01F0D94901EBC00118319DF85A
:1009C000980000EBC00001EB001001789DF8AC002E
:1009D00040F2231210FB02F0D04A00E0FEE302EBEB
:1009E000C000407981425FD19DF8AC0040F22311F4
:1009F00010FB01F0114601EBC00018309DF8981073
:100A000001EBC10100EB011090F83E0040BB012258
:100A10009DF8AC0040F2231110FB01F0BF4901EB3F
:100A2000C00118319DF8980000EBC00001EB0010E8
:100A300080F83D209DF8AC0000EB400101EB001078
:100A4000B84901EB001130319DF8980001EB00101E
:100A5000801C0990007820F00100401C0999087062
:100A60009DF8AC0000EB400101EB0010AD4901EB3B
:100A7000001030309DF8981000EB0110801C099098
:100A8000007820F0020209980270A74890F89007B9
:100A9000002874D1A54890F829000128F9D1A3486D
:100AA000D0F80C02A14900E0C1E1498D884266D22C
:100AB0009DF8AC0040F2231110FB01F0974901EBC7
:100AC000C00018309DF8981001EBC10100EB011037
:100AD00090F83D00012851D19DF8AC0040F223115F
:100AE00010FB01F08D4901EBC00018309DF8981003
:100AF00001EBC10100EB011090F87E00F0BB012278
:100B00009DF8AC0000EB400101EB0010854901EBC2
:100B1000001130319DF8980001EB0010C2724FF0C7
:100B200010429DF8AC0040F2231110FB01F07B490C
:100B300001EBC00118319DF8980000EBC00001EBFB
:100B4000001082609DF8AC0000EB400101EB00104A
:100B5000744901EB001130319DF8980001EB001051
:100B600001789DF8AC0040F2231210FB02F06B4AB2
:100B700002EBC00041709DF8AC0001E062E0F3E0E0
:100B800040F2231110FB01F0114601EBC0011831B6
:100B90009DF8980000EBC00001EB001001789DF873
:100BA000AC0040F2231210FB02F05C4A02EBC000E2
:100BB0004079814235D100229DF8AC0040F22311EA
:100BC00010FB01F0554901EBC00118319DF8980068
:100BD00000EBC00001EB0010C271A4229DF8AC0034
:100BE00040F2231110FB01F04C4901EBC001183118
:100BF0009DF8980000EBC00001EB00108270A3226A
:100C00009DF8AC0040F2231110FB01F0434901EBC9
:100C1000C00018309DF8981001EBC10100EB0110E5
:100C2000427100229DF8AC0000EB400101EB001086
:100C30003C4901EB001030309DF8981000EB01109A
:100C400042602CE29DF8AC0040F2231110FB01F051
:100C5000324901EBC00018309DF8981001EBC1013A
:100C600000EB011090F83D0001287DD19DF8AC000B
:100C700040F2231110FB01F0284901EBC0011831AB
:100C80009DF8980000EBC00001EB001090F87F0089
:100C900040F2231110FB01F0204901EBC001183193
:100CA0009DF8AC0040F2231210FB02F01B4A02EB4D
:100CB000C00018309DF8982002EBC20200EB021031
:100CC00090F8800000EBC00001EB001090F8770076
:100CD000032849D102229DF8AC0000EB400101EB52
:100CE0000010104901EB001130319DF8980001EB24
:100CF0000010C2724FF010429DF8AC0040F2231178
:100D000010FB01F0054901EBC00118319DF8980076
:100D100000EBC00001EB0010826009E0C444002039
:100D2000A477002004400020BC320020BC12002028
:100D30009DF8AC0000EB400101EB0010FA4901EB1B
:100D4000001130319DF8980001EB001001789DF8FA
:100D5000AC0040F2231210FB02F0F44A02EBC00098
:100D600041709DF8AC0000E096E140F2231110FBC9
:100D700001F0114601EBC00118319DF8980000EB1D
:100D8000C00001EB001001789DF8AC0040F2231286
:100D900010FB02F0E54A02EBC0004079814235D1F8
:100DA00000229DF8AC0040F2231110FB01F0DF4956
:100DB00001EBC00118319DF8980000EBC00001EB79
:100DC0000010C271A4229DF8AC0040F2231110FB68
:100DD00001F0D64901EBC00118319DF8980000EBF5
:100DE000C00001EB00108270A3229DF8AC0040F21D
:100DF000231110FB01F0CD4901EBC00018309DF824
:100E0000981001EBC10100EB0110427100229DF826
:100E1000AC0000EB400101EB0010C34901EB0010F6
:100E200030309DF8981000EB0110426037E19DF8DA
:100E3000AC0000EB4001C1EBC010BD4901EBC000AC
:100E4000407933287ED19DF8AC0000EB400101EBE6
:100E50000010B54901EB001030309DF8981000EB00
:100E60000110801C0990007820F00100401C0999B5
:100E700008709DF8AC0000EB400101EB0010AA499E
:100E800001EB001030309DF8981000EB0110801C31
:100E90000990007820F02002099802709DF8AC00BB
:100EA00000EB400101EB00109F4901EB00103030D6
:100EB0009DF8981000EB0110801C0990007820F03C
:100EC0000200801C099908709DF8AC0040F22311C3
:100ED00010FB01F0954901EBC00042799DF8AC0090
:100EE00040F2231110FB01F0904901EBC0001830D3
:100EF0009DF8981001EBC10100EB011002709DF804
:100F0000AC0000EB400101EB0010874901EB001041
:100F100030309DF8981000EB0110801C099000788B
:100F200020F080008030099908709DF8AC0000EB3B
:100F3000400101EB00107C4901EB001030309DF8BE
:100F4000981000E01DE000EB01108078C0F3400035
:100F500020B99DF8AC100220F9F766F8A2229DF89E
:100F6000AC0040F2231110FB01F0704901EBC0000E
:100F700018309DF8981001EBC10100EB0110827050
:100F80008DE09DF8AC0000EB4001C1EBC01068495A
:100F900001EBC000407934287ED19DF8AC0000EB15
:100FA000400101EB0010604901EB001030309DF86A
:100FB000981000EB0110801C0990007820F02002AE
:100FC000099802709DF8AC0000EB400101EB0010A5
:100FD000554901EB001030309DF8981000EB0110DE
:100FE000801C0990007820F002020998027001220A
:100FF0009DF8AC0040F2231110FB01F04B4901EBCE
:10100000C00018309DF8981001EBC10100EB0110F1
:1010100080F83E20A9229DF8AC0040F2231110FB7D
:1010200001F0424901EBC00018309DF8981001EB27
:10103000C10100EB011082709DF8AC0040F2231159
:1010400010FB01F0394901EBC00042799DF8AC007A
:1010500040F2231110FB01F0344901EBC0001830BD
:101060009DF8981001EBC10100EB011002709DF892
:10107000AC0000EB400101EB00102B4901EB00102C
:1010800030309DF8981000EB0110801C099000781A
:1010900020F08000803000E001E009990870002015
:1010A0002C902D900021379121E0DDE92C100001DA
:1010B00040EA11720901CDE92C129DF8AC0000EB59
:1010C0004001C1EBC0101A4901EBC001BDF8DC00C2
:1010D000801D085C3038C117DDE92C240243214310
:1010E000CDE92C21BDF8DC00401C81B23791BDF860
:1010F000DC000828D9DB9DF8AC002C9940F22312C3
:1011000010FB02F0094A02EBC00218329DF8980069
:1011100000EBC00002EB0010C0F81A1000222C9265
:101120002D920021379128E004400020C444002083
:10113000A4770020DDE92C10000140EA11720901BA
:10114000CDE92C129DF8AC0000EB4001C1EBC010C2
:10115000FE4901EBC001BDF8DC000F30085C3038FF
:10116000C117DDE92C34184341EA0402CDE92C0211
:10117000BDF8DC00401C80B23790BDF8DC000628CA
:10118000D8DB9DF8AC002C9940F2231210FB02F042
:10119000EF4A02EBC00218329DF8980000EBC00045
:1011A00002EB0010416300222C922D920021379116
:1011B00024E0DDE92C10000140EA11720901CDE9BB
:1011C0002C129DF8AC0000EB4001C1EBC010DF49D0
:1011D00001EBC001BDF8DC00153000E000E2085C66
:1011E0003038C117DDE92C34184341EA0402CDE957
:1011F0002C02BDF8DC00401C80B23790BDF8DC004A
:101200000828D6DB9DF8AC002C9940F2231210FB85
:1012100002F0CF4A02EBC00218329DF8980000EBB2
:10122000C00002EB0010C0F81E109DF8AC0000EBEF
:101230004001C1EBC010C54901EBC00042799DF8E7
:10124000AC0040F2231110FB01F0C14901EBC001D9
:1012500018319DF8980000EBC00001EB0010C2703F
:101260009DF8AC0000EB400101EB0010B94901EB27
:10127000001130319DF8980001EB001082789DF844
:10128000AC0040F2231110FB01F0B14901EBC001A9
:1012900018319DF8980000EBC00001EB00100276B9
:1012A0009DF8AC0040F2231110FB01F0A84901EBBE
:1012B000C00118319DF8980000EBC00001EB001050
:1012C00001789DF8AC0040F2231210FB02F0A04A16
:1012D00002EBC000407981427EDA00219DF8AC002B
:1012E00040F2231210FB02F0994A02EBC000017198
:1012F000A7229DF8AC0040F2231110FB01F09449A5
:1013000001EBC00118319DF8980000EBC00001EB23
:101310000010427101219DF8AC0040F2231210FB35
:1013200002F08B4A02EBC00001719DF8AC0040F264
:10133000231110FB01F0114601EBC00042799DF82A
:10134000AC0040F2231110FB01F0814901EBC00118
:1013500018319DF8980000EBC00001EB00100270FE
:10136000A1229DF8AC0040F2231110FB01F0784956
:1013700001EBC00118319DF8980000EBC00001EBB3
:10138000001042719DF8AC0000EB400101EB001031
:10139000704901EB001130319DF8980001EB00100D
:1013A000801C0990007820F0800080300999087036
:1013B0009DF8AC0000EB400101EB0010654901EB2A
:1013C000001030309DF8981000EB0110801C09903F
:1013D000007820F0040000E052E0001D0999087038
:1013E0009DF8AC0000EB400101EB0010594901EB06
:1013F000001030309DF8981000EB01108078C0F399
:101400004010E8B39DF8AC0000EB400101EB001088
:10141000504901EB001030309DF8981000EB01109E
:10142000801C0990007820F02002099802709DF835
:10143000AC0000EB400101EB0010464901EB00104D
:1014400030309DF8981000EB01108078C0F3400018
:10145000E8BB9DF8AC0000EB400101EB00103D49FA
:1014600001EB001030309DF8981000EB0110801C4B
:101470000990007820F0080108310998017000E017
:10148000ADE09DF8AC109DF8980000EB0110C2177C
:10149000CDE92C029DF8AC0040F2231110FB01F0C5
:1014A0002B4901EBC00018309DF8981001EBC101E9
:1014B00000EB0110223009902C9800EB40012648E7
:1014C00000EB41100D3010220890099900E081E0F6
:1014D000F6F7BBFE9DF8AC0040F2231110FB01F0C3
:1014E0001B4901EBC00118319DF8980000EBC000CA
:1014F00001EB00112C9800EB4002174800EB421062
:1015000051F81A2F40F8012F496841609DF8AC004E
:1015100000EB400101EB00100E4901EB00113031EE
:101520009DF8980001EB001001782C9800EB400228
:10153000094800EB421001702C9800EB400106486E
:1015400000EB41110548C2680AE00000A4770020C2
:10155000C444002004400020D8140020BC310020E6
:1015600041F81D2F008A88809DF8AC0040F22311BD
:1015700010FB01F0FE4901EBC00118319DF8980005
:1015800000EBC00001EB0010416B2C9800EB400217
:10159000F84800EB4210C0F809109DF8AC0000EBD1
:1015A000400101EB0010F44901EB001130319DF8CE
:1015B000980001EB001041682C9800EB4002ED48C8
:1015C00000EB4210C0F823102C9881B2082009913A
:1015D000F8F72AFD9DF8AC100220F8F725FDE2E3AC
:1015E00000202C902D900021379122E0DDE92C1075
:1015F000000140EA11720901CDE92C129DF8AC00FE
:1016000000EB4001C1EBC010DC4901EBC001BDF8AB
:10161000DC000B30085C3038C117DDE92C3418438E
:1016200041EA0402CDE92C02BDF8DC00401C80B286
:101630003790BDF8DC000C28D8DB9DF8AC00DDE964
:101640002C2140F2231310FB03F0C94B03EBC00322
:1016500018339DF8980000EBC00003EB001040F831
:10166000222F416000222C922D920021379122E0FE
:10167000DDE92C10000140EA11720901CDE92C12BC
:101680009DF8AC0000EB4001C1EBC010BB4901EB81
:10169000C001BDF8DC001730085C3038C117DDE947
:1016A0002C34184341EA0402CDE92C02BDF8DC00D9
:1016B000401C80B23790BDF8DC000C28D8DB9DF8C8
:1016C000AC00DDE92C1240F2231310FB03F0A84B11
:1016D00003EBC00318339DF8980000EBC00003EB48
:1016E000001022308160C26000219DF8AC0040F201
:1016F000231210FB02F09E4A02EBC00001719DF81C
:10170000AC0040F2231110FB01F0114601EBC000C8
:1017100018309DF8981001EBC10100EB0110007822
:10172000032812DC04229DF8AC0040F2231110FBC8
:1017300001F08F4901EBC00018309DF8981001EBC3
:10174000C10100EB0110027053E39DF8AC0040F2C0
:10175000231110FB01F0864901EBC00118319DF8FF
:10176000980000EBC00001EB001001789DF8AC0080
:1017700040F2231210FB02F07D4A02EBC0004079D8
:101780008142E1D19DF8AC009DF8981001EB00106A
:10179000C217CDE92C027A4890F8900708B39DF85B
:1017A000AC0000EB400101EB0010734901EB0010AD
:1017B00030309DF8981000EB0110807A022810D08C
:1017C0009DF8AC0000EB400101EB00106A4901EB11
:1017D000001030309DF8981000EB0110C07A0028FE
:1017E0007DDD00229DF8AC0000EB400101EB001014
:1017F000614901EB001030309DF8981000EB0110AA
:10180000C2726048D0F80C020521B0FBF1F201FB76
:10181000120000EB40015B482C3000EB41100D3012
:1018200009909DF8AC1040F2231011FB00F05049D4
:1018300001EBC00018309DF8981001EBC10100EBDE
:10184000011022301022014608900998F6F7FDFC9D
:101850004C48D0F80C020521B0FBF1F201FB12005C
:1018600000EB400147482C3000EB41129DF8AC00E2
:1018700040F2231110FB01F03D4901EBC00118318A
:101880009DF8980000EBC00001EB001050F81A1F03
:1018900042F8011F406850603A48D0F80C02052118
:1018A000B0FBF1F201FB120000EB400135482C3097
:1018B00000EB41129DF8AC0000EB400101EB001081
:1018C0002D4901EB001130319DF8980001EB00101B
:1018D000007810702B48D0F80C02052100E07BE165
:1018E000B0FBF1F201FB120000EB400125482C3067
:1018F00000EB41129DF8AC0040F2231110FB01F007
:101900001B4901EBC00118319DF8980000EBC000A5
:1019100001EB0010406BC2F809001A48D0F80C0225
:101920000521B0FBF1F201FB120000EB400115486C
:101930002C3000EB41111448C26841F81D2F008A79
:1019400088801048D0F80C020521B0FBF1F201FBB1
:10195000120000EB40010B482C3000EB41129DF8C7
:10196000AC0000EB400101EB001003490EE0000069
:10197000C4440020D814002004400020A477002094
:10198000BC320020BC120020BC31002001EB001151
:1019900030319DF8980001EB00104068C2F8230038
:1019A00000229DF8AC0000EB400101EB0010FE4965
:1019B00001EB001130319DF8980001EB00104260FE
:1019C000002137914BE0F948D0F80C020521B0FB1B
:1019D000F1F201FB120000EB4001F4482C3000EB67
:1019E00041112731BDF8DC409DF8AC0040F22312D4
:1019F00010FB02F0EE4A02EBC00218329DF898008C
:101A000000EBC00002EB001090F87F0040F22312C0
:101A100010FB02F0E64A02EBC00218329DF8AC005F
:101A200040F2231310FB03F0E14B03EBC003183328
:101A30009DF8980000EBC00003EB001090F88000C8
:101A400000EBC00002EB00123F32BDF8DC00001DCD
:101A5000105C0855BDF8DC00401C81B23791BDF820
:101A6000DC000628AFDB0020379039E000239DF82A
:101A7000AC0040F2231110FB01F0CD4901EBC00195
:101A800018319DF8980000EBC00001EB001090F8B1
:101A90007F0040F2231110FB01F0C54901EBC001AA
:101AA00018319DF8AC0040F2231210FB02F0C04A3E
:101AB00002EBC00218329DF8980000EBC00002EB68
:101AC000001090F8800000EBC00001EB00113F31E6
:101AD000BDF8DC000B54BDF8DC00401C81B237912E
:101AE000BDF8DC000A28C1DBB048D0F80C020521A3
:101AF000B0FBF1F080B2014609900220F7F7E8FA56
:101B000000210620F8F790FAA848D0F80C02A7495F
:101B1000498D884206D2A548D0F80C02401CA34942
:101B2000C1F80C0200210520F8F77EFA9DF8AC0000
:101B300000EB400101EB00109B4901EB001030303D
:101B40009DF8981000EB0110801C0990007820F09F
:101B50000802099802709548D0F80C020521B0FBE4
:101B6000F1F201FB120000EB400190482C3000EB39
:101B70004110D0F823202C9800EB40018D4800EB59
:101B80004110C0F823200020379020E08748D0F88B
:101B90000C020521B0FBF1F201FB120000EB400149
:101BA00082482C3000EB41102730BDF8DC10425C3D
:101BB0002C9800EB40017F4800EB41112731BDF824
:101BC000DC000A54BDF8DC00401C81B23791BDF83E
:101BD000DC000628DADB56E09DF8AC0000EB4001A3
:101BE00001EB0010704901EB001030309DF89810A7
:101BF00000EB0110801C0990007820F008000830EC
:101C0000099908709DF8AC0000EB400101EB001051
:101C1000654901EB001030309DF8981000EB011081
:101C200042682C9800EB4001624800EB4110C0F87C
:101C300023200020379022E09DF8AC0040F22311D1
:101C400010FB01F05A4901EBC00118319DF89800D2
:101C500000EBC00001EB00113F31BDF8DC000A5C75
:101C60002C9800EB4001534800EB41112731BDF89F
:101C7000DC000A54BDF8DC00401C81B23791BDF88D
:101C8000DC000628D8DB00229DF8AC0040F22311CE
:101C900010FB01F0464901EBC00118319DF8980096
:101CA00000EBC00001EB001080F83E209DF8AC1066
:101CB0000220F8F7B9F99DF8AC0040F2231110FBAF
:101CC00001F03B4901EBC00118319DF8980000EB91
:101CD000C00001EB0010223009902C9800EB40016D
:101CE000344800EB41100D30102208900999F6F7A6
:101CF000ACFA9DF8AC0040F2231110FB01F02C4926
:101D000001EBC00118319DF8980000EBC00001EB19
:101D100000112C9800EB4002264800EB421051F8CD
:101D20001A2F40F8012F496841609DF8AC0000EB84
:101D3000400101EB00101C4901EB001130319DF80E
:101D4000980001EB001001782C9800EB4002194834
:101D500000EB421001702C9800EB4001154800EB9D
:101D600041111548C26841F81D2F008A88809DF8EE
:101D7000AC0040F2231110FB01F00D4901EBC00152
:101D800018319DF8980000EBC00001EB0010416B8A
:101D90002C9800EB4002074800EB4210C0F80910F5
:101DA0009DF8AC000AE05CE004400020BC1200207A
:101DB000C4440020D8140020BC31002000EB4001B6
:101DC00001EB0010FE4901EB001130319DF8980045
:101DD00001EB001041682C9800EB4002F94800EB41
:101DE0004210C0F823102C9881B208200991F8F70E
:101DF0001BF900229DF8AC0040F2231110FB01F00A
:101E0000F14901EBC00118319DF8980000EBC000CA
:101E100001EB001080F83E20A7229DF8AC0040F2B4
:101E2000231110FB01F0E84901EBC00118319DF8C6
:101E3000980000EBC00001EB00104271A2229DF857
:101E4000AC0040F2231110FB01F0DF4901EBC000B0
:101E500018309DF8981001EBC10100EB0110827061
:101E600000BF00BF05F054BD0021D84A9DF8AC006A
:101E700002EB00129DF8980011549DF8AC0000EBA5
:101E80004001C1EBC010D24901EBC000407870287E
:101E90000ED19DF8AC0000EB4001C1EBC010CC4965
:101EA00001EBC0008078FA2802D1B120249042E0F2
:101EB0009DF8AC0000EB4001C1EBC010C44901EB40
:101EC000C000407800F0F000C0280ED19DF8AC00B2
:101ED00000EB4001C1EBC010BD4901EBC0008078B0
:101EE000FA2802D1B620249025E09DF8AC0000EB42
:101EF0004001C1EBC010B64911F8300000F0F0000D
:101F0000502818D19DF8AC0000EB4001C1EBC01087
:101F1000AF4901EBC000407800F0F00030280AD152
:101F20009DF8AC0000EB4001C1EBC010A84901EBEB
:101F3000C000817824919DF8AC0040F2231110FB81
:101F400001F0A14901EBC0008178269100219F4A50
:101F50009DF8AC0002EB00129DF8980011549D48CA
:101F600090F82800012815D19DF8AC0000EB400145
:101F700001EB0010924901EB001030309DF89810F1
:101F800000EB0110801C0990007820F08000803068
:101F900009990870BDF89000652874D004DC012808
:101FA00009D0032805D175E0B12802D0B62800D1A8
:101FB00000E085E184E19DF8AC0000EB4001C1EB5D
:101FC000C010834901EBC0000079012806D0022827
:101FD00005D0032804D005285AD102E058E057E084
:101FE00056E09DF8AC0040F2231110FB01F0764959
:101FF00001EBC00018309DF8981001EBC10100EB17
:1020000001100078F0BB00219DF8AC0040F22312D3
:1020100010FB02F06C4A02EBC000017101229DF836
:10202000AC0040F2231110FB01F0674901EBC00145
:1020300018319DF8980000EBC00001EB0010027011
:10204000B6229DF8AC0040F2231110FB01F05E496E
:1020500001EBC00118319DF8980000EBC00001EBC6
:1020600000104271B2229DF8AC0040F2231110FB27
:1020700001F0554901EBC00018309DF8981001EBB4
:10208000C10101E003E02DE000EB0110827000BF10
:1020900000BF15E19DF8AC0000EB4001C1EBC010A2
:1020A0004B4901EBC000C1794B4880F8041D9DF8F5
:1020B000AC0000EB400101EB0010414901EB0011C5
:1020C00030319DF8980001EB0010801C09904248C7
:1020D00090F8040DC2080998007862F3000009998D
:1020E0000870EDE09DF8AC0000EB4001C1EBC010C2
:1020F000374901EBC000007900F0F00010B9B820BA
:10210000249001E0B92024909DF8AC0000EB400140
:10211000C1EBC0102E4901EBC000007900F00F01A7
:1021200025910021379120E09DF8AC0000EB4001A3
:1021300001EB0010224901EB00113031BDF8DC0049
:1021400001EB001041789DF8AC0000EB4002C2EBBF
:10215000C0101F4A12F830005038814200D112E0FE
:10216000BDF8DC00401C81B237919DF8AC0000EB5B
:10217000400101EB0010124901EB0010C179BDF8DC
:10218000DC008142D0DC00BFBDF8DC109DF894007B
:102190000844C1B226919DF8AC0040F2231110FB17
:1021A00001F0094901EBC00018309DF8981001EBCF
:1021B000C10100EB0110007801283ED100210DE0A3
:1021C00004400020D8140020C4440020383E0020E1
:1021D000A4770020BC120020BC2200209DF8AC0097
:1021E00040F2231210FB02F0FE4A02EBC000017124
:1021F00002229DF8AC0040F2231110FB01F0F949D6
:1022000001EBC00118319DF8980000EBC00001EB14
:1022100000100270B9229DF8AC0040F2231110FBAF
:1022200001F0F04901EBC00018309DF8981001EB67
:10223000C10100EB0110427141E09DF8AC0040F299
:10224000231110FB01F0E74901EBC00018309DF8A5
:10225000981001EBC10100EB0110007801282ED18C
:1022600000219DF8AC0040F2231210FB02F0DD4A81
:1022700002EBC000017102229DF8AC0040F2231174
:1022800010FB01F0D74901EBC00118319DF898000F
:1022900000EBC00001EB00100270B9229DF8AC0009
:1022A00040F2231110FB01F0CE4901EBC0001830C1
:1022B0009DF8981001EBC10100EB0110427100BFC5
:1022C00000BFCFE59DF8AC0000EB400101EB001032
:1022D000C54901EB0010007B20B101287ED0022807
:1022E0007DD1E6E2C1499DF8AC0031F81000801FB5
:1022F00081B209919DF8AC0000EB4001C1EBC01127
:10230000BB4800EBC100401C08900999F7F7E2FABE
:102310000022CDE92E029DF8AC0000EB4001C1EB9C
:10232000C010B34901EBC002B0489DF8AC1030F8C2
:102330001100401F111809910421099816F0FEF8A8
:10234000C217CDE92C022DA819C82C99594060401C
:1023500001437DD1A74A9DF8AC0002EB001001704B
:102360009DF8AC0000EB4001C1EBC010A04901EBAF
:10237000C00001792491BDF89000312802D0452891
:1023800067D1EBE099489DF8AC1030F8110018388F
:10239000412190FBF1F0C217C1B2CDE92C02964861
:1023A00080F8AC1000203790CEE09DF8AC0000EB38
:1023B0004001C1EBC0108E4901EBC001BDF8DC004B
:1023C00000EB801014300A5C8B49AD31BDF8DC00A5
:1023D0000A549DF8AC0000EB400101E0C1E067E267
:1023E000C1EBC010824901EBC001BDF8DC0000EB7D
:1023F00080101A30014409910821099816F05CF800
:102400008DED0E0A7C4AB932BDF8DC000E9902EB64
:10241000001041609DF8AC0000EB4001C1EBC01022
:10242000734901EBC001BDF8DC0000EB80103230D5
:10243000014409910821099816F03EF88DED0E0A25
:102440006D4AB932BDF8DC000E9902EB001001E0D4
:1024500086E084E001609DF8AC0000EB4001C1EB38
:10246000C010634901EBC001BDF8DC0000EB801037
:102470003A30014409910821099816F01DF88DEDB4
:102480000E0A5D4AB932BDF8DC000E9902EB00106D
:1024900081609DF8AC0000EB4001C1EBC0105449D5
:1024A00001EBC001BDF8DC0000EB801042300144BC
:1024B00009910821099815F0FFFF8DED0E0A4E4A8B
:1024C000B932BDF8DC000E9902EB0010C1609DF836
:1024D000AC0000EB400101EB0010434901EB00119F
:1024E0003031BDF8DC0001EB0010801C0990007851
:1024F00020F080008030099908709DF8AC0000EB56
:102500004001C1EBC0103A4901EBC00237489DF8C9
:10251000AC1030F81100401E125C9DF8AC0040F287
:10252000231110FB01F02F4901EBC00018309DF87A
:10253000981001EBC10100EB011080F83C20BDF8C0
:10254000DC00401C80B23790BDF8DC000021DDE9E2
:102550002C34C01AA141FFF628AF00E000BF00BF35
:10256000BBE29DF8AC0000EB4001C1EBC01020497C
:1025700001EBC000407D9DF8AC1001EB4102C2EBC5
:10258000C1111B4A02EBC101897D40EA0120C2173B
:10259000CDE92C029DF8AC0000EB4001C1EBC0106E
:1025A000134901EBC001099115210998F7F776F954
:1025B0000022CDE92E02DDE92E42DDE92C1061403A
:1025C000504001437DD19DF8AC0000EB4001C1EBD0
:1025D000C010074911F83000401EC1B226910021F9
:1025E000044A0BE0C4440020044000202469002079
:1025F000A4770020383E0020BC3200209DF8AC00BB
:1026000002EB00129DF898001154FD4A9DF89800C5
:1026100011549FEDFC0A10EE101A0C329DF8980030
:1026200002EB001041609DF8AC0000EB4001C1EBF3
:10263000C010F54901EBC00081799DF8AC0000EBBA
:102640004002C2EBC010F04A02EBC000407941EA00
:10265000002000EE100AB8EEC00A9FEDEC1AC0EEA2
:10266000010A9DF8AC0000EB4001C1EBC01011461F
:1026700001EBC00001799DF8AC0000EB4002C2EB19
:10268000C010E14A02EBC000C07841EA002000EE31
:10269000100AB8EEC00A30EE800A10EE101AD84ABE
:1026A0000C329DF8980002EB001001609DF8AC0020
:1026B00000EB4001C1EBC010D34901EBC000817AAF
:1026C00000E0F5E09DF8AC0000EB4002C2EBC0106A
:1026D000CD4A02EBC000407A41EA002000EE100A29
:1026E000B8EEC00A9FEDC91AC0EE010A9DF8AC0011
:1026F00000EB4001C1EBC010114601EBC000017AB4
:102700009DF8AC0000EB4002C2EBC010BE4A02EBE9
:10271000C000C07941EA002000EE100AB8EEC00AFD
:1027200030EE800A10EE101AB54A0C329DF898006F
:1027300002EB001081609DF8AC0000EB4001C1EBA2
:10274000C010B14901EBC000C07A00F0800038BB76
:102750009DF8AC0000EB4001C1EBC010AA4901EBB1
:10276000C000017B9DF8AC0000EB4002C2EBC01042
:10277000A54A02EBC000C07A41EA002000EE100A30
:10278000F8EEC00AB3EE001A80EE810A10EE100ACD
:102790009B4A0C329DF8981002EB0111C86047E08B
:1027A0009DF8AC0000EB4001C1EBC010964901EB75
:1027B000C000017B9DF8AC0000EB4002C2EBC010F2
:1027C000914A02EBC000C07A41EA0020404280B248
:1027D00000EE100AB8EEC00A8DED030A0398F5F773
:1027E0009DFF9FED8B0B53EC102BCDE904019DED6C
:1027F000040B51EC100BF5F775FE9FED870B53ECB6
:10280000102BCDE906019DED060B51EC100BF5F7F1
:10281000F4FDCDE908019DED080B51EC100BF5F727
:1028200090FF774A0C329DF8981002EB0111C860B6
:102830009DF8AC0000EB400101EB0010784901EB82
:10284000001030309DF8981000EB0110801C0990AA
:10285000007820F080008030099908709DF8AC0065
:1028600000EB4001C1EBC010674901EBC000C27D25
:102870009DF8AC0040F2231110FB01F0694901EB17
:10288000C00018309DF8981001EBC10100EB011059
:1028900080F83C209DF8AC0000EB400101EB0010FB
:1028A0005F4901EB0010C1795548AD3880F8AC1094
:1028B00013E19DF8AC0000EB4001C1EBC0105249A0
:1028C00001EBC000C0799DF8AC1001EB4102C2EBF6
:1028D000C1114D4A02EBC101097A40EA0120C21739
:1028E000CDE92C029DF8AC0000EB4001C1EBC0101B
:1028F000454901EBC001099107210998F6F7CEFF80
:102900000022CDE92E02DDE92E42DDE92C106140E6
:102910005040014372D19DF8AC0000EB4001C1EB87
:10292000C010394911F83000401EC1B22691002173
:102930003D4A9DF8AC0002EB00100170304A9DF852
:10294000980011549DF8AC0000EB4001C1EBC010A1
:102950002D4901EBC000817908460191F5F758FE39
:10296000CDE902019DED021B9FED300B19F018FB24
:102970008DED060B9DF8AC0000EB4001C1EBC010E3
:10298000214901EBC00001799DF8AC0000EB400249
:10299000C2EBC0101C4A02EBC000C07841EA002024
:1029A00000EE100AB8EEC00A8DED030A0398F5F7A1
:1029B000B5FECDE904019DED060B53EC102B9DED0A
:1029C000040B51EC100BF5F78DFDCDE908019DEDE1
:1029D000080B51EC100BF5F7B4FE094A0C329DF8C8
:1029E000981002EB011148609FED060A10EE100AE4
:1029F0009DF8981002EB011108601BE06CE00000EC
:102A00006933002000000000A477002000FF7F470A
:102A10000000000000003040000000000000000046
:102A200004400020C4440020383E00200000000084
:102A3000000024401FED0D0A10EE100A9DF89810BA
:102A400002EB011188601FED110A10EE100A9DF8CB
:102A5000981002EB0111C8609DF8AC1001EB410029
:102A600000EB011002F68F4101EB001030309DF8B1
:102A7000981000EB0110801C0990007820F0800075
:102A80008030099908709DF8AC1001EB4100C0EB53
:102A9000C110FE4901EBC000427A9DF8AC0040F243
:102AA000231110FB01F0FA4901EBC00018309DF82A
:102AB000981001EBC10100EB011080F83C209DF85B
:102AC000AC1001EB410000EB0110F24901EB0010EA
:102AD000C179F14880F8AC1000BF00BF04F018BF06
:102AE0009DF8AC1001EB4100C0EBC110E74901EBD0
:102AF000C000C1789DF8AC0000EB4002C2EBC010F2
:102B0000E24A02EBC000807841EA002127919DF85B
:102B1000AC1001EB4100C0EBC110114601EBC0014C
:102B2000BDF89C00401C095C9DF8AC0000EB400225
:102B3000C2EBC010D54A02EBC002BDF89C00105C8D
:102B400041EA0020C217CDE92C029DF8AC1001EB40
:102B50004100C0EBC110CD4901EBC0000990BDF8A8
:102B60009C10F6F79BFE0022CDE92E022DA819C875
:102B70002C995940604001436FD19DF8AC1001EB96
:102B80004100C0EBC110C14901EBC0004178269162
:102B9000002137911CE09DF8AC1001EB410000EBE7
:102BA0000110BC4901EB00113031BDF8DC0001EB34
:102BB000001041789DF89800814204D1BDF8DC00F6
:102BC000C1B2269112E0BDF8DC00401C81B2379101
:102BD0009DF8AC1001EB410000EB0110AD4901EB99
:102BE0000010C179BDF8DC008142D4DC00BF9DF843
:102BF000AC1001EB410000EB0110A64901EB001005
:102C000030309DF8981000EB0110801C099000787E
:102C100020F080018031099801709DF8AC1001EB23
:102C20004100C0EBC110994901EBC000017924912A
:102C300000219A4A9DF8AC0002EB00129DF8980022
:102C40001154BDF89000F2287ED007DC05287CD016
:102C500006280AD0F12879D1FDE3FDE3F32876D0E8
:102C6000F42875D0F628F6D1F7E30621109100215B
:102C70003491F3E3BDF84000401C81B210919DF8FF
:102C8000AC1001EB4100C0EBC110804901EBC00169
:102C9000BDF84000095C2491BDF84000401C81B2A1
:102CA0001091BDF89000F12804D0F2287ED0F328CE
:102CB0007DD1FCE39DF8AC1001EB4100C0EBC110ED
:102CC000724901EBC001BDF84000095C2791BDF8D5
:102CD0004000401C81B210919DF8AC1001EB410006
:102CE00000EB01106B4901EB001130319DF8982089
:102CF000BDF8D000104401EB0010407A00F0010054
:102D000038B39DF8AC1040F2231011FB00F060497D
:102D100001EBC00118319DF89820BDF8D000104497
:102D200000EBC00001EB001090F88E0000F00100F5
:102D300078B99DF8AC1040F2231011FB00F0544913
:102D400001EBC001183105E0FDE3FDE3FDE3FDE328
:102D5000FDE349E09DF89820BDF8D000104400EB59
:102D6000C00001EB001090F88100E8B3002137911A
:102D70002FE09DF8AC1040F2231011FB00F0444905
:102D800001EBC00118319DF89820BDF8D000104427
:102D900000EBC00001EB001000F18201BDF8DC0087
:102DA0000A5C9DF8AC0000EB400101E0A1E39FE369
:102DB00001EB0010374901EB00100E30BDF8DC10BC
:102DC000405C824200D008E0BDF8DC00401C81B2CB
:102DD0003791BDF8DC000428CBDB00BFBDF8DC0078
:102DE000042860D1042100E05DE037912CE09DF8DB
:102DF000AC1040F2231011FB00F0254901EBC0019B
:102E000018319DF89820BDF8D000104400EBC000A8
:102E100001EB001000F18201BDF8DC000A5C9DF8B6
:102E2000AC0000EB400101EB00101A4901EB00106F
:102E30000E30BDF8DC10405C824200D008E0BDF8E6
:102E4000DC00401C81B23791BDF8DC000A28CEDBE3
:102E500000BFBDF8DC000A2825D09DF8AC1040F278
:102E6000231011FB00F00A4901EBC00018309DF857
:102E70009820BDF8D010114401EBC10100EB011006
:102E80008E300990007820F0010009E0A47700203E
:102E9000C444002004400020BC320020383E002002
:102EA000401C09990870BDF89C000F287ED19DF840
:102EB000AC1001EB410000EB0110F74901EB0011F0
:102EC00030319DF89820BDF8D000104401EB00107F
:102ED000801C0990007820F00400001D09990870FA
:102EE000002037902AE09DF8AC1001EB4100C0EBC8
:102EF000C110EA4901EBC001BDF84020BDF8DC007B
:102F000010440A5C9DF8AC0040F2231110FB01F064
:102F1000E34901EBC00118319DF89830BDF8D000AD
:102F2000184400EBC00001EB00113F31BDF8DC009C
:102F30000A54BDF8DC00401C81B23791BDF8DC00BA
:102F40000A28D0DBBDF840000A3081B21091002180
:102F500037912AE09DF8AC1001EB4100C0EBC110A5
:102F6000CE4901EBC001BDF84020BDF8DC001044A3
:102F70000A5C9DF8AC0040F2231110FB01F0C84937
:102F800001EBC00118319DF89830BDF8D00018440D
:102F900000EBC00001EB00115831BDF8DC000A5411
:102FA000BDF8DC00401C81B2379100E03EE2BDF884
:102FB000DC000228CEDBBDF84000801C81B21091FD
:102FC0009DF8AC1001EB4100C0EBC110B34901EB1F
:102FD000C001BDF84000085C01049DF8AC0000EBA6
:102FE0004002C2EBC010AD4A02EBC002BDF8400087
:102FF000401C105C41EA00219DF8AC0000EB40024F
:10300000C2EBC010A54A02EBC002BDF84000801C14
:10301000105C01439DF8AC0040F2231210FB02F05B
:103020009F4A02EBC00218329DF89830BDF8D000DC
:10303000184400EBC00002EB0010C166BDF8400070
:10304000C01C81B21091974890F89007F0BB002106
:1030500037911DE09DF8AC1040F2231011FB00F0F9
:103060008F4901EBC00118319DF89820BDF8D000C0
:10307000104400EBC00001EB00103F30BDF8DC1045
:10308000405C00B108E0BDF8DC00401C81B2379123
:10309000BDF8DC000A28DDDB00BFBDF8DC000A2833
:1030A00018D140229DF8AC0040F2231110FB01F032
:1030B0007B4901EBC00118319DF89830BDF8D00074
:1030C000184400EBC00001EB001000E055E080F870
:1030D00077204CE19DF8AC1040F2231011FB00F07A
:1030E0006F4901EBC00118319DF89820BDF8D00060
:1030F000104400EBC00001EB001090F87700E0BB3B
:10310000002128910DE10021359129E09DF8AC10B6
:1031100040F2231011FB00F0614901EBC0011831AE
:103120009DF89820BDF8D000104400EBC00001EBE2
:1031300000113F31BDF8D400001D095C9DF8A000CE
:1031400000EB4002584800EB4202BDF8D400105C8E
:10315000814200D008E0BDF8D400401C81B2359116
:10316000BDF8D4000628D1DB00BFBDF8D400062886
:103170007DD103229DF8AC0000E0F8E040F223117D
:1031800010FB01F0464901EBC00118319DF8983061
:10319000BDF8D000184400EBC00001EB001080F82F
:1031A00077209DF8AC1001EB410000EB01103A498B
:1031B00001EB001130319DF89820BDF8D00010448B
:1031C00001EB0010801C0990007820F0040209989F
:1031D0000270002037901CE020229DF8AC0040F2E5
:1031E000231110FB01F02E4901EBC00118319DF8AD
:1031F0009830BDF8D000184400EBC00001EB00117E
:103200004931BDF8DC000A54BDF8DC00401C81B235
:103210003791BDF8DC000F28DEDB002137911CE080
:1032200020229DF8AC0040F2231110FB01F01C4954
:1032300001EBC00118319DF89830BDF8D00018445A
:1032400000EBC00001EB00115B31BDF8DC000A545B
:10325000BDF8DC00401C81B23791BDF8DC000A28C3
:10326000DEDB00229DF8AC0040F2231100E053E0C9
:1032700010FB01F00A4901EBC00118319DF89830AC
:10328000BDF8D000184400EBC00001EB001080F83E
:1032900070200021379126E004400020A477002010
:1032A000C4440020BC3200203834002000229DF8A5
:1032B000AC0040F2231110FB01F0FE4901EBC0010C
:1032C00018319DF89830BDF8D000184400EBC000CC
:1032D00001EB00117131BDF8DC000A54BDF8DC00CF
:1032E000401C81B23791BDF8DC000528DEDB9DF87B
:1032F000AC1040F2231011FB00F0EE4901EBC001CD
:1033000018319DF89820BDF8D000104400EBC000A3
:1033100001EB0010C06E0CE09DF8A000401CC1B293
:103320002891E548B0F87A119DF8A00081423FF756
:10333000EAAE00BFE048B0F87A019DF8A0108842DC
:1033400015D140229DF8AC0040F2231110FB01F092
:10335000D84901EBC00118319DF89830BDF8D00074
:10336000184400EBC00001EB001080F877209DF8B6
:10337000AC1040F2231011FB00F0CE4901EBC0016C
:1033800018319DF89820BDF8D000104400EBC00023
:1033900001EB001090F87700032804D0112818D012
:1033A000402842D12BE0F2229DF8AC0040F22311DC
:1033B00010FB01F0BF4901EBC00118319DF89830B6
:1033C000BDF8D000184400EBC00001EB00104271C2
:1033D0002BE0F3229DF8AC0040F2231110FB01F02A
:1033E000B44901EBC00118319DF89830BDF8D00008
:1033F000184400EBC00001EB0010427115E0F2220E
:103400009DF8AC0040F2231110FB01F0A94901EB3B
:10341000C00118319DF89830BDF8D000184400EB79
:10342000C00001EB0010427100BF61E09DF8AC10DC
:1034300001EB410000EB0110A04901EB001130311C
:103440009DF89820BDF8D000104401EB0010801CBE
:103450000990007803E0C3E0F1E3F1E3B0E020F08D
:103460000402099802709DF8AC1040F2231011FB81
:1034700000F0904901EBC00018309DF89820BDF88D
:10348000D010114401EBC10100EB011090F88E0047
:1034900000F0010060B300229DF8AC0040F223115F
:1034A00010FB01F0834901EBC001183100E06BE033
:1034B0009DF89830BDF8D000184400EBC00001EB37
:1034C0000010A0F88C2005229DF8AC0040F22311DA
:1034D00010FB01F0774901EBC00118319DF89830DD
:1034E000BDF8D000184400EBC00001EB00104271A1
:1034F00060E09DF8AC1040F2231011FB00F06D4924
:1035000001EBC00118319DF89820BDF8D00010449F
:1035100000EBC00001EB001090F8770040281CD1B0
:1035200000229DF8AC0040F2231110FB01F061492C
:1035300001EBC00118319DF89830BDF8D000184457
:1035400000EBC00004E0F0E3F0E3F0E3F0E3F0E3CD
:1035500001EB001080F8772000BF00BFF1229DF83A
:10356000AC0040F2231110FB01F0524901EBC00105
:1035700018319DF89830BDF8D000184400EBC00019
:1035800001EB0010427115E0F1229DF8AC0040F211
:10359000231110FB01F0474901EBC00118319DF8E0
:1035A0009830BDF8D000184400EBC00001EB0010CB
:1035B000427100BF00BFBDF8D000401C81B2349101
:1035C0009DF8AC0000EB4001C1EBC0103C4901EBA1
:1035D000C0004179BDF8D00081423FF74BABA6E374
:1035E0009DF8AC0040F2231110FB01F0314901EBD2
:1035F000C00018309DF8981001EBC10100EB0110DC
:10360000007820BB01229DF8AC0040F2231110FB92
:1036100001F0284901EBC00118319DF8980000EB3A
:10362000C00001EB00100270F4229DF8AC0040F2E3
:10363000231110FB01F01F4901EBC00018309DF869
:10364000981001EBC10100EB01104271C7E09DF839
:10365000AC0000EB400101EB0010184901EB001039
:1036600030309DF8981000EB0110407A00F0010016
:10367000F8B19DF8AC0040F2231110FB01F00D49A8
:1036800001EBC00018309DF8981001EBC10100EB70
:10369000011090F88E0000F0010050B99DF8AC00C8
:1036A00040F2231110FB01F0024901EBC000183079
:1036B00008E048E0C4440020BC3200200440002060
:1036C000A47700209DF8981001EBC10100EB0110D8
:1036D00090F88100B8B30020379029E09DF8AC0045
:1036E00040F2231110FB01F0F74901EBC001183142
:1036F0009DF8980000EBC00001EB001000F1820182
:10370000BDF8DC000A5C9DF8AC0000EB400101EB69
:103710000010EE4901EB00100E30BDF8DC10405CEB
:10372000824200D008E0BDF8DC00401C81B2379135
:10373000BDF8DC000428D1DB00BFBDF8DC000428A4
:103740004DD137902AE04AE09DF8AC0040F22311B9
:1037500010FB01F0DC4901EBC00118319DF8980025
:1037600000EBC00001EB001000F18201BDF8DC00AD
:103770000A5C9DF8AC0000EB400101EB0010D3495E
:1037800001EB00100E30BDF8DC10405C824200D02E
:1037900008E0BDF8DC00401C81B23791BDF8DC00C8
:1037A0000A28D1DB00BFBDF8DC000A2817D09DF83D
:1037B000AC0040F2231110FB01F0C34901EBC00043
:1037C00018309DF8981001EBC10100EB01108E300C
:1037D0000990007820F00100401C09990870BDF89C
:1037E0009C00112871D19DF8AC0000EB400101EB69
:1037F0000010B64901EB001030309DF8981000EB36
:103800000110801C0990007820F00400001D099927
:1038100008700020379025E09DF8AC0000EB4001D7
:10382000C1EBC010AA4901EBC001BDF8DC00401D8E
:103830000A5C9DF8AC0040F2231110FB01F0A24994
:1038400001EBC00118319DF8980000EBC00001EBBE
:1038500000113F31BDF8DC000A54BDF8DC00401C0B
:1038600081B23791BDF8DC000A28D5DB0020379003
:1038700025E09DF8AC0000EB4001C1EBC01094497D
:1038800001EBC001BDF8DC000F300A5C9DF8AC0014
:1038900040F2231110FB01F08B4901EBC0011831FC
:1038A0009DF8980000EBC00001EB00115831BDF805
:1038B000DC000A54BDF8DC00401C81B23791BDF831
:1038C000DC000228D5DBBEE2FFE7BDF89C0014282F
:1038D0007DD19DF8AC0000EB400101EB00107B496D
:1038E00001EB001030309DF8981000EB0110801CA7
:1038F0000990007820F00400001D0999087000204C
:10390000379025E09DF8AC0000EB4001C1EBC01002
:103910006F4901EBC001BDF8DC00401D0A5C9DF859
:10392000AC0040F2231110FB01F0674901EBC0012C
:1039300018319DF8980000EBC00001EB00113F31F9
:10394000BDF8DC000A54BDF8DC00401C81B23791A0
:10395000BDF8DC000A28D5DB0020379025E09DF873
:10396000AC0000EB4001C1EBC010594901EBC001B4
:10397000BDF8DC000F300A5C9DF8AC0040F223116A
:1039800010FB01F0504901EBC00118319DF898007F
:1039900000EBC00001EB00115831BDF8DC000A5407
:1039A000BDF8DC00401C81B23791BDF8DC00022874
:1039B000D5DB9DF8AC0000EB4001C1EBC0104449E1
:1039C00001EBC000407C01049DF8AC0000E0EBE19D
:1039D00000EB4002C2EBC0103D4A02EBC000807C0D
:1039E00041EA00219DF8AC0000EB4002C2EBC010A0
:1039F000374A02EBC000C07C01439DF8AC0040F2A6
:103A0000231210FB02F0304A02EBC00018309DF880
:103A1000982002EBC20200EB0210C1662D4890F81C
:103A20009007C8BB002037901AE09DF8AC0040F228
:103A3000231110FB01F0244901EBC00118319DF85E
:103A4000980000EBC00001EB00103F30BDF8DC1027
:103A5000405C00B108E0BDF8DC00401C81B2379149
:103A6000BDF8DC000A28E0DB00BFBDF8DC000A2856
:103A700013D140229DF8AC0040F2231110FB01F05D
:103A8000114901EBC00018309DF8981001EBC101FD
:103A900000EB011080F877202EE19DF8AC0040F299
:103AA000231110FB01F0084901EBC00018309DF80C
:103AB000981001EBC10100EB011090F8770080BB7A
:103AC00000202890F5E00000C444002004400020BD
:103AD000A4770020BC3200200020359027E09DF81C
:103AE000AC0040F2231110FB01F0FE4901EBC001D4
:103AF00018319DF8980000EBC00001EB00113F3138
:103B0000BDF8D400001D095C9DF8A00000EB400248
:103B1000F54800EB4202BDF8D400105C814201D0B0
:103B200009E0E9E0BDF8D400401C81B23591BDF850
:103B3000D4000628D3DB00BFBDF8D40006287DD111
:103B400003229DF8AC0040F2231110FB01F0E5497F
:103B500001EBC00118319DF8980000EBC00001EBAB
:103B6000001080F877209DF8AC0000EB400101EBDD
:103B70000010DE4901EB001130319DF8980001EB97
:103B80000010801C0990007820F00402099802704F
:103B90000020379019E020229DF8AC0040F223115C
:103BA00010FB01F0CF4901EBC00118319DF89800DE
:103BB00000EBC00001EB00114931BDF8DC000A54F4
:103BC000BDF8DC00401C81B23791BDF8DC000F2845
:103BD000E1DB0020379019E020229DF8AC0040F294
:103BE000231110FB01F0BF4901EBC00118319DF812
:103BF000980000EBC00001EB00115B31BDF8DC0068
:103C00000A54BDF8DC00401C81B23791BDF8DC00DD
:103C10000A28E1DB00229DF8AC0040F2231110FBE2
:103C200001F0B04901EBC00118319DF8980000EB9C
:103C3000C00001EB001080F8702002E034E0A5E243
:103C40005AE10021379119E000229DF8AC0040F2C2
:103C5000231110FB01F0A34901EBC00118319DF8BD
:103C6000980000EBC00001EB00117131BDF8DC00E1
:103C70000A54BDF8DC00401C81B23791BDF8DC006D
:103C80000528E1DB9DF8AC0040F2231110FB01F0A8
:103C9000944901EBC00018309DF8981001EBC10168
:103CA00000EB0110C06E0CE09DF8A000401CC1B2FA
:103CB00028918F48B0F87A019DF8A01088423FF70C
:103CC0000BAF00BF8A48B0F87A019DF8A010884277
:103CD00012D140229DF8AC0040F2231110FB01F0FC
:103CE000804901EBC00018309DF8981001EBC1012C
:103CF00000EB011080F877209DF8AC0040F2231112
:103D000010FB01F0774901EBC00018309DF89810C6
:103D100001EBC10100EB011090F87700032809D0F6
:103D200011281AD040283ED12AE08DE0BDE12CE2D6
:103D3000C6E006E1F2229DF8AC0040F2231110FB30
:103D400001F0684901EBC00018309DF8981001EBB4
:103D5000C10100EB0110427125E0F3229DF8AC0097
:103D600040F2231110FB01F05E4901EBC000183056
:103D70009DF8981001EBC10100EB0110427112E0B7
:103D8000F2229DF8AC0040F2231110FB01F05549DE
:103D900001EBC00018309DF8981001EBC10100EB59
:103DA0000110427100BF4EE09DF8AC0000EB4001F5
:103DB00001EB00104D4901EB001030309DF89810D8
:103DC00000EB0110801C0990007820F00402099893
:103DD00002709DF8AC0040F2231110FB01F0414944
:103DE00001EBC00018309DF8981001EBC10100EB09
:103DF000011090F88E0000F0010020B300229DF821
:103E0000AC0040F2231110FB01F0364901EBC00178
:103E100018319DF8980000EBC00001EB0010A0F8ED
:103E20008C2005229DF8AC0040F2231110FB01F01C
:103E30002C4901EBC00018309DF8981001EBC1012E
:103E400000EB01104271A0E19DF8AC0040F223119B
:103E500010FB01F0234901EBC00018309DF89810C9
:103E600001EBC10100EB011090F87700402813D15D
:103E700000229DF8AC0040F2231110FB01F019491B
:103E800001EBC00018309DF8981001EBC10100EB68
:103E9000011080F8772000BF00BFF1229DF8AC0030
:103EA00040F2231110FB01F00E4901EBC000183065
:103EB0009DF8981001EBC10100EB0110427164E123
:103EC000F1229DF8AC0040F2231110FB01F00549EE
:103ED00001EBC00018309DF8981001EBC10100EB18
:103EE000011007E0C44400203834002004400020C2
:103EF000BC320020427148E103229DF8AC0040F240
:103F0000231110FB01F0FE4901EBC00118319DF8AF
:103F1000980000EBC00001EB00100270F1229DF848
:103F2000AC0040F2231110FB01F0F54901EBC00099
:103F300018309DF8981001EBC10100EB011042719F
:103F400023E102229DF8AC0040F2231110FB01F0A6
:103F5000EB4901EBC00118319DF8980000EBC0005F
:103F600001EB00100270F6229DF8AC0040F2231124
:103F700010FB01F0E24901EBC00118319DF89800F7
:103F800000EBC00001EB0010427101229DF8AC0073
:103F900040F2231110FB01F0D94901EBC0011831A7
:103FA0009DF8980000EBC00001EB001080F8812024
:103FB0000021379126E09DF8AC0000EB4001C1EBF9
:103FC000C010D04901EBC001BDF8DC00401D0A5C07
:103FD0009DF8AC0040F2231110FB01F0C84901EB41
:103FE000C00118319DF8980000EBC00001EB0010F3
:103FF00000F18201BDF8DC000A54BDF8DC00401C71
:1040000081B23791BDF8DC000A28D4DBBDF89C00F2
:10401000152849D19DF8AC0000EB4001C1EBC01060
:10402000B84901EBC000C27B9DF8AC0040F22311FF
:1040300010FB01F0B24901EBC00118319DF8980066
:1040400000EBC00001EB001080F8782000213791D0
:1040500026E09DF8AC0000EB4001C1EBC010A9497F
:1040600001EBC001BDF8DC0010300A5C9DF8AC002B
:1040700040F2231110FB01F0A14901EBC0011831FE
:104080009DF8980000EBC00001EB001000F17A01F0
:10409000BDF8DC000A54BDF8DC00401C81B2379149
:1040A000BDF8DC000428D4DB6FE09DF8AC0000EB29
:1040B0004001C1EBC010934901EBC00081799DF82C
:1040C000AC0000EB4002C2EBC0108E4A02EBC00015
:1040D000407941EA00229DF8AC0040F2231110FB28
:1040E00001F0874901EBC00118319DF8980000EB01
:1040F000C00001EB0010A0F88C209DF8AC0040F24D
:10410000231110FB01F07E4901EBC00118319DF82D
:10411000980000EBC00001EB0010B0F88C109DF887
:10412000AC0000EB400202EB0010774A02EB0010FB
:10413000408B814228DBF1229DF8AC0040F2231134
:1041400010FB01F06E4901EBC00118319DF8980099
:1041500000EBC00001EB001042719DF8AC0040F292
:10416000231110FB01F0664901EBC00118319DF8E5
:10417000980000EBC00001EB00108E300990007831
:1041800020F001020998027000BF00BF03F0C0BB1D
:104190009DF8AC0000EB4001C1EBC010594901EBA8
:1041A000C00001792691002134911CE09DF8AC00FB
:1041B00000EB400101EB0010534901EB00113031DD
:1041C000BDF8D00001EB001041789DF898008142C5
:1041D00004D1BDF8D000C1B2269112E0BDF8D000E4
:1041E000401C81B234919DF8AC0000EB400101EB22
:1041F0000010454901EB0010C179BDF8D0008142A3
:10420000D4DC00BF9DF8AC0000EB4001C1EBC01056
:104210003C4901EBC000C1782491BDF890001728FB
:1042200034D2DFE800F0330C0F331215181B1E33A5
:10423000333333333321242733332A2D30000720FF
:10424000279023E00720279020E0062027901DE0FC
:10425000062027901AE00620279017E012202790CA
:1042600014E00720279011E0092027900EE0062097
:1042700027900BE00620279008E00B20279005E010
:104280000B20279002E02A20279000BF00BFBDF836
:104290009C00001FC1B209919DF8AC0000EB4001E9
:1042A000C1EBC010174901EBC000C01C0890099970
:1042B000F5F710F935909DF8AC0000EB4001C1EB2B
:1042C000C010104901EBC001BDF89C00401E095C04
:1042D000BDF8D40081427DD19DF8AC0000EB4001D7
:1042E000C1EBC010074901EBC0004078002871DD28
:1042F0009DF8AC0000EB4001C1EBC010014905E0A6
:10430000C4440020A47700200440002001EBC00139
:10431000BDF89C000A5C9DF8AC0040F2231110FB34
:1043200001F0FE4901EBC00118319DF8980000EB47
:10433000C00001EB001080F83C200021F84A9DF8F5
:10434000AC0002EB00129DF898001154F54890F86B
:104350002800012815D19DF8AC0000EB400101EBCD
:104360000010F14901EB001030309DF8981000EB7F
:104370000110801C0990007820F08000803009999D
:104380000870BDF8900007287ED00ADC07287CD290
:10439000DFE810F07B009B05F8057B0088055405DD
:1043A0008E0B10380728F2D2DFE810F0E60BD30BA3
:1043B0006F006F0007000800200600BFBDF89000E6
:1043C00014287DD19DF8AC0000EB4001C1EBC0107A
:1043D000D64900E0FEE301EBC000407901069DF8FC
:1043E000AC0000EB4002C2EBC010D04A02EBC000B0
:1043F000807941EA00419DF8AC0000EB4002C2EB3D
:10440000C010CA4A02EBC000C07941EA00219DF801
:10441000AC0000EB4002C2EBC010C44A02EBC0008B
:10442000007A01439DF8AC0040F2231210FB02F029
:10443000BA4A02EBC00218329DF8980000EBC000A7
:1044400002EB0010C0F81A109DF8AC0040F22311E6
:1044500010FB01F0B14901EBC00118319DF8980043
:1044600000EBC00001EB0010D0F81A1008460991CB
:1044700000210AF02FF9CDE92C019DF8AC0000EBEA
:10448000400101EB001001E0FEE3FEE3A64901EB71
:104490000010007F00F003019DF8AC0000EB40022B
:1044A00002EB0010A04A02EB0010007FC0F30110E5
:1044B00001449DF8AC0000EB400202EB001000E06C
:1044C00062E0994A02EB0010007FC0F38100091AF4
:1044D00008460591F4F78BF8CDE906019DED061B22
:1044E0009FED930B17F05CFD8DED080B9DED080B18
:1044F00051EC100BF4F7EDF8CDE92E019DF8AC006E
:1045000040F2231110FB01F0844901EBC001183186
:104510009DF8980000EBC00001EB0010416B0846CD
:10452000079100210AF0D6F8DDE92C32A0FB034503
:1045300001FB035100FB021502220023DDE92E01DD
:10454000F3F740FE20186941CDE90801DDE92E238B
:10455000F3F738FECDE92C01DDE92C010AF06EFEFF
:1045600001469DF8AC0040F2231210FB02F06B4AAA
:1045700002EBC00018309DF8982002EBC20200EB5D
:104580000210C0F81E1043E0BDF8900015283FD17E
:104590009DF8AC0000EB4001C1EBC010634901EB9A
:1045A000C000407901069DF8AC0000EB4002C2EB70
:1045B000C0105E4A02EBC000807941EA00419DF8DC
:1045C000AC0000EB4002C2EBC010584A02EBC00046
:1045D000C07941EA00219DF8AC0000EB4002C2EB3B
:1045E000C010524A02EBC000007A01439DF8AC00B3
:1045F00040F2231210FB02F0484A02EBC0001830D0
:104600009DF8982002EBC20200EB0210C0F81E10C9
:104610009DF8AC0000EB4001C1EBC010434901EB39
:10462000C000417A444880F8031D9DF8AC0000EBBF
:10463000400101EB00103C4901EB001130319DF8C5
:10464000980001EB0010801C09903B4890F8030D86
:10465000C2090998007862F3000009990870364889
:1046600090F8030D00F00300012806D0324890F8BE
:10467000030D00F0030003282BD19DF8AC0000EBE4
:10468000400101EB0010284901EB001030309DF88B
:10469000981000EB0110801C0990007820F00200B7
:1046A000801C099908709DF8AC0000EB400101EBFB
:1046B00000101D4901EB001030309DF8981000EB00
:1046C0000110801C0990007820F0200209980270E7
:1046D00014E09DF8AC0000EB400101EB0010124922
:1046E00001EB001030309DF8981000EB0110801C99
:1046F0000990007820F00202099802709DF8AC0041
:1047000000EB400101EB0010074901EB00113031D3
:104710009DF8980001EB001080780FE0C444002061
:10472000383E0020BC12002004400020A477002066
:104730000000000000002440BC220020C0F3400222
:104740009DF8AC0040F2231110FB01F0FD4901EB94
:10475000C00018309DF8981001EBC10100EB01106A
:10476000007EC0F34000824266D09DF8AC0040F26B
:10477000231110FB01F0F34901EBC00018309DF844
:10478000981001EBC10100EB0110183009909DF861
:10479000AC0000EB400101EB0010EB4901EB001015
:1047A00030309DF8981000EB01108078420809988D
:1047B000007862F34100099908709DF8AC0000EBA5
:1047C000400101EB0010E04901EB001030309DF892
:1047D000981000EB01108078C0F3400038BB9DF8C2
:1047E000AC0000EB400101EB0010D74901EB0010D9
:1047F00030309DF8981000EB0110801C0990007873
:1048000020F020020998027001229DF8AC0040F2CD
:10481000231110FB01F0CB4901EBC00018309DF8CB
:10482000981001EBC10100EB011080F83E209DF8CB
:10483000AC100220F5F7F8FB9DF8AC0000EB40014E
:1048400001EB0010C04901EB001130319DF89800D8
:1048500001EB0010807800F001029DF8AC0040F2FE
:10486000231110FB01F0B74901EBC00018309DF88F
:10487000981001EBC10100EB0110007E00F0010077
:1048800082425FD09DF8AC0040F2231110FB01F092
:10489000AC4901EBC00018309DF8981001EBC10144
:1048A00000EB0110183009909DF8AC0000EB4001BE
:1048B00001EB0010A44901EB001130319DF8980084
:1048C00001EB001081780998027861F30002027010
:1048D0009DF8AC0000EB400101EB00109A4901EBA0
:1048E000001030309DF8981000EB0110807800F037
:1048F000010040BB9DF8AC0000EB400101EB001053
:10490000914901EB001030309DF8981000EB011038
:10491000801C0990007820F0200209980270002283
:104920009DF8AC0040F2231110FB01F0854901EB2A
:10493000C00018309DF8981001EBC10100EB011088
:1049400080F83D20DBE19DF8AC0040F2231110FB24
:1049500001F07C4901EBC00018309DF8981001EB84
:10496000C10100EB011090F83E0098B901229DF8BA
:10497000AC0040F2231110FB01F0724901EBC000C2
:1049800018309DF8981001EBC10100EB011080F880
:104990003D2027E000229DF8AC0040F2231110FBDF
:1049A00001F0684901EBC00118319DF8980000EB57
:1049B000C00001EB001080F83D209DF8AC0000EB3A
:1049C000400101EB0010604901EB001130319DF80E
:1049D000980001EB0010801C0990007820F0010283
:1049E00009980270594890F89007E8BB584890F829
:1049F000290001287ED15648D0F80C025449498D2F
:104A0000884277D29DF8AC0040F2231110FB01F0F0
:104A10004C4901EBC00018309DF8981001EBC10122
:104A200000EB011090F83D0001281DD19DF8AC006D
:104A300040F2231110FB01F0424901EBC000183095
:104A40009DF8981001EBC10100EB011090F87E0079
:104A500050B901229DF8AC0000EB400101EB0010C1
:104A6000394901EB001100E010E130319DF8980068
:104A700001EB0010C2729DF8AC0000EB400101EBAD
:104A80000010314901EB001130319DF8980001EB25
:104A9000001001789DF8AC0040F2231210FB02F0E8
:104AA000284A02EBC000417005229DF8AC0040F29C
:104AB000231110FB01F0234901EBC00118319DF8CF
:104AC000980000EBC00001EB0010427100229DF83D
:104AD000AC0000EB400101EB00101B4901EB0011A1
:104AE00030319DF8980001EB001042609DF8AC1049
:104AF000022000E04DE0F5F797FA0021379119E028
:104B000000229DF8AC0040F2231110FB01F00D498A
:104B100001EBC00118319DF8980000EBC00001EBDB
:104B200000113F31BDF8DC000A54BDF8DC00401C28
:104B300081B23791BDF8DC001428E1DB002037900A
:104B400022E00000C444002004400020BC320020C9
:104B5000BC12002000229DF8AC0040F2231110FB93
:104B600001F0FE4901EBC00118319DF8980000EBFF
:104B7000C00001EB00115B31BDF8DC000A54BDF848
:104B8000DC00401C81B23791BDF8DC000A28E1DB73
:104B9000B5E09DF8AC0040F2231110FB01F0EF49A5
:104BA00001EBC00018309DF8981001EBC10100EB3B
:104BB000011090F83D00012868D19DF8AC0040F24A
:104BC000231110FB01F0E54901EBC00118319DF8FC
:104BD000980000E0F5E300EBC00001EB001090F856
:104BE0007F0040F2231110FB01F0DC4901EBC00112
:104BF00018319DF8AC0040F2231210FB02F0D74AA6
:104C000002EBC00018309DF8982002EBC20200EBC6
:104C1000021090F8800000EBC00001EB001090F84B
:104C2000770003286BD102229DF8AC0000EB400115
:104C300001EB0010CA4901EB001130319DF89800DA
:104C400001EB0010C2729DF8AC0000EB400101EBDB
:104C50000010C34901EB001130319DF8980001EBC1
:104C6000001001789DF8AC0040F2231210FB02F016
:104C7000BA4A02EBC00041709DF8AC0040F223112B
:104C800010FB01F0114602E07FE27DE237E001EB2C
:104C9000C00118319DF8980000EBC00001EB001036
:104CA00001789DF8AC0040F2231210FB02F0AB4AF1
:104CB00002EBC0004079814211D105229DF8AC0081
:104CC00040F2231110FB01F0A44901EBC0001830A1
:104CD0009DF8981001EBC10100EB01104271002218
:104CE0009DF8AC0000EB400101EB00109C4901EB8A
:104CF000001030309DF8981000EB011042609DF8D4
:104D0000AC0040F2231110FB01F0944901EBC0000C
:104D100018309DF8981001EBC10100EB01100078EC
:104D2000012812DC02229DF8AC0040F2231110FB96
:104D300001F08A4901EBC00018309DF8981001EB92
:104D4000C10100EB0110027077E09DF8AC0040F269
:104D5000231110FB01F0814901EBC00018309DF8D0
:104D6000981001EBC10100EB0110007802282FDC44
:104D700000219DF8AC0040F2231210FB02F0774AAC
:104D800002EBC000017103229DF8AC0040F2231138
:104D900010FB01F0714901EBC00118319DF898003A
:104DA00000EBC00001EB0010027007229DF8AC0080
:104DB00040F2231110FB01F0684901EBC0001830EC
:104DC0009DF8981001EBC10100EB0110427134E035
:104DD0009DF8AC0040F2231110FB01F05F4901EB9C
:104DE000C00118319DF8980000EBC00001EB0010E5
:104DF00001789DF8AC0040F2231210FB02F0574AF4
:104E000002EBC0004079814217D1564890F8030D5B
:104E1000C0F3401088B116229DF8AC0040F2231177
:104E200010FB01F04D4901EBC00018309DF89810BF
:104E300001EBC10100EB01104271A5E114229DF8C4
:104E4000AC0040F2231110FB01F0444901EBC0011A
:104E500018319DF8980000EBC00001EB0010427182
:104E600001219DF8AC0040F2231210FB02F03B4AF6
:104E700002EBC00001719DF8AC0000EB400101EBBA
:104E80000010374901EB001130319DF8980001EB1B
:104E90000010801C0990007820F020002030099933
:104EA000087071E114229DF8AC0040F2231110FB50
:104EB00001F02A4901EBC00018309DF8981001EB71
:104EC000C10100EB011042715EE19DF8AC0040F2BF
:104ED000231110FB01F0214901EBC0001830BDF88F
:104EE000D01001EBC10100EB01108079012824D121
:104EF00000229DF8AC0040F2231110FB01F017498D
:104F000001EBC0011831BDF8D00000EBC00001EB8F
:104F10000010827114229DF8AC0040F2231110FBA6
:104F200001F00E4901EBC00018309DF8981001EB1C
:104F3000C10100EB0110427123E000219DF8AC009B
:104F400040F2231210FB02F0044A02EBC000017190
:104F500005229DF8AC0040F2231105E0C444002076
:104F600004400020BC22002010FB01F0FE4901EBB0
:104F7000C00018309DF8981001EBC10100EB011042
:104F8000427101E101219DF8AC0040F2231210FBB7
:104F900002F0F54A02EBC000017114229DF8AC004A
:104FA00040F2231110FB01F0EF4901EBC001183171
:104FB0009DF8980000EBC00001EB001042719DF8D5
:104FC000AC0000EB400101EB0010E84901EB0010E0
:104FD00030309DF8981000EB0110801C099000788B
:104FE00020F00400001D09990870CDE000202C90ED
:104FF0002D90002137911FE0DDE92C10000240EADE
:1050000011620902CDE92C129DF8AC0000EB4001C1
:10501000C1EBC010D64901EBC001BDF8DC00401D5A
:10502000085CDDE92C3440EA0302CDE92C24BDF80C
:10503000DC00401C81B23791BDF8DC000328DBDBCB
:10504000DDE92C010AF0FAF801469DF8AC0040F2C7
:10505000231210FB02F0C44A02EBC00218329DF882
:10506000980000EBC00002EB0010C0F81E100022F8
:105070002C922D92002137911EE0DDE92C100002C8
:1050800040EA11620902CDE92C129DF8AC0000EB58
:105090004001C1EBC010B64901EBC001BDF8DC0016
:1050A0000830085CDDE92C341843CDE92C04BDF848
:1050B000DC00401C80B23790BDF8DC000328DCDB4C
:1050C000DDE92C010AF0BAF801469DF8AC0040F287
:1050D000231210FB02F0A44A02EBC00218329DF822
:1050E000980000EBC00002EB0010C0F81A1000227C
:1050F0002C922D92002137911EE0DDE92C10000248
:1051000040EA11620902CDE92C129DF8AC0000EBD7
:105110004001C1EBC010964901EBC001BDF8DC00B5
:105120001330085CDDE92C341843CDE92C04BDF8BC
:10513000DC00401C80B23790BDF8DC000328DCDBCB
:105140009DF8AC002C9940F2231210FB02F0864A25
:1051500002EBC00218329DF8980000EBC00002EB91
:105160000010416307229DF8AC0040F2231110FBB0
:1051700001F07D4901EBC00018309DF8981001EB5B
:10518000C10100EB01104271FDE300202C902D9035
:10519000002137911EE0DDE92C10000240EA116287
:1051A0000902CDE92C129DF8AC0000EB4001C1EBE7
:1051B000C0106F4901EBC001BDF8DC00401D085C68
:1051C000DDE92C341843CDE92C04BDF8DC00401C8B
:1051D00080B23790BDF8DC000428DCDBDDE92C016F
:1051E0000AF02CF89DF8AC2040F2231312FB03F2D6
:1051F0005D4B03EBC20318339DF8982002EBC2020B
:1052000003EB021222329060D16000222C922D9288
:10521000002137911EE0DDE92C10000240EA116206
:105220000902CDE92C129DF8AC0000EB4001C1EB66
:10523000C0104F4901EBC001BDF8DC000930085C2B
:10524000DDE92C341843CDE92C04BDF8DC00401C0A
:1052500080B23790BDF8DC000428DCDBDDE92C01EE
:1052600009F0ECFF9DF8AC2040F2231312FB03F28F
:105270003D4B03EBC20318339DF8982002EBC202AA
:1052800003EB021242F8220F51609DF8AC0040F28D
:10529000231110FB01F0344901EBC00118319DF8D6
:1052A000980000EBC00001EB001001789DF8AC0005
:1052B00040F2231210FB02F02B4A02EBC0004079AF
:1052C00081427DD12B4890F8030DC0F3401090B17E
:1052D00017229DF8AC0040F2231110FB01F0224987
:1052E00001EBC00018309DF8981001EBC10100EBF4
:1052F0000110427111E014229DF8AC0040F223111C
:1053000010FB01F0184901EBC00018309DF898100F
:1053100001EBC10100EB011042719DF8AC009DF85A
:10532000981001EB0010C217CDE92C02124890F83A
:105330009007C0B19DF8AC0000EB400101EB0010FC
:105340000A4901EB001030309DF8981000EB011075
:10535000807A02281CD09DF8AC0000EB400101EBE4
:10536000001002490AE013E0C44400200440002079
:10537000A4770020BC220020BC32002001EB0010EA
:1053800030309DF8981000EB0110C07A00287CDDC9
:1053900000229DF8AC0040F2231110FB01F0FC4903
:1053A00001EBC00118319DF8980000EBC00001EB43
:1053B000001080F83E209DF8AC0000EB400101E0B9
:1053C000F4E2EDE301EB0010F24901EB00113031A2
:1053D0009DF8980001EB0010C272EF48D0F80C0263
:1053E0000521B0FBF1F201FB120000EB4001EA489D
:1053F0002C3000EB41100D3009909DF8AC1040F2BC
:10540000231011FB00F0E24901EBC00018309DF8B9
:10541000981001EBC10100EB01102230102201466F
:1054200008900998F2F711FFDB48D0F80C0205212B
:10543000B0FBF1F201FB120000EB4001D6482C302A
:1054400000EB41129DF8AC0040F2231110FB01F07B
:10545000CF4901EBC00118319DF8980000EBC00066
:1054600001EB001050F81A1F42F8011F406850600D
:10547000C948D0F80C020521B0FBF1F201FB120083
:1054800000EB4001C4482C3000E08BE100EB4112FE
:105490009DF8AC0000EB400101EB0010BD4901EBB1
:1054A000001130319DF8980001EB00100078107069
:1054B000B948D0F80C020521B0FBF1F201FB120053
:1054C00000EB4001B4482C3000EB41129DF8AC00D9
:1054D00040F2231110FB01F0AD4901EBC00118317E
:1054E0009DF8980000EBC00001EB0010406BC2F883
:1054F0000900A948D0F80C020521B0FBF1F201FB2C
:10550000120000EB4001A4482C3000EB4111A348ED
:10551000C26841F81D2F008A88809F48D0F80C028D
:105520000521B0FBF1F201FB120000EB40019A48AB
:105530002C3000EB41129DF8AC0000EB400101EB78
:105540000010944901EB001130319DF8980001EBF7
:1055500000104068C2F8230000229DF8AC0000EB68
:10556000400101EB00108B4901EB001130319DF837
:10557000980001EB00104260002137914BE0864813
:10558000D0F80C020521B0FBF1F201FB120000EB98
:10559000400181482C3000EB41112731BDF8DC403F
:1055A0009DF8AC0040F2231210FB02F0784A02EBA7
:1055B000C00218329DF8980000EBC00002EB00100A
:1055C00090F87F0040F2231210FB02F0704A02EBC9
:1055D000C00218329DF8AC0040F2231310FB03F018
:1055E0006B4B03EBC00318339DF8980000EBC00031
:1055F00003EB001090F8800000EBC00002EB0012FB
:105600003F32BDF8DC00001D105C0855BDF8DC0021
:10561000401C81B23791BDF8DC000628AFDB0021C9
:10562000379139E000239DF8AC0040F2231110FBC4
:1056300001F0574901EBC00118319DF8980000EBCB
:10564000C00001EB001090F87F0040F2231110FB26
:1056500001F04F4901EBC00118319DF8AC0040F258
:10566000231210FB02F04A4A02EBC00218329DF8E6
:10567000980000EBC00002EB001090F8800000EBF7
:10568000C00001EB00113F31BDF8DC000B54BDF848
:10569000DC00401C81B23791BDF8DC000A28C1DB78
:1056A0003D48D0F80C020521B0FBF1F080B2014674
:1056B00009900220F3F70CFD00210620F4F7B4FC5A
:1056C0003548D0F80C023449498D884206D2324818
:1056D000D0F80C02401C3049C1F80C020021052012
:1056E000F4F7A2FC9DF8AC0000EB400101EB0010C8
:1056F000284901EB001030309DF8981000EB0110A4
:10570000801C0990007820F0080209980270224855
:10571000D0F80C020521B0FBF1F201FB120000EB06
:1057200040011D482C3000EB4110D0F823202C986C
:1057300000EB40011A4800EB4110C0F82320002084
:10574000379020E01448D0F80C020521B0FBF1F2AC
:1057500001FB120000EB40010F482C3000EB411020
:105760002730BDF8DC10425C2C9800EB40010C485F
:1057700000EB41112731BDF8DC000A54BDF8DC0014
:10578000401C81B23791BDF8DC000628DADB73E0FB
:10579000C444002004400020BC120020BC31002082
:1057A000D814002000229DF8AC0040F2231110FB19
:1057B00001F0FC4901EBC00118319DF8980000EBA5
:1057C000C00001EB001080F83E209DF8AC0000EB1B
:1057D000400101EB0010F44901EB001030309DF85E
:1057E000981000EB0110801C0990007820F0080050
:1057F0000830099908709DF8AC0000EB400101EBFE
:105800000010E94901EB001030309DF8981000EBD2
:10581000011042682C9800EB4001E44800EB411075
:10582000C0F823200020379022E09DF8AC0040F221
:10583000231110FB01F0DB4901EBC00118319DF889
:10584000980000EBC00001EB00113F31BDF8DC0017
:105850000A5C2C9800EB4001D44800EB4111273141
:10586000BDF8DC000A54BDF8DC00401C81B2379161
:10587000BDF8DC000628D8DB9DF8AC100220F4F758
:10588000D3FB9DF8AC0040F2231110FB01F0C54999
:1058900001EBC00018309DF8981001EBC10100EB3E
:1058A0000110223009902C9800EB4001BF4800EB1A
:1058B00041100D30102208900999F2F7C6FC9DF8AE
:1058C000AC0040F2231110FB01F0B64901EBC0011E
:1058D00018319DF8980000EBC00001EB00112C98E6
:1058E00000EB4002B14800EB421051F81A2F40F88B
:1058F000012F496841609DF8AC0000EB400101EBCD
:105900000010A94901EB001130319DF8980001EB1E
:10591000001001782C9800EB4002A44800EB4210E4
:1059200001702C9800EB4001A04800EB4111A04809
:10593000C26841F81D2F008A88809DF8AC0040F2B3
:10594000231110FB01F0974901EBC00118319DF8BC
:10595000980000EBC00001EB0010416B2C9800EBAD
:105960004002924800EB4210C0F809109DF8AC00CC
:1059700000EB400101EB00108B4901EB00113031CD
:105980009DF8980000E00AE101EB001041682C98B6
:1059900000EB4002854800EB4210C0F823102C9821
:1059A00081B208200991F4F73FFB80E09DF8AC003C
:1059B00040F2231110FB01F07A4901EBC0011831CC
:1059C0009DF8980000EBC00001EB001001789DF8F5
:1059D000AC0040F2231210FB02F0724A02EBC0004E
:1059E0004079814263DA9DF8AC0000EB400101EBA5
:1059F00000106D4901EB001030309DF8981000EB5D
:105A00000110801C0990007820F00400001D099905
:105A100008709DF8AC0000EB400101EB00106249FA
:105A200001EB001030309DF8981000EB0110801C45
:105A30000990007820F080008030099908700120DA
:105A40009DF8AC1040F2231211FB02F1554A02EB13
:105A5000C10108719DF8AC0040F2231110FB01F068
:105A6000114601EBC00042799DF8AC0040F22311D1
:105A700010FB01F04B4901EBC00018309DF8981065
:105A800001EBC10100EB0110027014229DF8AC0083
:105A900040F2231110FB01F0424901EBC000183025
:105AA0009DF8981001EBC10100EB0110427176E006
:105AB0000121404880F8B4169DF8AC0040F2231153
:105AC00010FB01F0374901EBC00118319DF8980037
:105AD00000EBC00001EB001001789DF8AC0040F233
:105AE000231210FB02F02F4A02EBC00040798142E2
:105AF0002EDA00219DF8AC0040F2231210FB02F0D8
:105B0000284A02EBC000017101229DF8AC0040F26E
:105B1000231110FB01F0234901EBC00118319DF85E
:105B2000980000EBC00001EB0010027014229DF8F9
:105B3000AC0040F2231110FB01F01A4901EBC00048
:105B400018309DF8981001EBC10100EB0110427173
:105B500025E014229DF8AC0040F2231110FB01F067
:105B6000104901EBC00018309DF8981001EBC101FD
:105B700000EB0110427112E014229DF8AC0040F2DB
:105B8000231110FB01F0074901EBC00018309DF80C
:105B9000981001EBC10100EB0110427100BF00BF82
:105BA00001F0B6BEC444002004400020D8140020F8
:105BB000BC310020BC3200209DF8AC0040F2231123
:105BC00010FB01F0FE4901EBC000817826919DF8A1
:105BD000AC0000EB4001C1EBC010FA4911F83010E5
:105BE00027919DF8AC0040F2231110FB01F0F4491D
:105BF00001EBC00118319DF8980000EBC00001EBEB
:105C00000010417924919DF8AC0000EB4001C1EBFC
:105C1000C010EC4901EBC0010991BDF89C10099836
:105C2000F4F79AFF35909DF8AC0000EB4001C1EB12
:105C3000C010E44901EBC001BDF89C00095CBDF84F
:105C4000D400814241F063869DF8AC0000EB400136
:105C5000C1EBC010DB4901EBC0004078002841F3E4
:105C600056860021D84A9DF8AC0002EB00129DF840
:105C700098001154BDF8900089287DD00EDC1428BE
:105C800001F0298605DC082877D0102841F03E86EF
:105C9000EFE3152872D08028F8D1EBE38B286ED083
:105CA0008C286DD08E286CD08F28EFD1BDF89C0049
:105CB0000D2867D19DF8AC0000EB4001C1EBC0108E
:105CC000C04901EBC0004178C04880F8051D9DF82F
:105CD000AC0000EB4001C1EBC010BA4901EBC000C1
:105CE000C17ABA4880F8061D9DF8AC0040F2231135
:105CF00010FB01F0B24901EBC00018309DF898107C
:105D000001EBC10100EB0110007803287EDCAF48F5
:105D100090F8060D00287ADD9DF8AC0040F22311C2
:105D200010FB01F0A64901EBC00118319DF8980065
:105D300000EBC00001EB001109910878401CC1B2D2
:105D4000099801709DF8AC0040F2231110FB01F09E
:105D50009B4901EBC00018309DF8981001EBC10180
:105D600000EB01100078042851DB9DF8AC0000EB3B
:105D7000400101EB001006E0FEE3FEE3FEE3FEE37C
:105D8000FEE3FEE3FEE3924901EB001030309DF8A4
:105D9000981000EB0110801C09908C4890F8060DBB
:105DA000C0F30010C0F101000999097860F3000107
:105DB00009980170854890F8050DC0F3C00038BB04
:105DC0009DF8AC0000EB400101EB0010804901EBB5
:105DD000001030309DF8981000EB01108078C0F36F
:105DE0004010A8B19DF8AC0000EB400101EB0010A1
:105DF000774901EB001030309DF8981000EB01104E
:105E0000801C0990007820F0020002E051E0E1E0FF
:105E10001FE0801C099908709DF8AC0040F2231126
:105E200010FB01F0664901EBC00018309DF8981096
:105E300001EBC10100EB011018300990007820F04F
:105E40000200801C099908709DF8AC100220F4F73C
:105E5000EBF800219DF8AC0040F2231210FB02F099
:105E6000574A02EBC000017104229DF8AC0040F2D9
:105E7000231110FB01F0524901EBC00118319DF8CC
:105E8000980000EBC00001EB001002708C229DF81E
:105E9000AC0040F2231110FB01F0494901EBC001B5
:105EA00018319DF8980000EBC00001EB0010427122
:105EB00090E09DF8AC0040F2231110FB01F0404946
:105EC00001EBC00118319DF8980000EBC00001EB18
:105ED000001001789DF8AC0040F2231210FB02F094
:105EE000374A02EBC0004079814273D19DF8AC0083
:105EF00000EB400101EB0010354901EB00103030A0
:105F00009DF8981000EB0110801C09902F4890F824
:105F1000060DC0F30010C0F101010998027861F389
:105F2000000202709DF8AC0000EB400101EB001094
:105F3000274901EB001130319DF8980001EB00106A
:105F4000801C0990214890F8050DC2080998017835
:105F500062F3410101709DF8AC0000EB400101EBE0
:105F600000101B4901EB001130319DF8980001EB46
:105F700000108078C0F340029DF8AC0040F223117D
:105F800010FB01F00E4901EBC00018309DF898108D
:105F900001EBC10100EB0110007EC0F34000824222
:105FA0006ED09DF8AC0040F2231110FB01F00449C3
:105FB00001EBC00018309DF8981001EBC1010AE018
:105FC000C4440020A4770020383E0020BC220020DA
:105FD0000440002082E300EB0110183009909DF886
:105FE000AC0000EB400101EB0010FD4901EB00109B
:105FF00030309DF8981000EB011080784208099825
:10600000007862F34100099908709DF8AC0000EB3C
:10601000400101EB0010F24901EB001030309DF817
:10602000981000EB01108078C0F3400018BB0122EB
:106030009DF8AC0040F2231110FB01F0E94901EB9F
:10604000C00118319DF8980000EBC00001EB001072
:1060500042739DF8AC0040F2231110FB01F0E149BE
:1060600001EBC00018309DF8981001EBC10100EB66
:10607000011080F83E209DF8AC100220F3F7D4FF09
:106080009DF8AC0000EB400101EB0010D44901EB9E
:10609000001130319DF8980001EB0010807800F07D
:1060A00001029DF8AC0040F2231110FB01F0CD4934
:1060B00001EBC00018309DF8981001EBC10100EB16
:1060C0000110007E00F00100824276D09DF8AC0005
:1060D00040F2231110FB01F0C24901EBC00018305F
:1060E0009DF8981001EBC10100EB011018300990E8
:1060F0009DF8AC0000EB400101EB0010B84901EB4A
:10610000001130319DF8980001EB00108278099859
:10611000017862F3000101709DF8AC0000EB4001D2
:1061200001EB0010AE4901EB001030309DF89810E3
:1061300000EB0110807800F00100E8BB9DF8AC0096
:1061400000EB400101EB0010A54901EB00103030DD
:106150009DF8981000EB01108078C0F3401068B3F0
:106160009DF8AC0040F2231110FB01F09D4901EBBA
:10617000C00018309DF8981001EBC10100EB011030
:1061800090F83E00D0B99DF8AC0040F2231110FB0E
:1061900001F0944901EBC00018309DF8981001EB14
:1061A000C10100EB0110407B40B99DF8AC0000EB51
:1061B000400101EB001002E045E022E22FE08849B7
:1061C00001EB001030309DF8981000EB0110807842
:1061D000C0F3400018BB01229DF8AC0040F223112F
:1061E00010FB01F07F4901EBC00118319DF89800C8
:1061F00000EBC00001EB001042739DF8AC0040F2D0
:10620000231110FB01F0774901EBC00018309DF815
:10621000981001EBC10100EB011080F83E20002234
:106220009DF8AC0040F2231110FB01F06D4901EB29
:10623000C00018309DF8981001EBC10100EB01106F
:1062400080F83D20D8E19DF8AC0040F2231110FB0E
:1062500001F0644901EBC00018309DF8981001EB83
:10626000C10100EB011090F83E0098B901229DF8A1
:10627000AC0040F2231110FB01F05A4901EBC000C1
:1062800018309DF8981001EBC10100EB011080F867
:106290003D2027E000229DF8AC0040F2231110FBC6
:1062A00001F0504901EBC00118319DF8980000EB56
:1062B000C00001EB001080F83D209DF8AC0000EB21
:1062C000400101EB0010464901EB001030309DF811
:1062D000981000EB0110801C0990007820F001025A
:1062E00009980270404890F8900780B19DF8AC0082
:1062F00000EB400101EB0010394901EB0010303098
:106300009DF8981000EB0110807A022870D1374870
:1063100090F8290001286BD13448D0F80C02334999
:10632000498D884264D29DF8AC0040F2231110FBE5
:1063300001F02C4901EBC00018309DF8981001EBDA
:10634000C10100EB011090F83D00012847D19DF8F4
:10635000AC0040F2231110FB01F0224901EBC00018
:1063600018309DF8981001EBC10100EB011090F876
:106370007E00A0BB01229DF8AC0000EB400101EBC8
:106380000010174901EB001130319DF8980001EB26
:106390000010C2729DF8AC0000EB400101EB001050
:1063A0000F4901EB001130319DF8980001EB00100E
:1063B00001789DF8AC0040F2231210FB02F0094A6C
:1063C00002EBC000417008229DF8AC0040F223119E
:1063D00010FB01F0034901EBC001183109E069E04D
:1063E00004400020C4440020BC320020BC12002025
:1063F000F1E09DF8980000EBC00001EB0010427145
:1064000000229DF8AC0000EB400101EB0010FE49BA
:1064100001EB001130319DF8980001EB0010426053
:106420009DF8AC100220F3F7FFFD0021379119E031
:1064300000229DF8AC0040F2231110FB01F0F3495B
:1064400001EBC00118319DF8980000EBC00001EB92
:1064500000113F31BDF8DC000A54BDF8DC00401CDF
:1064600081B23791BDF8DC001428E1DB00213791BF
:106470001BE0ABE2F8E300229DF8AC0040F22311F0
:1064800010FB01F0E14901EBC00118319DF89800C3
:1064900000EBC00001EB00115B31BDF8DC000A54D9
:1064A000BDF8DC00401C81B23791BDF8DC000A2841
:1064B000E1DBA1E09DF8AC0040F2231110FB01F0FC
:1064C000D24901EBC00018309DF8981001EBC101D2
:1064D00000EB011090F83D0001287CD19DF8AC0044
:1064E00040F2231110FB01F0C84901EBC001183143
:1064F0009DF8980000EBC00001EB001090F87F00C1
:1065000040F2231110FB01F0C04901EBC00118312A
:106510009DF8AC0040F2231210FB02F0BB4A02EBE4
:10652000C00018309DF8982002EBC20200EB021068
:1065300090F8800000EBC00001EB001090F87700AD
:10654000032859D102229DF8AC0000EB400101EB79
:106550000010AD4901EB001130319DF8980001EBBE
:106560000010C2729DF8AC0000EB400101EB00107E
:10657000A54901EB001106E03FE205E2F0E396E2F7
:10658000EFE2EEE3FFE130319DF8980001EB0010FF
:1065900001789DF8AC0040F2231210FB02F09B4AF8
:1065A00002EBC000417008229DF8AC0040F22311BC
:1065B00010FB01F0954901EBC00118319DF89800DE
:1065C00000EBC00001EB0010427100229DF8AC000E
:1065D00000EB400100E00FE001EB00108A4901EB05
:1065E000001130319DF8980001EB001042609DF8D9
:1065F000AC100220F3F718FD9DF8AC100220F3F761
:1066000013FD9DF8AC0040F2231110FB01F07F490F
:1066100001EBC00018309DF8981001EBC10100EBB0
:1066200001108078802835D19DF8AC0000EB400146
:1066300001EB0010744901EB001030309DF8981008
:1066400000EB01108078C0F3400018BB9DF8AC004F
:1066500000EB400101EB00106B4901EB0010303002
:106660009DF8981000EB01108078C0F3401088B9B5
:1066700015229DF8AC0040F2231110FB01F0634994
:1066800001EBC00018309DF8981001EBC10100EB40
:10669000011042719DF8AC0000EB400101EB0010CD
:1066A000594901EB001030309DF8981000EB0110B3
:1066B0008078C0F3400090B18F229DF8AC0040F28A
:1066C000231110FB01F0514901EBC00018309DF877
:1066D000981001EBC10100EB0110427141E09DF8FF
:1066E000AC0040F2231110FB01F0484901EBC0005F
:1066F00018309DF8981001EBC10100EB0110807B70
:1067000001282ED100229DF8AC0040F2231110FB8D
:1067100001F03E4901EBC00118319DF8980000EBF3
:10672000C00001EB001082738C229DF8AC0040F297
:10673000231110FB01F0354901EBC00118319DF820
:10674000980000EBC00001EB0010427100219DF8A1
:10675000AC0040F2231210FB02F02C4A02EBC00006
:1067600001719DF8AC0000EB400101EB00102649DF
:1067700001EB0010007BE8BB9DF8AC0000EB400192
:10678000C1EBC010224901EBC000807801049DF8E4
:10679000AC0000EB4002C2EBC0101D4A02EBC0008F
:1067A000C07841EA00219DF8AC0000EB4002C2EB4A
:1067B000C010174A02EBC00000790843C117CDE9A9
:1067C000080108F03BFD9DF8AC1040F2231211FBCC
:1067D00002F10E4A02EBC10218329DF8981001EB4B
:1067E000C10102EB0111C1F81E009DF8AC0000EBE5
:1067F000400100E03DE0C1EBC010054901EBC000E5
:106800004079000406E0000004400020C444002059
:10681000A47700209DF8AC1001EB4102C2EBC1113E
:10682000FE4A02EBC101897940EA01209DF8AC10D3
:1068300001EB4102C2EBC111F84A02EBC101C97977
:106840000843C117CDE9080108F0F8FC9DF8AC1029
:1068500040F2231211FB02F1F14A02EBC10118319F
:106860009DF8982002EBC20201EB0211C1F81A0058
:1068700089E09DF8AC0000EB4001C1EBC010E74996
:1068800001EBC000807801069DF8AC0000EB4002EF
:10689000C2EBC010E14A02EBC000C07841EA0041FF
:1068A0009DF8AC0000EB4002C2EBC010DB4A02EBEB
:1068B000C000007941EA00219DF8AC0000EB4002E5
:1068C000C2EBC010D54A02EBC00040790843C117A3
:1068D000CDE9080108F0B2FC9DF8AC1040F223129B
:1068E00011FB02F1CE4A02EBC10218329DF898105A
:1068F00001EBC10102EB0111C1F81E009DF8AC00D3
:1069000000EB4001C1EBC010C44901EBC00080792D
:1069100000069DF8AC1001EB4102C2EBC111BF4A69
:1069200002EBC101C97940EA01409DF8AC1001EBCE
:106930004102C2EBC111B94A02EBC101097A40EA36
:1069400001209DF8AC1001EB4102C2EBC111B34A2A
:1069500002EBC101497A0843C117CDE9080108F0EB
:106960006DFC9DF8AC1040F2231211FB02F1AC4A11
:1069700002EBC10118319DF8982002EBC20201EB35
:106980000211C1F81A0020E2BDF89C0003281CD1B6
:106990008F229DF8AC0040F2231110FB01F0A049BA
:1069A00001EBC00118319DF8980000EBC00001EB2D
:1069B0000010427101219DF8AC0040F2231210FB3F
:1069C00002F0974A02EBC0000171FEE1BDF89C00A5
:1069D000032811D18F229DF8AC0040F2231110FB47
:1069E00001F08F4901EBC00018309DF8981001EBC1
:1069F000C10100EB01104271E7E1BDF89C000328E2
:106A000054D19DF8AC0040F2231110FB01F08449F1
:106A100001EBC0001830BDF8D01001EBC10100EB54
:106A200001108079012824D100229DF8AC0040F2A9
:106A3000231110FB01F07A4901EBC0011831BDF8B8
:106A4000D00000EBC00001EB001082718F229DF896
:106A5000AC0040F2231110FB01F0714901EBC001C1
:106A600018319DF8980000EBC00001EB0010427156
:106A70001CE008229DF8AC0040F2231110FB01F04D
:106A8000674901EBC00118319DF8980000EBC00088
:106A900001EB0010427100219DF8AC0040F223127E
:106AA00010FB02F05E4A02EBC00001718DE1BDF8FF
:106AB0009C00032854D19DF8AC0040F2231110FB38
:106AC00001F0574901EBC0001830BDF8D01001EBC0
:106AD000C10100EB01108079012824D100229DF82A
:106AE000AC0040F2231110FB01F04D4901EBC00155
:106AF0001831BDF8D00000EBC00001EB001082712E
:106B00008F229DF8AC0040F2231110FB01F04449A4
:106B100001EBC00018309DF8981001EBC10100EBAB
:106B2000011042711CE008229DF8AC0040F22311D4
:106B300010FB01F03A4901EBC00118319DF89800B3
:106B400000EBC00001EB0010427100219DF8AC0089
:106B500040F2231210FB02F0314A02EBC000017137
:106B600033E1BDF89C0008287DD19DF8AC0000EB16
:106B70004001C1EBC010294901EBC000807801063B
:106B80009DF8AC0000EB4002C2EBC010234A02EBC0
:106B9000C000C07841EA00419DF8AC0000EB400223
:106BA000C2EBC0101D4A02EBC000007941EA002090
:106BB0009DF8AC1001EB4102C2EBC111174A02EB88
:106BC000C10149790843C117CDE9080108F036FB36
:106BD0009DF8AC1040F2231211FB02F1104A02EBB7
:106BE000C10218329DF8981001EBC10102EB0111AE
:106BF00048639DF8AC0040F2231110FB01F00849F6
:106C000001EBC00018309DF8981001EBC10100EBBA
:106C1000011000789DF8AC1004E00000A47700207B
:106C2000C444002040F2231211FB02F1FE4A02EBA1
:106C3000C1014979884232DA00219DF8AC0040F266
:106C4000231210FB02F0F84A02EBC000017105228A
:106C50009DF8AC0040F2231110FB01F0F24901EB6A
:106C6000C001183101E07AE07CE09DF8980000EB6B
:106C7000C00001EB001002708E229DF8AC0040F2C3
:106C8000231110FB01F0E84901EBC00018309DF81A
:106C9000981001EBC10100EB011042715FE09DF81B
:106CA000AC0040F2231110FB01F0DF4901EBC00002
:106CB0001830BDF8D01001EBC10100EB0110807954
:106CC00001282FD100229DF8AC0040F2231110FBC7
:106CD00001F0D54901EBC0011831BDF8D00000EB3F
:106CE000C00001EB001082718F229DF8AC0040F2D1
:106CF000231110FB01F0CC4901EBC00118319DF8C4
:106D0000980000EBC00001EB0010427101219DF8DA
:106D1000AC0040F2231210FB02F0C34A02EBC000A9
:106D200001711CE08E229DF8AC0040F2231110FB93
:106D300001F0BD4901EBC00118319DF8980000EB4E
:106D4000C00001EB0010427100219DF8AC0040F240
:106D5000231210FB02F0B44A02EBC000017134E0D0
:106D6000FEE333E0BDF89C0003282ED100219DF8FE
:106D7000AC0040F2231210FB02F0AB4A02EBC00061
:106D8000017101229DF8AC0040F2231110FB01F0CB
:106D9000A54901EBC0011831BDF8D00000EBC000DF
:106DA00001EB001082718C229DF8AC0040F223119F
:106DB00010FB01F09C4901EBC00018309DF89810C1
:106DC00001EBC10100EB01104271FCE3BDF89C0036
:106DD0000F287CD19DF8AC0000EB400101EB0010C6
:106DE000924901EB0010007BE8BB00202C902D9015
:106DF0000021379120E0DDE92C10000240EA116209
:106E00000902CDE92C129DF8AC0000EB4001C1EB6A
:106E1000C010874901EBC001BDF8DC00C0F10600DD
:106E2000085CDDE92C3440EA0302CDE92C24BDF8EE
:106E3000DC00401C81B23791BDF8DC000528DADBAC
:106E40009DF8AC00DDE92C2140F2231310FB03F088
:106E5000754B03EBC00318339DF8980000EBC0009E
:106E600003EB001000E045E040F8222F41600022D3
:106E70002C922D920021379120E0DDE92C100002A8
:106E800040EA11620902CDE92C129DF8AC0000EB3A
:106E90004001C1EBC010664901EBC001BDF8DC0048
:106EA000C0F10B00085CDDE92C3440EA0302CDE9B7
:106EB0002C24BDF8DC00401C81B23791BDF8DC0009
:106EC0000528DADB9DF8AC00DDE92C1200E0F9E3DF
:106ED00040F2231310FB03F0534B03EBC0001830B8
:106EE0009DF8983003EBC30300EB03102230816060
:106EF000C2607EE000202C902D900021379120E090
:106F0000DDE92C10000240EA11620902CDE92C12E1
:106F10009DF8AC0000EB4001C1EBC010444901EB0F
:106F2000C001BDF8DC00C0F10700085CDDE92C34CD
:106F300040EA0302CDE92C24BDF8DC00401C81B2FC
:106F40003791BDF8DC000628DADB9DF8AC00DDE9FE
:106F50002C1240F2231310FB03F0334B03EBC0035E
:106F600018339DF8980000EBC00003EB001040F8C8
:106F7000221F426000222C922D92002137911FE0A7
:106F8000DDE92C10000240EA11620902CDE92C1261
:106F90009DF8AC0000EB4001C1EBC010244901EBAF
:106FA000C001BDF8DC00C0F10D00085CDDE92C3447
:106FB0001843CDE92C04BDF8DC00401C80B23790AA
:106FC000BDF8DC000628DBDB9DF8AC00DDE92C21F8
:106FD00040F2231310FB03F0134B03EBC0001830F7
:106FE0009DF8983003EBC30300EB0310223082605E
:106FF000C1609DF8AC0040F2231110FB01F00A497A
:1070000001EBC00118319DF8980000EBC00001EBC6
:10701000001001789DF8AC0040F2231210FB02F042
:10702000014A02EBC00005E0C444002004400020F7
:10703000A4770020407981427ED19DF8AC009DF874
:10704000981001EB0010C217CDE92C02FE4890F811
:10705000900708B39DF8AC0000EB400101EB001075
:10706000FA4901EB001030309DF8981000EB011048
:10707000807A022810D09DF8AC0000EB400101EBB3
:107080000010F24901EB001030309DF8981000EB31
:107090000110C07A00287CDD00229DF8AC0000EBD6
:1070A000400101EB0010E94901EB001030309DF880
:1070B000981000EB0110C272E548D0F80C020521CF
:1070C000B0FBF1F201FB120000EB4001E0482C3074
:1070D00000EB41100D3009909DF8AC0040F22311F7
:1070E00010FB01F0DB4901EBC00018309DF898104F
:1070F00001EBC10100EB0110223010220146089083
:107100000998F1F7A2F8D248D0F80C020521B0FB9B
:10711000F1F201FB120000EB4001CD482C3000EBF6
:1071200041129DF8AC0040F2231110FB01F0C94957
:1071300001EBC001183100E0C5E29DF8980000EBBA
:10714000C00001EB001050F81A1F42F8011F406800
:107150005060BF48D0F80C020521B0FBF1F201FBF2
:10716000120000EB4001BA482C3000EB41129DF8B0
:10717000AC0000EB400101EB0010B44901EB001141
:1071800030319DF8980001EB001000781070B04885
:1071900000E07CE1D0F80C020521B0FBF1F201FB2C
:1071A000120000EB4001AA482C3000EB4111AA4824
:1071B000C26841F81D2F008A8880A548D0F80C02CB
:1071C0000521B0FBF1F201FB120000EB4001A048E9
:1071D0002C3000EB41129DF8AC0040F2231110FB63
:1071E00001F09C4901EBC00118319DF8980000EBBB
:1071F000C00001EB0010406BC2F809009448D0F8C1
:107200000C020521B0FBF1F201FB120000EB400182
:107210008F482C3000EB41129DF8AC0000EB400190
:1072200001EB0010894901EB001130319DF8980005
:1072300001EB00104068C2F8230000229DF8AC006A
:1072400000EB400101EB0010804901EB00113031EF
:107250009DF8980001EB00104260002137914BE04F
:107260007B48D0F80C020521B0FBF1F201FB1200C3
:1072700000EB400176482C3000EB41112731BDF87E
:10728000DC409DF8AC0040F2231210FB02F0714A82
:1072900002EBC00218329DF8980000EBC00002EB30
:1072A000001090F87F0040F2231210FB02F0694AB0
:1072B00002EBC00218329DF8AC0040F2231310FB21
:1072C00003F0644B03EBC00318339DF8980000EB08
:1072D000C00003EB001090F8800000EBC00002EB50
:1072E00000123F32BDF8DC00001D105C0855BDF8EF
:1072F000DC00401C81B23791BDF8DC000628AFDB12
:107300000021379139E000239DF8AC0040F22311B1
:1073100010FB01F04F4901EBC00118319DF89800B6
:1073200000EBC00001EB001090F87F0040F2231149
:1073300010FB01F0474901EBC00118319DF8AC008A
:1073400040F2231210FB02F0424A02EBC002183254
:107350009DF8980000EBC00002EB001090F8800050
:1073600000EBC00001EB00113F31BDF8DC000B5415
:10737000BDF8DC00401C81B23791BDF8DC000A2862
:10738000C1DB3348D0F80C020521B0FBF1F080B22C
:10739000014609900220F1F79BFE00210620F2F73A
:1073A00043FE2B48D0F80C022949498D884206D269
:1073B0002748D0F80C02401C2549C1F80C020021D6
:1073C0000520F2F731FE9DF8AC0000EB400101EB27
:1073D00000101E4901EB001030309DF8981000EBB2
:1073E0000110801C0990007820F0080209980270B2
:1073F0001748D0F80C020521B0FBF1F201FB120096
:1074000000EB400112482C3000EB4110D0F8232053
:107410002C9800EB4001114800EB4110C0F82320EC
:10742000002037902EE00A48D0F80C020521B0FB6E
:10743000F1F201FB120000EB400105482C3000EB9B
:10744000411027300CE00000BC3200200440002036
:10745000BC120020C4440020BC310020D8140020FD
:10746000BDF8DC10425C2C9800EB4001FE4800EBBC
:1074700041112731BDF8DC000A54BDF8DC00401C86
:1074800081B23791BDF8DC000628CCDB56E09DF8D0
:10749000AC0000EB400101EB0010F44901EB0010DF
:1074A00030309DF8981000EB0110801C0990007896
:1074B00020F008010831099801709DF8AC0000EB3C
:1074C000400101EB0010E94901EB001130319DF85A
:1074D000980001EB001041682C9800EB4002E24854
:1074E00000EB4210C0F823100021379122E09DF8F4
:1074F000AC0040F2231110FB01F0DD4901EBC001AB
:1075000018319DF8980000EBC00001EB00113F31ED
:10751000BDF8DC000A5C2C9800EB4001D24800EB7F
:1075200041112731BDF8DC000A54BDF8DC00401CD5
:1075300081B23791BDF8DC000628D8DB9DF8AC009D
:1075400000EB400101EB0010C84901EB00103030A6
:107550009DF8981000EB0110801C0990007800E065
:1075600016E120F02002099802709DF8AC1002206C
:10757000F2F75AFD9DF8AC0040F2231110FB01F028
:10758000BB4901EBC00018309DF8981001EBC10118
:1075900000EB0110223009902C9800EB4001B2481A
:1075A00000EB41100D30102208900999F0F74DFEC4
:1075B0009DF8AC0040F2231110FB01F0AC4901EB47
:1075C000C001183100E0A1E19DF8980000EBC00077
:1075D00001EB00112C9800EB4002A34800EB421095
:1075E00051F81A2F40F8012F496841609DF8AC000E
:1075F00000EB400101EB00109C4901EB0011303120
:107600009DF8980001EB001001782C9800EB4002E7
:10761000954800EB421001702C9800EB4001924815
:1076200000EB41119348C26841F81D2F008A888001
:107630009DF8AC0040F2231110FB01F08C4901EBE6
:10764000C00118319DF8980000EBC00001EB00105C
:10765000416B2C9800EB4002834800EB4210C0F8CD
:1076600009109DF8AC0000EB400101EB00107F49D0
:1076700001EB001130319DF8980001EB00104168DA
:107680002C9800EB4002784800EB4210C0F8231021
:107690002C9881B208200991F2F7C6FC00229DF8CF
:1076A000AC0040F2231110FB01F0714901EBC00066
:1076B00018309DF8981001EBC10100EB011080F823
:1076C0003E2052E063E09DF8AC0000EB400101EB8E
:1076D0000010664901EB001030309DF8981000EB67
:1076E0000110801C0990007820F00400001D099909
:1076F00008709DF8AC0000EB400101EB00105B4905
:1077000001EB001030309DF8981000EB0110801C48
:107710000990007820F080008030099908700120DD
:107720009DF8AC1040F2231211FB02F1504A02EB1B
:10773000C10108719DF8AC0040F2231110FB01F06B
:10774000114601EBC00042799DF8AC0040F22311D4
:1077500010FB01F0464901EBC00018309DF898106D
:1077600001EBC10100EB011002708F229DF8AC000B
:1077700040F2231110FB01F03D4901EBC00018302D
:107780009DF8981001EBC10100EB01104271BDE0C2
:10779000BDF89C0003284FD10121374880F8B4166A
:1077A0009DF8AC0040F2231110FB01F0304901EBD1
:1077B000C00118319DF8980000EBC00001EB0010EB
:1077C00001789DF8AC0040F2231210FB02F0284A29
:1077D00002EBC000407981422FDA00219DF8AC0015
:1077E00040F2231210FB02F0214A02EBC0000171AB
:1077F00001229DF8AC0040F2231110FB01F01C495E
:1078000001EBC00118319DF8980000EBC00001EBBE
:10781000001002708F229DF8AC0040F2231110FB83
:1078200001F0134901EBC00018309DF8981001EBEE
:10783000C10100EB011042714CE09DF8AC0040F238
:10784000231110FB01F00A4901EBC00018309DF82C
:10785000981001EBC10100EB01108078802839D12C
:1078600000219DF8AC0009E0D8140020044000205D
:10787000C4440020BC310020BC32002040F223125E
:1078800010FB02F0FE4A02EBC000017180229DF85D
:10789000AC0040F2231110FB01F0F94901EBC001EB
:1078A00018319DF8980000EBC00001EB0010427108
:1078B00000229DF8AC0040F2231110FB01F0F049CA
:1078C00001EBC00018309DF8981001EBC10100EBEE
:1078D000011082701AE0BDF89C00032815D1002128
:1078E000E84880F8B4168F229DF8AC0040F22311CE
:1078F00010FB01F0E24901EBC00018309DF8981030
:1079000001EBC10100EB0110427100BF00BF00BFDD
:1079100000BFDD4890F80B0FB0B1DC499DF8AC001A
:1079200031F8101009919DF8AC1001EB4100C0EB4B
:10793000C110D74901EBC001012308919DF8AC208B
:10794000DDE90801F3F720F90021379111E000216A
:107950009DF8AC0000EB4002C2EBC010CC4A02EB39
:10796000C002BDF8DC001154BDF8DC00401C81B23F
:107970003791BDF8DC00142843DAE8E7C5499DF8E3
:10798000AC0011F81000C009D8BB9DF8AC0011F88C
:107990001000C0F3C300062832D2DFE800F0036213
:1079A00091FEFD339DF8AC0000EB4001C1EBC0102F
:1079B000B74901EBC0010991B7A1099815F02EFE56
:1079C00011901198E0B100219DF8AC0000EB40004F
:1079D000B04A3C3202EB8000416001219DF8AC00CE
:1079E00000EB400002EB80008170AA499DF8AC00DA
:1079F00001EB40010991087820F0780028300870E8
:107A000062E162E19DF8AC0000EB4001C1EBC01007
:107A10009F4901EBC00109919FA1099815F0FEFD56
:107A200011901198E0B100219DF8AC0000EB4000EE
:107A3000984A3C3202EB8000416001219DF8AC0085
:107A400000EB400002EB8000817092499DF8AC0091
:107A500001EB40010991087820F07800203008708F
:107A600032E19DF8AC0000EB4001C1EBC010884949
:107A700001EBC001099188A1099815F0CFFD119083
:107A80001198E0B100219DF8AC0000EB4000814A64
:107A90003C3202EB8000416001219DF8AC0000EB1C
:107AA000400002EB800081707A499DF8AC0001EB48
:107AB00040010991087820F078001830087003E13F
:107AC00000219DF8AC0000EB4000724A3C3202EB12
:107AD0008000416001219DF8AC0000EB400002EB0A
:107AE000800081709DF8AC0000EB4001C1EBC0103C
:107AF000674901EBC0011198801D095C30399DF880
:107B0000AC0000EB4002C2EBC010614A02EBC003C4
:107B10001198401D185C303841EA0010C117CDE9BA
:107B2000080106F0D7FD5D4988719DF8AC0000EBB7
:107B30004001C1EBC010564901EBC001099158A1A9
:107B4000099815F06BFD1190119838B39DF8AC00B1
:107B500000EB4001C1EBC0104D4901EBC001119891
:107B6000401C085C302826DB9DF8AC0000EB40018F
:107B7000C1EBC010464901EBC0011198401C085CE4
:107B800030389DF8AC1001EB4102C2EBC111404A04
:107B900002EBC103119902E058E02BE01EE0595CB2
:107BA000303940EA0110C117CDE9080106F092FD15
:107BB0003A49C87112E09DF8AC0000EB4001C1EBFE
:107BC000C010334901EBC0011198085C3038C1176F
:107BD000CDE9080106F07EFD3049C8712D499DF8B8
:107BE000AC0001EB40010991087820F078001830D2
:107BF000087069E09DF8AC0000EB4001C1EBC010DB
:107C0000234901EBC001099123A1099815F006FD54
:107C100011901198C8B10020224908601D499DF8B3
:107C2000AC0001EB40010991087820F0800180311F
:107C3000099801704FF47A719DF8AC0000EB400098
:107C4000144A3C3202EB800081603DE09DF8AC00BC
:107C500000EB4001C1EBC0100D4901EBC0010991DF
:107C60000DA1099815F0DAFC1190119858B3054848
:107C700090F8B60620F08001024880F8B61613E0AE
:107C8000C4440020BC320020BC2200202469002013
:107C9000A4770020CC3D00204F4B00004C3A002040
:107CA0002C0000008802424210499DF8AC0001EB14
:107CB00040010991087820F0780008300870002011
:107CC0000B498870486000BF00BF0A4800780A4925
:107CD0000978084409490978084409490978084499
:107CE000002873F467A938B070BD0000CC3D0020B7
:107CF00064690020120000201300002014000020FE
:107D00001500002007B5D4B000211A9119911891DF
:107D100017911691159114910022129213921092BC
:107D200011920F910E910D910C910B910A91F7A068
:107D300006C8CDE90812F7A006C8CDE90612002151
:107D400005910020F5490870549800EB400101EBC3
:107D50000010F34901EB001081791691F149549814
:107D600001EB00115598085C05287DDD0621ED4AE0
:107D7000549802EB001255981154002240F223113E
:107D800054984843E84901EBC0011831559800EB7D
:107D9000C00001EB00100270549800EB400101EBB1
:107DA0000010DF4901EB00113031559801EB001054
:107DB000807820F08002549800EB400101EB001025
:107DC000D74901EB00113031559801EB001082705A
:107DD00040F2231154984843D34901EBC0011831B4
:107DE000559800EBC00001EB001090F88E0020F0D9
:107DF000080240F2231154984843CB4901EBC001DB
:107E00001831559800EBC00001EB001080F88E206F
:107E100040F2231154984843C34901EBC001183183
:107E2000559800EBC00001EB001090F88E0020F098
:107E3000010240F2231154984843BB4901EBC001B1
:107E40001831559800EBC00001EB001080F88E202F
:107E5000549800EB400101EB0010B14901EB001018
:107E60008079092817D200E087E0DFE800F0850577
:107E70001525354555657500E52240F223115498C6
:107E80004843A94901EBC0001830559901EBC101E5
:107E900000EB011042716FE0A12240F223115498CF
:107EA0004843A14901EBC0001830559901EBC101CD
:107EB00000EB011042715FE0A12240F223115498BF
:107EC0004843994901EBC0001830559901EBC101B5
:107ED00000EB011042714FE0B12240F2231154989F
:107EE0004843914901EBC0001830559901EBC1019D
:107EF00000EB011042713FE0312240F2231154980F
:107F00004843894901EBC0001830559901EBC10184
:107F100000EB011042712FE0F42240F2231154983B
:107F20004843814901EBC0001830559901EBC1016C
:107F300000EB011042711FE0062240F22311549819
:107F40004843794901EBC0001830559901EBC10154
:107F500000EB011042710FE0152240F223115498FA
:107F60004843714901EBC0001830559901EBC1013C
:107F700000EB0110427100BF00BF6A496C39549890
:107F800011F810000121B1EBD01F46F0B98167480C
:107F900090F82800012806F0A4819DF858000028D8
:107FA000F9D09DF858000A2886F03281DFE810F0F9
:107FB000E12A0A0048090C0E8012F61538172D2008
:107FC000E326642D549800EB400101EB0010544966
:107FD00001EB00113031559801EB00104178084653
:107FE0000491002107F02AF9C1B2159140F2231142
:107FF000549848434C4901EBC0011831559800EBA7
:10800000C00001EB0010017840F223125498504355
:10801000454A02EBC0004079814208D1012140F27B
:10802000231254985043404A02EBC00001713D496D
:10803000549801EB00115598085C401CC1B2394AB4
:10804000549802EB00125598115440F223115498A1
:108050004843354901EBC0001830559901EBC10187
:1080600000EB011090F88E00C0F3C00090B154985E
:1080700000EB400101EB0010294901EB00104179B0
:108080000B464FF4805204914FF4E131549806F0BE
:10809000C3FF19E0549800EB400101EB00102049A8
:1080A00001EB001041790491549800EB400101EB81
:1080B00000101B4901EB0010016803914FF480523E
:1080C000049B549806F0A8FF5698C52876D012DC79
:1080D000B52874D008DC112872D0122871D013286A
:1080E00070D0B22869D1A0E3B6286CD0B9286BD083
:1080F000C328F7D1DCE2D92868D019DCCA287DD0A2
:10810000CE287CD0D528EDD119E0000001693230AD
:108110003130300001693230453030001600002027
:1081200004400020383E0020C4440020BC1200203F
:10813000E12865D0E5287DD0E728D3D1FAE3F52101
:108140005498C0EB001000EB8000F54A02F83010A4
:108150009DF854105498C0EB001000EB800002EB27
:10816000C0004170A2215498C0EB001000EB8000C9
:1081700002EBC0008170D5215498C0EB001000EBD9
:10818000800002EBC000C1705498C0EB001000EBFF
:108190008000114601EBC00104910321049806F010
:1081A00029FF01465498C0EB001000EB8000DC4A28
:1081B00002EBC000017105210F91FDE3FDE34AE0F0
:1081C000FCE3FCE3FCE3F1E258E1FFE7F52154981E
:1081D000C0EB001000EB8000D14A02F830109DF88F
:1081E00054105498C0EB001000EB800002EBC0006C
:1081F0004170A2215498C0EB001002E097E2F4E332
:10820000F4E300EB800002EBC0008170D9215498A8
:10821000C0EB001000EB800002EBC000C17054986E
:10822000C0EB001000EB8000114601EBC00104918F
:10823000032100E0FAE3049806F0DCFE01465498BE
:10824000C0EB001000EB8000B54A02EBC0000171EA
:1082500005210F91B1E7F5215498C0EB001000EB18
:108260008000AF4A02F830109DF854105498C0EBCB
:10827000001000EB800002EBC0004170549800EB4E
:10828000400101EB0010A74901EB0010007B002822
:108290007AD140F2231154984843A34901EBC0001E
:1082A0001830559901EBC10100EB01108068B0F561
:1082B000100F05D34FF410000021CDE9100110E09C
:1082C00040F2231154984843974901EBC0001830FD
:1082D000559901EBC10100EB011080680022CDE946
:1082E0001002A5215498C0EB001000EB80008C4ACE
:1082F00002EBC000817000211A911CE0BDF86800FB
:10830000C0F10200C200DDE91001CDE91B10EFF75A
:108310008AFFC2B25498C0EB001000EB8000804985
:1083200001EBC003BDF86800C01C1A54BDF868001A
:10833000401C80B21A90BDF868000328DEDBB5212E
:108340005498C0EB001000EB8000754A02EBC000AF
:1083500081715498C0EB001000EB8000114601EBD6
:10836000C00104910621049806F044FE0146549889
:10837000C0EB001000EB8000694A02EBC000C17145
:1083800008210F9179E0FFE740F223115498484308
:10839000654901EBC0001830559901EBC10100EBB4
:1083A00001108068B0F1104F05D34FF0104000214C
:1083B000CDE9100110E040F22311549848435A4986
:1083C00001EBC0001830559901EBC10100EB011021
:1083D00080680022CDE91002A6215498C0EB00105D
:1083E00000EB80004E4A02EBC000817000211A9120
:1083F0001CE0BDF86800C0F10300C200DDE9100117
:10840000CDE91D10EFF70FFFC2B25498C0EB00107A
:1084100000EB8000424901EBC003BDF86800C01CBE
:108420001A54BDF86800401C80B21A90BDF868006C
:108430000428DEDBB5215498C0EB001000EB80006F
:10844000374A02EBC000C1715498C0EB001000EB3A
:108450008000114601EBC00104910721049806F049
:10846000C9FD01465498C0EB001000EB80002C4A77
:1084700002EBC000017209210F919EE6F52154988C
:10848000C0EB001000EB8000254A02F830109DF888
:1084900054105498C0EB001000EB800002EBC000B9
:1084A0004170549800EB400101EB00101D4901EBB5
:1084B0000010007BD0BB40F22311549848431A4966
:1084C00001EBC0001830559901EBC10100EB011020
:1084D0008068B0F5100F05D14FF410000021CDE9F0
:1084E000100110E040F22311549848430E4901EB6B
:1084F000C0001830559901EBC10100EB01108068F4
:108500000022CDE91002A5215498C0EB001000EB29
:108510008000034A02EBC000817000211A9123E021
:10852000446E002004400020C444002044E0BDF814
:108530006800C0F10200C200DDE91001CDE91F10A2
:10854000EFF771FEC2B25498C0EB001000EB800050
:10855000F94901EBC003BDF86800C01C1A54BDF80E
:108560006800401C80B21A90BDF868000328DEDB6A
:10857000B9215498C0EB001000EB8000EE4A02EBEA
:10858000C00081715498C0EB001000EB80001146D0
:1085900001EBC00104910621049806F02BFD014671
:1085A0005498C0EB001000EB8000E34A02EBC000DF
:1085B000C17108210F917AE040F223115498484389
:1085C000DE4901EBC0001830559901EBC10100EB09
:1085D00001108068B0F1104F05D14FF0104000211C
:1085E000CDE9100110E040F2231154984843D349DB
:1085F00001EBC0001830559901EBC10100EB0110EF
:1086000080680022CDE91002A6215498C0EB00102A
:1086100000EB8000C84A02EBC000817000211A9173
:108620001EE0BDF86800C0F10300C200DDE91010D3
:10863000CDE9210108462199EFF7F5FDC2B2549822
:10864000C0EB001000EB8000BB4901EBC003BDF89C
:108650006800C01C1A54BDF86800401C80B21A9013
:10866000BDF868000428DCDBB9215498C0EB001089
:1086700000EB8000B04A02EBC000C1715498C0EB1F
:10868000001000EB8000114601EBC00104910721AE
:10869000049806F0AFFC01465498C0EB001000EBC4
:1086A0008000A54A02EBC000017209210F9184E508
:1086B000F5215498C0EB001000EB80009E4A02F8B0
:1086C00030109DF854105498C0EB001000EB80005F
:1086D00002EBC0004170A2215498C0EB001000EBE7
:1086E000800002EBC0008170C3215498C0EB0010E1
:1086F00000EB800002EBC000C1705498C0EB00108A
:1087000000EB8000114601EBC001049103210498A5
:1087100006F070FC01465498C0EB001000EB80009E
:10872000854A02EBC000017105210F9145E5F52155
:108730005498C0EB001000EB80007F4A02F8301024
:108740009DF854105498C0EB001000EB800002EB31
:10875000C0004170A2215498C0EB001000EB8000D3
:1087600002EBC0008170CA215498C0EB001000EBEE
:10877000800002EBC000C1705498C0EB001000EB09
:108780008000114601EBC00104910321049806F01A
:1087900031FC01465498C0EB001000EB8000664AA3
:1087A00002EBC000017105210F9106E5F5215498F7
:1087B000C0EB001000EB80005F4A02F830109DF81B
:1087C00054105498C0EB001000EB800002EBC00086
:1087D0004170A2215498C0EB001000EB800002EB26
:1087E000C0008170B6215498C0EB001000EB8000EF
:1087F00002EBC000C1705498C0EB001000EB800089
:10880000114601EBC00104910321049806F0F2FB2C
:1088100001465498C0EB001000EB8000464A02EB82
:10882000C000017105210F91C7E4F5215498C0EBF8
:10883000001000EB8000404A02F830109DF8541000
:108840005498C0EB001000EB800002EBC0004170B8
:10885000549800EB400101EB0010394901EB001086
:10886000007BE0BBA4215498C0EB001000EB80001B
:1088700002EBC000817000211A9124E040F2231124
:10888000549848432D4901EBC0011831559800EB2D
:10889000C00001EB0010416BBDF86800C0F10100A1
:1088A000C000C1405498C0EB001000EB8000224A89
:1088B00002EBC002BDF86800C01C1154BDF868008E
:1088C000401C81B21A91BDF868000228D6DBB221A3
:1088D0005498C0EB001000EB8000174A00E01CE049
:1088E00002EBC00041715498C0EB001000EB800017
:1088F000114601EBC00104910521049806F07AFBB2
:1089000001465498C0EB001000EB80000A4A02EBCD
:10891000C000817107210F9166E0A5215498C0EB3A
:10892000001000EB8000044A02EBC00081700021BF
:108930001A912CE092E20000446E0020C444002012
:108940000440002040F2231154984843F74901EBBA
:10895000C0011831559800EBC00001EB0010416BCD
:10896000BDF86800C0F10200C000C1405498C0EBDF
:10897000001000EB8000EE4A02EBC002BDF8680078
:10898000C01C1154BDF86800401C81B21A91BDF89A
:1089900068000328D6DBB2215498C0EB001000EB2E
:1089A0008000E34A02EBC00081715498C0EB0010D4
:1089B00000EB8000114604E010E285E08DE2E9E280
:1089C00042E301EBC00104910621049806F012FB7A
:1089D00001465498C0EB001000EB8000D44A02EB33
:1089E000C000C17108210F91F8E1ACE0FFE7F5216B
:1089F0005498C0EB001000EB8000CD4A02F8301014
:108A00009DF854105498C0EB001000EB800002EB6E
:108A1000C0004170A6215498C0EB001000EB80000C
:108A200002EBC000817000211A9125E0D7E140F2ED
:108A3000231154984843BD4901EBC00118315598A2
:108A400000EBC00001EB0010816BBDF86800C0F1C5
:108A50000300C000C1405498C0EB001000EB800040
:108A6000B34A02EBC002BDF86800C01C1154BDF847
:108A70006800401C81B21A91BDF868000428D6DB5A
:108A8000E1215498C0EB001000EB8000A84A02EBF3
:108A9000C000C1715498C0EB001000EB800011467B
:108AA00001EBC00104910721049806F0A3FA0146E6
:108AB0005498C0EB001000EB80009D4A02EBC00010
:108AC000017209210F91B8E3F5215498C0EB001011
:108AD00000EB8000964A02F830109DF8541054982C
:108AE000C0EB001000EB800002EBC0004170A2213F
:108AF0005498C0EB001000EB800002EBC0008170C6
:108B0000C5215498C0EB001000EB800002EBC000C0
:108B1000C1705498C0EB001000EB8000114601EBCF
:108B2000C00104910321049806F064FA01465498A8
:108B3000C0EB001000EB80007D4A02EBC000017129
:108B400005210F9179E3F5215498C0EB001000EB5B
:108B50008000774A02F830109DF854105498C0EB0A
:108B6000001000EB800002EBC0004170549800EB55
:108B7000400101EB00116F4800EB0110007BE8BBE6
:108B8000AC215498C0EB001000EB800002EBC00059
:108B9000817000211A912CE040F22311549848432F
:108BA000624901EBC0001830559901EBC10100EB9F
:108BB000011050F8221F4068BDF86820C2F104027D
:108BC000D200CDE9230108462399EFF72CFBC2B26E
:108BD0005498C0EB001000EB8000554901EBC00336
:108BE000BDF86800C01C1A54BDF86800401C80B273
:108BF0001A90BDF868000528CEDB00E057E00021A0
:108C00001A912CE040F2231154984843474901EB54
:108C1000C0001830559901EBC10100EB0110223062
:108C20008168C068BDF86820C2F10402D200CDE9B5
:108C3000250108462599EFF7F6FAC2B25498C0EB21
:108C4000001000EB80003A4901EBC003BDF868005A
:108C500008301A54BDF86800401C80B21A90BDF864
:108C600068000528CEDBCE215498C0EB001000EB45
:108C700080002F4A02EBC00041735498C0EB0010F3
:108C800000EB8000114601EBC00104910D21049816
:108C900006F0B0F901465498C0EB001000EB8000DC
:108CA000234A02EBC00081730F210F9196E0AE21A1
:108CB0005498C0EB001000EB80001D4A02EBC0008E
:108CC000817000211A912AE040F223115498484300
:108CD000164901EBC0001830559901EBC10100EBBA
:108CE000011151F8220F4968BDF86820C2F1050250
:108CF000D200CDE92710EFF796FAC2B25498C0EB34
:108D0000001000EB80000A4901EBC003BDF86800C9
:108D1000C01C1A54BDF86800401C80B21A90BDF8FF
:108D200068000628D0DB00211A9130E0C4440020FE
:108D3000446E00200440002040F223115498484320
:108D4000FE4901EBC0001830559901EBC10100EB61
:108D5000011122318868C968BDF86820C2F1050296
:108D6000D200CDE92910EFF75EFAC2B25498C0EBF9
:108D7000001000EB8000F24901EBC003BDF8680071
:108D800009301A54BDF86800401C80B21A90BDF832
:108D900068000628D0DBCE215498C0EB001000EB11
:108DA0008000E74A02EBC000C1735498C0EB00108A
:108DB00000EB8000114601EBC00104910F210498E3
:108DC00006F018F901465498C0EB001000EB800043
:108DD000DB4A02EBC000017411210F912DE2F52155
:108DE0005498C0EB001000EB8000D54A02F8301018
:108DF0009DF854105498C0EB001000EB800002EB7B
:108E0000C0004170A2215498C0EB001000EB80001C
:108E100002EBC0008170E5215498C0EB001000EB1C
:108E2000800002EBC000C1705498C0EB001000EB52
:108E30008000114601EBC00104910321049806F063
:108E4000D9F801465498C0EB001000EB8000BC4AF2
:108E500002EBC000017105210F91EEE1F52154985C
:108E6000C0EB001000EB8000B54A02F830109DF80E
:108E700054105498C0EB001000EB800002EBC000CF
:108E80004170A2215498C0EB001000EB800002EB6F
:108E9000C0008170E7215498C0EB001000EB800007
:108EA00002EBC000C1705498C0EB001000EB8000D2
:108EB000114601EBC00104910321049806F09AF8D1
:108EC00001465498C0EB001000EB80009C4A02EB76
:108ED000C000017105210F91AFE1F5215498C0EB5D
:108EE000001000EB8000964A02F830109DF85410F4
:108EF0005498C0EB001000EB800002EBC000417002
:108F0000A2215498C0EB001000EB800002EBC000DF
:108F1000817011215498C0EB001000EB800002EB2F
:108F2000C000C1705498C0EB001000EB80001146E7
:108F300001EBC00104910321049806F05BF801469F
:108F40005498C0EB001000EB80007D4A02EBC0009B
:108F5000017105210F91012240F2231154984843D9
:108F6000764901EBC0011831559800EBC00001EBC8
:108F700000100270D52240F22311549848436F49E3
:108F800001EBC0001830559901EBC10100EB011055
:108F9000427152E1F5215498C0EB001000EB8000C3
:108FA000674A02F830109DF854105498C0EB001036
:108FB00000EB800002EBC0004170A5215498C0EB8B
:108FC000001000EB800002EBC0008170012154987A
:108FD000C0EB001000EB800002EBC000C170C221AA
:108FE0005498C0EB001000EB800002EBC000017150
:108FF00000215498C0EB001000EB800002EBC00091
:10900000417112215498C0EB001000EB800002EB7C
:10901000C00081715498C0EB001000EB8000114635
:1090200001EBC00104910621049805F0E3FF01461D
:109030005498C0EB001000EB8000414A02EBC000E6
:10904000C17108210F91F8E0F5215498C0EB001090
:1090500000EB80003A4A02F830109DF85410549802
:10906000C0EB001000EB800002EBC0004170FF215C
:109070005498C0EB001000EB800002EBC000817040
:1090800000211A911CE0549800EB400101EB001004
:109090002C4901EB00110E31BDF86800095C5498B1
:1090A000C0EB001000EB8000254A02EBC002BDF8C7
:1090B0006800C01C1154BDF86800401C81B21A91B0
:1090C000BDF868000A28DEDB549800EB400101EB94
:1090D00000101C4901EB0010408B01125498C0EBAA
:1090E000001000EB8000164A02EBC0004173549858
:1090F00000EB400101EB0010124901EB0010408B26
:10910000C1B25498C0EB001000EB800002EBC0002D
:10911000817340F2231154984843084901EBC00180
:109120001831559800EBC00001EB0010B0F88C002E
:1091300001125498C0EB001006E00000C444002067
:10914000446E00200440002000EB800002EBC000D1
:10915000C17340F2231154984843FC4901EBC0010C
:109160001831559800EBC00001EB0010B0F88C00EE
:10917000C1B25498C0EB001000EB800002EBC000BD
:10918000017440F2231154984843F04901EBC001A7
:109190001831559800EBC00001EB0010B0F88C10AE
:1091A000549801EB802081B203200491EFF7F4FE84
:1091B00000211A9114E0E649BDF86800095C549852
:1091C000C0EB001000EB8000E24A02EBC002BDF8E9
:1091D000680011301154BDF86800401C81B21A912A
:1091E000BDF86800B0F5007FE5DB13215498C0EBB3
:1091F000001000EB8000D74A02EBC00080F811128B
:109200005498C0EB001000EB8000114601EBC00148
:10921000049140F21121049805F0ECFE01465498A7
:10922000C0EB001000EB8000CA4A02EBC00080F8DF
:10923000121240F213210F9100BF00BF04F0E8BFEB
:10924000549800EB400101EB0010C34901EB001101
:109250003031559801EB00104178159140F22311FF
:1092600054984843B94901EBC0011831559800EBB7
:10927000C00001EB0010017840F2231254985043D3
:10928000B24A02EBC0004079814208D1012140F28C
:10929000231254985043AD4A02EBC0000171AF490C
:1092A000549801EB00115598085C401CC1B2AB4AC0
:1092B000549802EB0012559811549DF85400002860
:1092C00004DD9DF85400401EC1B215915698A13896
:1092D0000A287CD2DFE800F0FEFDFCFBFAF9F80575
:1092E000F7F602215498C0EB001000EB8000994A79
:1092F00002F830109DF854004030C1B25498C0EBD1
:10930000001000EB800002EBC00041704121549836
:10931000C0EB001000EB800002EBC0008170302138
:109320005498C0EB001000EB800002EBC000C1704D
:109330005498C0EB001000EB800002EBC0000171FC
:1093400040F2231154984843804901EBC001183181
:10935000559800EBC00001EB00100079010954980A
:10936000C0EB001000EB800002EBC000417154988C
:10937000C0EB001000EB8000114601EBC00040790B
:109380000A2812DA5498C0EB001000EB800001EBC1
:10939000C00040793030C1B25498C0EB001000EBEF
:1093A000800002EBC000417115E05498C0EB001042
:1093B00000EB8000674901EBC00040793730C1B253
:1093C0005498C0EB001000EB8000624A00E005E218
:1093D00002EBC000417140F22311549848435B49AD
:1093E00001EBC0011831559800EBC00001EB0010F3
:1093F000007900F00F015498C0EB001000EB8000E2
:10940000544A02EBC00081715498C0EB001000EB8D
:109410008000114601EBC00080790A2812DA5498C6
:10942000C0EB001000EB800001EBC0008079303011
:10943000C1B25498C0EB001000EB800002EBC000FA
:10944000817113E05498C0EB001000EB800041499B
:1094500001EBC00080793730C1B25498C0EB0010E6
:1094600000EB80003B4A02EBC0008171032254985C
:10947000C0EB001000EB8000364901EBC000C27168
:109480005498C0EB001000EB800001EBC000401CC2
:1094900007210490F0F71EF801465498C0EB001025
:1094A00000EB80002B4A02EBC000017209210F91F2
:1094B000002140F2231254985043244A02EBC0008A
:1094C000017108E01CE19EE066E350E3A1E286E161
:1094D000ECE045E00FE0082240F2231154984843A5
:1094E0001A4901EBC0011831559800EBC00001EB9F
:1094F0000010027065E304215498C0EB001000EBEB
:109500008000144A02F830109DF854004030C1B277
:109510005498C0EB001000EB800002EBC0004170DB
:1095200051215498C0EB001000EB800002EBC0000A
:10953000817005215498C0EB001000EB800002EB15
:10954000C000C17004210F913BE30000C44400201F
:10955000C62F0020446E002004400020383E00202A
:1095600002215498C0EB001000EB8000FE4A02F884
:1095700030109DF854004030C1B25498C0EB001038
:1095800000EB800002EBC000417041215498C0EB19
:10959000001000EB800002EBC00081703121549874
:1095A000C0EB001000EB800002EBC000C170352161
:1095B0005498C0EB001000EB800002EBC00001717A
:1095C00003215498C0EB001000EB800002EBC000B8
:1095D00041715498C0EB001000EB8000114601EB84
:1095E000C000401C05210490EFF774FF0146549819
:1095F000C0EB001000EB8000DB4A02EBC000817181
:1096000007210F91DDE202215498C0EB001000EB1E
:109610008000D54A02F830109DF854004030C1B2A5
:109620005498C0EB001000EB800002EBC0004170CA
:1096300041215498C0EB001000EB800002EBC00009
:10964000817032215498C0EB001000EB800002EBD7
:10965000C000C17030215498C0EB001000EB8000B6
:1096600002EBC000017103215498C0EB001000EB25
:10967000800002EBC00041715498C0EB001000EB79
:109680008000114601EBC000401C05210490EFF75B
:1096900021FF01465498C0EB001000EB8000B24A55
:1096A00002EBC000817107210F918AE204215498D6
:1096B000C0EB001000EB8000AB4A02F830109DF8C0
:1096C00054004030C1B25498C0EB001000EB800051
:1096D00002EBC000417041215498C0EB001000EB38
:1096E000800002EBC000817005215498C0EB00108F
:1096F00000EB800002EBC000C17004210F9160E21A
:1097000002215498C0EB001000EB8000964A02F84A
:1097100030109DF854004030C1B25498C0EB001096
:1097200000EB800002EBC000417041215498C0EB77
:10973000001000EB800002EBC000817031215498D2
:10974000C0EB001000EB800002EBC000C1703221C2
:109750005498C0EB001000EB800002EBC0000171D8
:1097600003215498C0EB001000EB800002EBC00016
:1097700041715498C0EB001000EB8000114601EBE2
:10978000C000401C05210490EFF7A4FE0146549848
:10979000C0EB001000EB8000734A02EBC000817147
:1097A00007210F91549800EB400101EB00106F4925
:1097B00001EB00113031559801EB0010807820F05A
:1097C0002002549800EB400101EB0010674901EBC7
:1097D00000103030559900EB01108270F1E1022148
:1097E0005498C0EB001000EB80005F4A02F8301084
:1097F0009DF854004030C1B25498C0EB001000EB0B
:10980000800002EBC000417041215498C0EB001071
:1098100000EB800002EBC000817031215498C0EB56
:10982000001000EB800002EBC000C17030215498A2
:10983000C0EB001000EB800002EBC000017140F2B1
:109840002311549848434A4901EBC00018305599F8
:1098500001EBC10100EB01108068B0F5100F09D3D6
:1098600030215498C0EB001000EB800002EBC000E8
:10987000417109E032215498C0EB001000EB8000E8
:10988000394A02EBC000417140F223115498484319
:10989000374901EBC0001830559901EBC10100EBCD
:1098A0000110C07901280AD131215498C0EB001071
:1098B00000EB80002C4A02EBC000817118E040F2FE
:1098C0002311549848432A4901EBC0001830559998
:1098D00001EBC10100EB0110C07948B93221549865
:1098E000C0EB001000EB80001F4A02EBC00081714A
:1098F00000201A9027E040F22311549848431C4955
:1099000001EBC0011831559800EBC00001EB0010CD
:109910008168BDF86800C0F105008000C14001F019
:109920000F0130315498C0EB001000EB80000E4A5C
:1099300002EBC002BDF86800C01D1154BDF86800FC
:10994000401C81B21A91BDF868000628D3DB322191
:109950005498C0EB001000EB8000034A02EBC000FB
:10996000417300211A912DE0446E00200440002034
:10997000C444002040F2231154984843F94901EBB4
:10998000C0011831559800EBC00001EB0010416B8D
:10999000BDF86800C0F103008000C14001F00F0174
:1099A00030315498C0EB001000EB8000EE4A02EB1F
:1099B000C002BDF868000E301154BDF86800401CAC
:1099C00081B21A91BDF868000428D3DB03225498B1
:1099D000C0EB001000EB8000E34901EBC000827493
:1099E0005498C0EB001000EB800001EBC000401C5D
:1099F00012210490EFF76EFD01465498C0EB001061
:109A000000EB8000D84A02EBC000C17414210F9112
:109A1000D7E002215498C0EB001000EB8000D24A3E
:109A200002F830109DF854004030C1B25498C0EB99
:109A3000001000EB800002EBC000417041215498FF
:109A4000C0EB001000EB800002EBC00081703221FF
:109A50005498C0EB001000EB800002EBC000C17016
:109A600031215498C0EB001000EB800002EBC000E5
:109A7000017132215498C0EB001000EB800002EB22
:109A8000C00041715498C0EB001000EB800002EB65
:109A9000C000817100211A9127E040F223115498EF
:109AA0004843B04901EBC0011831559800EBC000A4
:109AB00001EB0010416BBDF86800C0F103008000AD
:109AC000C14001F00F0130315498C0EB001000EBA1
:109AD0008000A54A02EBC002BDF86800C01D115409
:109AE000BDF86800401C81B21A91BDF868000428D6
:109AF000D3DB00201A9011E030215498C0EB001005
:109B000000EB8000984A02EBC002BDF868000B3001
:109B10001154BDF86800401C81B21A91BDF868006C
:109B20001928E9DB03225498C0EB001000EB8000F9
:109B30008D4901EBC00080F824205498C0EB001040
:109B400000EB800001EBC000401C24210490EFF7E3
:109B5000C1FC01465498C0EB001000EB8000824A23
:109B600002EBC00080F8251026210F9129E010217A
:109B70005498C0EB001000EB80007B4A02F83010D4
:109B800030215498C0EB001000EB800002EBC000C5
:109B9000417002210F9114E010215498C0EB001085
:109BA00000EB8000704A02F8301031215498C0EB6D
:109BB000001000EB800002EBC000417002210F9109
:109BC00000BF00BF04F024BB549800EB400101EB40
:109BD0000010664901EB00113031559801EB00107F
:109BE0004178159140F22311549848435D4901EBA7
:109BF000C0011831559800EBC00001EB001001784E
